:020000040000FA
:040000006FD00400B9
:101000006F00507B000000000000000090200020D6
:10101000AA220020A9BDF9F56C23002000000000E1
:10102000000000006C230020902000200000000041
:101030000000000090200020000000009020002010
:101040000000000090200020902000209020002030
:101050009020002090200020242F00205E240020DB
:101060000000000090200020902000200424002098
:1010700090200020D22300209020002090200020EB
:101080009020002090200020902000209020002020
:101090009020002001A04111B7170040985F3AC688
:1010A000945F3247E39CE6FE3245410182800111A4
:1010B00013078008F337078093F787083EC20100C3
:1010C0000100B7170040930570052380B70413068D
:1010D00080FA2380C7040100010083C6B70493F699
:1010E000F60DA385D704238007049246F3A6068055
:1010F0000100010093760502D5CEF336078093F602
:10110000860836C4010001002380B7042380C70489
:1011100001000100B70614007D89558D88C70100C4
:1011200001000100010023800704A246F3A6068007
:101130000100010073370780137787083AC6010062
:1011400001002380B7042380C704010001000100CF
:1011500001003727004093061005A303D7802380A2
:101160000704B247F3A70780010001009307800836
:10117000F3B7078093F787083ECE01000100B71749
:101180000040130770052380E704130780FA2380CB
:10119000E7040100010003C7B70413670708A3852C
:1011A000E70423800704F247F3A70780010001004A
:1011B0000561828093760504BDC6F336078093F6F9
:1011C000860836C8010001002380B7042380C704C5
:1011D00001000100B7061400938606047D89558D31
:1011E00088C7010001000100010023800704C246F6
:1011F000F3A6068001000100733707801377870884
:101200003ACA010001002380B7042380C70401000B
:1012100001003727004093062005A303D7802380D1
:101220000704D24781B773370780137787083ACC12
:10123000010001002380B7042380C70401000100DE
:1012400098471367070C98C723800704E24719BF24
:101250000111814601468145114506CE97000000E7
:10126000E780005593078008F3B7078093F7870856
:101270003EC601000100B717004013077005238028
:10128000E704130780FA2380E7040100010003C785
:101290006704136717002383E70423800704B2471A
:1012A000F3A7078001000100F2400561828041112F
:1012B000814601468145114597000000E780404F77
:1012C00013078008F337078093F787083EC40100AF
:1012D0000100B7170040130670052380C70493066A
:1012E00080FA2380D70401000100FD552396B70240
:1012F00023800704A245F3A5058001000100733790
:101300000780137787083AC6010001002380C704CD
:101310002380D7040100010003C767041367170087
:101320002383E70423800704B247F3A70780010063
:10133000010001A0BD473305F50201007D1575FDD3
:101340008280411122C426C206C6AA8401446317C2
:101350009400B24022449244410182800504130566
:10136000803E420497000000E78000FD4180C5B741
:101370009305000273A04580824573901534924016
:101380002242B2424243D2436244F2440255925551
:101390002256B2564257D2576258F25806499649D9
:1013A000264AB64A464BD64B664CF64C065D965DD1
:1013B000265EB65E465FD65F09617300203041113C
:1013C000B7170040985F3AC6945F3247E39CE6FE49
:1013D000324541018280B71700401307000323887C
:1013E000E702854717170000232EF74273002030CD
:1013F000411122C406C637040020976000E0E78050
:10140000E0E41C408297D5BF373700408347470050
:101410009146BD8B6389D70099466394D700834773
:101420005740730020309736000083C6662C9387A0
:10143000160017360000230DF62A0347870097375A
:1014400000009387E71AB6972380E700B7E7040008
:10145000BC4F0946894517150000034565F482977E
:10146000C9B7B787004003C76700098B6309071036
:1014700003C777009306000313770703630DD708AC
:10148000173800000348586217360000130606613B
:101490000547B30606012380E60083C577001737AA
:1014A000000013072760429793F5F50F2300B7005C
:1014B00003C58700973500009385855EC295137537
:1014C000F50F2380A5000347070089451377F7032D
:1014D000630CB70C63E7E50A6306071A8545630CDE
:1014E000B7129737000083C7375C3307F60003470E
:1014F00007001377F70F19CB850793F7F70F0D4701
:101500006363F71A17370000A300F75AB787004044
:1015100009472383E700B787004083C77700E207C6
:10152000E18763DE07049737000083C7F757173753
:1015300000001307A7563E9785462300D7001737AC
:101540000000130727563E97930600032300D70099
:10155000173700001307C7543E97A146850723009D
:10156000D70093F7F70F0D476364F71417370000A0
:10157000A30CF752B787004009472383E7007300A5
:101580002030930610026300D70E930620026305F5
:10159000D70693060002E316D7F403C72702137792
:1015A000C70F13672700D5A803C767001377070481
:1015B00065CB03C7A702173800001308A82F1735FB
:1015C00000001305E526134707082385E70203C734
:1015D000A7021377370F136787002385E702814738
:1015E00013070004B305F5008C41B306F80091071A
:1015F0008CC2E399E7FEF5B503C7A70213470704BA
:101600002385E70203C7A7021377C70F13672700D5
:101610002385E702F9B503C767001377070449C3B9
:1016200003C76702173800001308881C173500002D
:101630001305C513134707082383E70203C767028F
:101640001377370F136787002383E7028147130758
:101650000004B305F5008C41B306F80091078CC275
:10166000E399E7FEBDBD03C7670213470704238361
:10167000E70203C767021377C70F136727002383A7
:10168000E70285B503C767001377070411CB03C7CB
:1016900027021377370F136787002381E70291B57D
:1016A000238006003DBD97370000A38F073EB9BDDC
:1016B00097370000A38A073E75BD230304801547B2
:1016C0002303E48001002302A480828083076480D6
:1016D000E3CE07FE23030480828083076480E3CE89
:1016E00007FE03454480828083076480E3CE07FEC3
:1016F0002302A4808280411126C44AC24EC006C67D
:101700001377F50BAD47AA892E899544630CF70032
:10171000194597000000E78080FA97000000E780F5
:1017200020FB8D444E8597000000E78040F9FD596D
:10173000FD1463983401B240A24412498249410128
:101740008280135509011375F50F97000000E7809B
:10175000E0F92209F1BF011126CC06CEB70408003A
:1017600097000000E780C0F6154597000000E7806D
:1017700000F597000000E78080F697000000E78002
:1017800000F62AC697000000E78080F43245937780
:10179000150089EB136515001375F50FF240E2444F
:1017A00005618280FD14E9F00145CDBF397126DC69
:1017B0004ADA4ED852D656D45AD25ED006DE62CE1F
:1017C00066CCB7E700E07D5783AA070022C603AACC
:1017D000470023A0E71823A2E718B7170040130714
:1017E00070052380E704130780FA2380E70483C78A
:1017F0004704930B75FFB684E20793FBFB0F854606
:10180000AA892E8B328937240040E187015763FA79
:1018100076016308D5008946130700026313D500DB
:101820000157D98F93F7F70FB71C00402382FC04B0
:1018300011472303E4801305F00F97000000E780B1
:1018400000E8094C97000000E78080E863657C159C
:10185000B7050700DA9537870700795563FEE50479
:10186000B3879500636AF704370B0800A94733EB89
:1018700065016395F90881E8814497000000E780DD
:1018800020E5268515A8DA85094597000000E78040
:10189000C0E605090345F9FFFD14050B970000009C
:1018A000E780C0E481C49377FB0FE5F79700000061
:1018B000E780A0EA69F17D55B7170040130770056E
:1018C0002380E704130780FA2380E70403C7470453
:1018D000418B2382E704F250B7E700E023A05711C1
:1018E00023A24711E25432445259C259325AA25AE1
:1018F000125B825B724CE24C21618280A547639B44
:10190000F90685691309F00FB3069900B3742B012A
:10191000B6941349F9FFB3749900856B3379690163
:10192000416B9387F9FFB3F7270199E363FC340117
:1019300093D94900C147E3E637FF3DBF0569C16957
:101940007D19D9B71305800D63886901130500025D
:101950006384790113051008CA8597000000E780A9
:10196000C0D997000000E78040DF31D54E99B3849D
:1019700034416DBFDA852D4597000000E780E0D740
:10198000CA94E30B99EE050997000000E78020D583
:10199000A30FA9FEFDB79387F9FF93F7F70F636DC8
:1019A000FC0C83C71C04130730086315F7063707C0
:1019B00008006361EB06B3079B00B706100063FBEA
:1019C000D704334BEB0089476399F9068980D549E1
:1019D000E38404EADA85094597000000E780E0D156
:1019E00011090327C9FF91472320E480030764807E
:1019F000E34E07FE23033481FD17EDFBFD14110BAD
:101A000081C49377FB0FE9FF97000000E780E0D4E3
:101A100061F155B5B717004003C75704B707080071
:101A20001377070219E3B78707007955E376FBE8D8
:101A300033079B00E3F9E7F841B58547E380F9F008
:101A4000DA852D4597000000E78020CB9389F4FFCD
:101A5000E38404E297000000E78060C893F7390050
:101A600091EB832604800327090093074900E3963E
:101A7000E6E03E89CE84D9BFB5476399F9001305E6
:101A8000900B97000000E78080C3FDB3B1471305BA
:101A9000B00AE388F9FE99476397F904B70508008F
:101AA000B365BB002D4597000000E78000C5814469
:101AB0008D4BA14997000000E78060C263967401D6
:101AC000832704802320F9008504E39534FF8327CE
:101AD000048013172B01635507002312F90069BB1B
:101AE0002322F90051BB9D47639FF90281451305ED
:101AF000B00497000000E78040C0BD4423200900E7
:101B000023220900FD5997000000E78040BD93F7AC
:101B10007400CA9703C70700FD14398D2380A700FE
:101B2000E39334FF91BBA1476397F9069700000048
:101B3000E780A0C28144630D0B008D479304C0036E
:101B40006308FB009304000563048B0193044004C5
:101B50001375C507E30295D2194597000000E78089
:101B600000B697000000E780A0B60545970000008A
:101B7000E780E0B4268597000000E78020B709459C
:101B800097000000E78080B697000000E780E0BC87
:101B9000E31405CE0DB39147639FF900130560066A
:101BA00097000000E780A0B197000000E78040B2F6
:101BB00013059009F9B5E38109CCF1547DB9BD66EF
:101BC0000147173600001306660B938606A6854567
:101BD0008347060093F7F70F91C382800507E3F967
:101BE000E6FE97370000238BB708DDB77D16620647
:101BF000618693178601E18763D4070001458280DF
:101C0000931726003307F500AE9718439C4363E70C
:101C1000E7007D16E37FF7FC7D55828005458280D5
:101C2000FD15E205E18513978501618793F7F50FAF
:101C300063480700FD15139725002A97584365D779
:101C4000138517006205618582803308B5021C4246
:101C500083A80600B335B502C29733B50701AE9825
:101C6000469585486367B5006394A50063E3070163
:101C700081480C43C6950CC388C21CC28280814730
:101C80001397870161876343B7008280139727000A
:101C90002A97232007008507E5B7814701479396D8
:101CA0008701E18663C5B6001335170082809396DD
:101CB0002700AA9694428507558FD5B793D75540EC
:101CC0008A07AA979C4305453315B5007D8D828010
:101CD00017F3FFDFE702A33D2A8497000000E780A7
:101CE00060F405C5931725003E940327C4FF814780
:101CF00011EB7D1516053E954205418517F3FFDF73
:101D00006700233D05838507E5B70145C5BF8147CA
:101D10001397870161876343C70082801397270069
:101D2000B386E50094422A97850714C3D5B77D167C
:101D300062066186014793178601E18763D5070034
:101D400013351700828093172600B306F500AE976F
:101D500094429C437D16B58F5D8FF1BF8A05AA958D
:101D600001476363B500828083A6C5FFF11593D751
:101D70001600D98F9CC11397F601E5B72A83014855
:101D8000014701456343D7008280B387050183A8DB
:101D90000700B30706019C43C697AA976384F8001F
:101DA00033B517010507B3080301620723A0F80044
:101DB00061871108C1BF2A8301478147014563C379
:101DC000D70082803388E50083280800330EE600C0
:101DD000032E0E003388A8403308C84163840801ED
:101DE00033B508018507B308E300E20723A0080123
:101DF000E1871107E9B717F3FFDFE702432B011172
:101E0000B286B2842E86AA850A8597000000E780F4
:101E1000C0FA2A84A6850A8597000000E78020E89A
:101E200033348000060413351500018D056117F366
:101E3000FFDF6700032A17F3FFDFE702C324411126
:101E4000AA89AE8A328BB68402C202C402C6014499
:101E5000131C8401135C8C4163499C02939B140006
:101E6000FD1B0549138CF4FFF15C33048901620406
:101E700061846340740792478E04CE9423AEF4FECF
:101E8000410117F3FFDF6700832313192400B30B0D
:101E90002B01014A93172A00D69783A50B0088438C
:101EA00078003400500097000000E78040DA050A0F
:101EB00093178A01E187F11BE35EFCFC92474E9980
:101EC00005042320F900A2473EC2B24702C63EC421
:101ED00041B7131A8901135A8A41131D240093171D
:101EE0008A01E18763CF970092470A044E941CC091
:101EF000A24705091379F90F3EC2B24702C63EC494
:101F0000ADB7B3079A0313152A0056950841780018
:101F100034005000050AEA97DA978C4397000000D6
:101F2000E780E0D26DBF0000197106C212C416C668
:101F30001AC81ECA22CC26CE2AD02ED232D436D6E9
:101F40003AD83EDA42DC46DECAC0CEC2D2C4D6C6D9
:101F5000DAC8DECAE2CCE6CEEAD0EED2F2D4F6D6C9
:101F6000FAD8FEDA971500009385458B8841E70083
:101F7000050092402242B2424243D2436244F244BC
:101F8000025592552256B2564257D2576258F258CD
:101F900006499649264AB64A464BD64B664CF64CFD
:101FA000065D965D265EB65E465FD65F096173008C
:101FB00020300000972100209381C1041751002098
:101FC0001301418417F5FFFF130505049705002051
:101FD00093854503171600201306C6FD63FAC50056
:101FE0008322050023A0550011059105E3EAC5FEF3
:101FF00017050200130545DC97150020938585FB26
:10200000171600201306066563FAC5008322050033
:1020100023A0550011059105E3EAC5FE1715002020
:102020001305456397450020938545116377B500F7
:10203000232005001105E36DB5FEFD42739002BC3F
:102040008D4273904280B722000093828288739001
:102050000230970200209382E2FA93E232007390FA
:102060005230975200009382E294739012346FB012
:10207000347973002030397101436EC619A039716B
:1020800041536AC866CA62CC5ECE19A03971015349
:102090005AD056D252D44ED64AD826DA22DC06DEA0
:1020A00033016140828241114AC026C222C406C661
:1020B0008282B24D4101024D924C224CB24B410101
:1020C000024B924A224AB2494101024992442244B7
:1020D000B240410182803D432A876373C3029377F4
:1020E000F700BDEFADE5937606FF3D8ABA960CC3C7
:1020F0004CC30CC74CC74107E36BD7FE11E282808B
:10210000B306C3408A069702000096966780A60031
:102110002307B700A306B7002306B700A305B7003F
:102120002305B700A304B7002304B700A303B70037
:102130002303B700A302B7002302B700A301B7002F
:102140002301B700A300B7002300B700828093F5F6
:10215000F50F93968500D58D93960501D58D61B7C2
:10216000939627009702000096968682E78086FA6B
:102170009680C1171D8F3E96E374C3F8A5B73367E9
:10218000B500FD530D8B79E7B7877F7F9387F7F70E
:1021900010419441B372F6003363F600BE92B3E28D
:1021A00062006397720C6318D6065041D441B37233
:1021B000F6003363F600BE92B3E262006398720ADF
:1021C000631BD60410459445B372F6003363F600E2
:1021D000BE92B3E262006391720A631ED60250455A
:1021E000D445B372F6003363F600BE92B3E26200E8
:1021F000639A72086311D60210499449B372F600CB
:102200003363F600BE92B3E2620063937208510535
:10221000D105E30FD6F61317060193970601631C49
:10222000F7001357060193D706013305F74093755E
:10223000F50F91E982804183C1833305F74093759F
:10224000F50F91E182801377F70F93F7F70F3305BE
:10225000F74082800346050083C605000505850515
:102260006313D60065FA3305D640828011059105C7
:10227000E312D6FE014582802105A105E31CD6FCB0
:10228000014582803105B105E316D6FC0145828007
:102290004105C105E310D6FC01458280B717004017
:1022A00003C777051377E70FA38BE704130700F83D
:1022B000A38DE7043D47238CE70413075003A38C49
:1022C000E70403C7A7051377D70F238DE7048280A0
:1022D000B717004003C7E7020D8941111377C70FF5
:1022E000498F93068008F3B6068093F6860836C6B3
:1022F00001000100930670052380D704930680FA3D
:102300002380D704010001002387E702238007040C
:10231000B247F3A70780010001004101828041110B
:102320002A83014E930E407E130F0019930F40062F
:1023300063E56E129308001913034006B378150382
:10234000854E0D4FA14F337365020D89133515006E
:1023500063EFBE121308F6FF7946729842081358CD
:1023600008013307C70213D61700BE07329761462C
:10237000B3F6C60213068070B386C6023697A1660E
:10238000F58F42075D8FB716004083C7F60293F7BB
:102390000708A303F1000346710083C7F60293F711
:1023A0000708E394C7FE83477100B716004093F710
:1023B000F70F6388071293078008F3B7078093F736
:1023C00087083EC401000100B7170040930670055E
:1023D0002380D704930680FA2380D70401000100EC
:1023E00023AA070383C6170393E60608A388D70228
:1023F00023800704A247F3A70780010001001166AC
:10240000B71700407D16D45BC85F93854703A98E3C
:10241000F18EF5FA93068008F3B6068093F68608E7
:1024200036C601000100930670052380D704930689
:1024300080FA2380D7040100010098C103C7170365
:1024400013670704A388E70223800704B247F3A7B2
:10245000078001000100410182807D133368E3039E
:102460009308E016630E08003368F3039308D01650
:10247000630808009378330093B818009388D8163F
:1024800033081E01131E0801135E0E0155B5639338
:10249000E5030548638608000148630303002A88B2
:1024A00071087298FD15131E0801C205135E0E0116
:1024B000C18179BD13F8150063F4BF007908D5B761
:1024C00013381800E5BF83C7F60293F70708A30384
:1024D000F1000346710083C7F60293F70708E394FF
:1024E000C7FE8347710093F7F70FF1DFE9B531714C
:1024F0004AD966CB06DF22DD26DB4ED752D556D32E
:102500005AD15ECF62CD6AC96EC7AA8C02D8971025
:102510000000E78020B12A8993078008F3B707807D
:1025200093F787083EDA01000100B7170040130750
:1025300070052380E704130780FA2380E704010075
:10254000010003C7F7021377770FA387E70203C7DA
:10255000F70213678700A387E70223800704D25797
:10256000F3A7078001000100054597000000E78000
:1025700060D6130780C13347E902116A93070AE85E
:1025800093065002BD69930BA004814A014B1304CA
:102590008008930470057D1AB347F9023307D70208
:1025A0003EC0FD873ECC938709A69309803E334702
:1025B000F7023AC27D873AC4334739038549B39954
:1025C000990193D93940B306D702B30B7703B3C649
:1025D000F602B3CBFB0236C6FD8636C893D6FB4166
:1025E00036CEB7460F00938606243349D902856656
:1025F000938606FAB3969601B389E90213076055EC
:102600003309D90293060010B389E9023349D9028C
:10261000B3C9F9029316390036CA37190040FD864E
:1026200036D0930D090493D7F9413ED2F336048096
:1026300093F6860836DC01000100930770052380BD
:10264000FD00930680FA2380DD000100010083462F
:10265000390593F6860FA309D9048346390593E615
:102660001600A309D90423800D00E256F3A60680C4
:1026700001000100130C80FA116DF336048093F60B
:10268000860836DE01000100930770052380FD00F7
:1026900023808D010100010083463905216693E600
:1026A0000602A309D90483560905B3E6A601231837
:1026B000D90483560905D18E2318D90423800D002F
:1026C000F256F3A60680010001008346390593F611
:1026D00006026381061A03463905218A6DDE081851
:1026E00097100000E7800098733604801376860800
:1026F000B2C20100010023809D0023808D010100F2
:102700000100B717004003C637051376F60DA389FD
:10271000C70403C6370513660602A389C704835698
:1027200009052166B3E6A6012318D90483560905D5
:10273000D18E2318D90423800D009646F3A6068077
:10274000010001008346390593F60602638B0614E7
:1027500083463905A18AEDFE97000020E780A0930B
:10276000AA8636D497000020E780E092A256E30ABA
:10277000D5FE835609054255B3E6A6012318D904B0
:1027800097100000E780C08F83463905A18AEDDEEF
:10279000035609058346290582473376CA00B306E6
:1027A000DA0293D5F641B296B388F640E24733B8E1
:1027B000C6002E983308F840A247B3B61601330876
:1027C000D84063C70701631DF800924763FA1701F9
:1027D000C247634FF80E63950701B24763EAF80EEC
:1027E000894663E9660FF2469315180013D3F80182
:1027F0005E8613951800B365B30042D646D497B0F1
:102800000100E780E07E3258050B137BFB0F634726
:102810000001631A0838A2586387083813081500A6
:10282000B336A800B69513D6F5013298B336C80072
:10283000AE9613581800FE06B3E606017336048000
:1028400013768608B2C60100010023809D00238014
:102850008D01010001000356C902B296C206C18271
:102860002316D90223800D00B646F3A60680010088
:10287000010021B5F336048093F68608B6C0010046
:10288000010023809D0023808D010100010083460B
:10289000390593E60602A309D90423800D00864674
:1028A0000DB5F336048093F68608B6C40100010026
:1028B00023809D0023808D0101000100834639059E
:1028C00093E60602A309D90423800D00A646BDB5F0
:1028D000E30B0BF0F336048093F68608B6C80100CC
:1028E0000100930680FA23809D002380DD00010013
:1028F00001008346390593F5FC0F93F6860FA30973
:10290000D90483463905CD8EA309D90423800D004F
:10291000C646F3A6068001000100130580FA0346AF
:102920003905930639051D8A631C96297336048080
:1029300013768608B2CC01000100130680FA2380CA
:102940009D002380CD000100010003C60600137620
:10295000F60D2380C60003C6060013660602238018
:10296000C600835609051166D18E2318D9048356F3
:1029700009052166D18E2318D90423800D00E6466F
:10298000F3A6068001000100130680FA834639058C
:1029900093F606026380062683463905130C390533
:1029A000A18AFDDA081897000000E780A06BF336D3
:1029B000048093F68608B6D001000100930680FAE1
:1029C00023809D002380DD000100010083460C0070
:1029D000116693F6F60D2300DC0083460C0093E6A7
:1029E00006022300DC0083560905D18E2318D90482
:1029F000835609052166D18E2318D90423800D0042
:102A00008656F3A6068001000100130680FA83466D
:102A1000390593F60602638A062083463905A18AA2
:102A2000EDFE97F0FF1FE78000672A8C97F0FF1FED
:102A3000E7806066E30C85FF835609051166425501
:102A4000D18E2318D90497000000E7806063834685
:102A5000390513063905A18AFDDAF336048093F6A9
:102A60008608B6D401000100930680FA23809D00F9
:102A70002380DD00010001008346060093F6F60D79
:102A80002300D60023800D00A656F3A60680010081
:102A900001008356090503462905D247B376DA00BB
:102AA0003306CA021305800C9355F6413696330D52
:102AB000F6408257333CD6002E9C3336A601330CA9
:102AC000FC40330CCC403308850392564E86B33518
:102AD000A5033305A503C29597B00100E7804051D7
:102AE00063468001631E0C16630C0D161306150059
:102AF0003335A6002E959356F5013696B335D6009C
:102B0000AA959396F50105828585D18E6346B0001E
:102B1000639D051A638B061A0356C9021582330595
:102B2000D6003336C500B2956348B00063910524E2
:102B30001306F00F637DA622894663F356159307AB
:102B40008008F3B7078093F78708BED6010001001D
:102B500037170040930770052300F704930780FAA6
:102B60002300F704010001008356C702896781171B
:102B7000D58FC207C1832316F70223000704B65777
:102B8000F3A7078001000100FA506A54DA544A5949
:102B9000BA592A5A9A5A0A5BFA4B6A4CDA4C4A4D8D
:102BA000BA4D296182801308F5FF3335A800FD1561
:102BB0002E951356F5013298B336C800AA9695B9EA
:102BC000F336048093F68608B6CA0100010023801C
:102BD0009D002380AD000100010083463905CD8EA4
:102BE000A309D90423800D00D646F3A60680010070
:102BF000010035B3F336048093F68608B6CE0100A3
:102C0000010023809D002380CD0001000100834648
:102C1000390593E60602A309D90423800D00F64680
:102C2000F3A606800100010095B3F336048093F605
:102C30008608B6D20100010023809D002380CD00CC
:102C4000010001008346390593E60602A309D90471
:102C500023800D009656F3A606800100010045BBB7
:102C60009306F5FF33B5A600FD152E959355F50196
:102C7000AE96B3B5B600AA951396F501858269B5EF
:102C8000F336048093F68608B6D801000100930657
:102C900080FA23809D002380DD000100010083561F
:102CA000C9020566011693F6F60FD18EC206C182DF
:102CB0002316D90223800D00C656F3A60680010014
:102CC0000100850A93FAFA0F95B233E6B60045C2C1
:102CD0000356C9023305D0403338A000B305B040D5
:102CE000B385054115826345B000D1E16371A60843
:102CF000894663F0560593078008F3B7078093F77A
:102D00008708BEDA01000100B717004013077005FD
:102D10002380E704130780FA2380E7040100010001
:102D200003D7C7027D8B2396E70223800704D6577B
:102D300081BDF336048093F68608B6DC01000100FD
:102D4000930680FA23809D002380DD0001000100AE
:102D50008356C9020566011693F6F60FD18EC20698
:102D6000C1822316D90223800D00E656B9B7930716
:102D70008008F3B7078093F78708BEDE01000100E3
:102D800037170040930770052300F704930780FA74
:102D90002300F704010001000356C7029397560071
:102DA000B297C207C1832316F70223000704F65720
:102DB000C1BB914763EEB70217D701001307C70ED7
:102DC0008A05BA959C41BA978287B717004003A736
:102DD000470B1345F5FF698F23AAE70A03A7070BE3
:102DE000698F23A8E70A03A7070A798D23A0A70AFA
:102DF0008280B717004083A6470B1347F5FFF98E73
:102E000023AAD70A83A6070B558D23A8A70A83A652
:102E1000070A758F23A0E70A8280B717004003A72F
:102E2000470B498F23AAE70A03A7070B1345F5FFB2
:102E300045BFB717004083A6470B1347F5FF758FB3
:102E400023AAE70A03A7070A598D4DB7B717004011
:102E500003A7470B498FEDB7914763EEB70217D72A
:102E600001001307A7058A05BA959C41BA97828786
:102E7000B717004003A7470D1345F5FF698F23AA35
:102E8000E70C03A7070D698F23A8E70C03A7070C1E
:102E9000798D23A0A70C8280B717004083A6470D29
:102EA0001347F5FFF98E23AAD70C83A6070D558D7E
:102EB00023A8A70C83A6070C758F23A0E70C82809C
:102EC000B717004003A7470D498F23AAE70C03A7B4
:102ED000070D1345F5FF45BFB717004083A6470D03
:102EE0001347F5FF758F23AAE70C03A7070C598D2D
:102EF0004DB7B717004003A7470D498FEDB779715C
:102F000022D43714004026D24AD0035924028354D5
:102F1000040206D64209C2044ECE52CC56CA1359F8
:102F20000901C1802DE11379F9F793F4F49F420967
:102F3000C20413590901C18093078008F3B70780C1
:102F400093F787083EC40100010093077005230032
:102F5000F404930780FA2300F40401000100231114
:102F600024032310940223000404A247F3A707803C
:102F700001000100B250225492540259F249624AAF
:102F8000D24A45618280B7F5070081463000B1051D
:102F9000194597000020E7806081A2471397270119
:102FA000E34A07FC1369090893E404409309800885
:102FB000F3B7098093F787083EC001000100930A28
:102FC000700523005405130A80FA2300440501000C
:102FD00001002311240323109402230004048247D8
:102FE000F3A7078001000100294597F0FF1FE78044
:102FF0006034F3B9098093F989084EC201000100D9
:1030000023005405230044050100010083570402F6
:1030100093E707202310F402230004049247B9B772
:10302000B71700408847420541819377050491EB2B
:103030009377F5013755E801130505803345F5020F
:1030400082809377050C130700046397E70093775A
:10305000F50137459C1CCDB72165130505D082804D
:1030600037E700E01C435443A183E206D58F1CC11F
:10307000FD572320F7182322F718828013178500A5
:10308000B7E700E023A0E710618123A2A7108280A8
:10309000B7F700E08847CC47828081473737004048
:1030A000A14663C4C700328582800345B740E38EE2
:1030B000A6FE3385F5000345050085072304A740D8
:1030C000CDB7970700209387E7EE9C431737002082
:1030D0001307C7063E95636EE500173700201307F8
:1030E00067526368A700170700202325A7EC3E85D9
:1030F0008280FD57EDBF8280411122C406C62A841A
:1031000097000000E78000F22947B307E502B240CC
:103110008D83B3D7870222449507B3D7E7023737A9
:103120000040C207C1832316F7004101828041118C
:1031300037150E0006C697000000E78020FCB73761
:103140000040130770F82381E7000D47A381E700D3
:1031500013070004A380E70005472387E700B24078
:103160004101828037370040834727001A0593F7D3
:10317000F703C98F93F7F70F2301F7008280B73762
:10318000004003C7170019C9D98DA380B70003C732
:103190000700136787002380E700828093C5F5FF4F
:1031A000F98DA380B7008280AE872A87B7360040AA
:1031B00021463738004089E7170300006700E3F332
:1031C00083C8B600E30916FF05078348F7FFFD171C
:1031D000C20723041801C183F9BF411122C406C6E6
:1031E0002A8497000000E780E0E32947B307E5025F
:1031F000B2408D83B3D7870222449507B3D7E70245
:1032000037370040C207C1832316F740410182804F
:10321000716541111305052006C697000000E7807F
:1032200000FCB7370040130770F82381E7400D47D3
:10323000A381E74013070004A380E74005472387E5
:10324000E740B24041018280CC41411106C632853F
:1032500003C6150083C5050022064D8E42068D6506
:103260004186138875A2630C0611634BC80413884A
:1032700045A26300060D634AC800938535A2630129
:10328000B6082390060029464DA0138855A2630571
:10329000060D938565A2E316B6FE8D451D4663E6D1
:1032A000E5081146198E63F3C7003E86B7E70400B0
:1032B0002390C600FC4797D50100938565C29DA069
:1032C000138895A263030611634E060D1388A5A209
:1032D00063000613938505A5E315B6FA99451D46C7
:1032E00063E5E504198E63F3C7003E86B7E7040083
:1032F0002390C600FC47970500209385E5D51DA0C7
:103300009D451D4663E3E5022146198E63F3C70020
:103310003E86B7E70400FC472390C60097050020CF
:103320009385C533BA9582970146B24032854101F3
:103330008280AD451D46E3EAE5FE3146198E63F312
:10334000C7003E86B7E704002390C600FC4797D528
:103350000100938565BBF9B7B1451D46E3E7E5FC80
:103360003546198E63F3C7003E86B7E70400239005
:10337000C600FC4797D50100938505BA65B78D4512
:103380001D46E3E4E5FA1146198E63F3C7003E8655
:10339000B7E704002390C600FC4797D5010093854A
:1033A000E5B449B78D451D46E3E1E5F81146198EB0
:1033B00063F3C7003E86B7E704002390C600FC47CE
:1033C00097D50100938505B7B1BFA5451D46E3EE2E
:1033D000E5F42946198E63F3C7003E86B7E704007B
:1033E0002390C600FC4797D501009385E5B01DBF2B
:1033F000B5451D46E3EBE5F23946198E63F3C70088
:103400003E86B7E704002390C600FC4797D501002D
:10341000938505AC01BFB7E7040003A30713970624
:103420000020938666C24146A54517050020130576
:10343000A5B802832D455DE703C505000947631F55
:10344000E50803A84500411106C603471800328568
:103450000346080022074168518F930828FE63073E
:10346000170563E9E80005186303070323900600C6
:10347000294591A8130648FE630AC7041518E317E7
:1034800007FF15463E87637BF600154701A8130624
:1034900000023E876374F60013070002B7E70400DA
:1034A0002390E600FC471316070111A83E8691C33E
:1034B0000546B7E70400FC472390C6004206CC450A
:1034C000418282970145B240410182801306000883
:1034D0003E87E375F6FC13070008C9B72390060082
:1034E000054582808280416779176304E5044111B4
:1034F00022C406C685472A84639FF500B7E7040007
:1035000022852244B24003A38713970500209385A8
:10351000252F4101028389476399F500B7E704002D
:1035200083A7070B8545829771D9B2402244410198
:1035300082808280797122D452CC2E842A8A97D5B7
:103540000100938525A117D50100130525A306D6F3
:103550003AC626D24AD0B68432894ECE97B0010000
:10356000E78040F4A68517D50100130525A297B082
:103570000100E78020F3294597B00100E78060F75C
:103580008347840093F70702E1E7834904008947F2
:10359000054532476396F908544083C7160083C631
:1035A0000600A207D58FC166138616FE638CC7027C
:1035B0008D16638FD7068D66938626902945639175
:1035C000D706B7E70400A285225403A34714B250DC
:1035D000F249A6864A86925402595285624A854724
:1035E000456102832D450DEF93070002354563E9E0
:1035F0009702B7E70400FC47484413060002CA8557
:103600008297814997070020938747209C43014573
:1036100081CB9C4391C74E852686CA8582970145FA
:10362000B250225492540259F249624A4561828052
:103630002D457DF79307700F3545E3E397FEB7E718
:103640000400FC4748441306700FCA8582975DBF8B
:103650002145F9B7411122C437E4040083278413BC
:1036600026C2AA84416506C69705002093854519A0
:103670007D1582978327C40A170500001305E5E628
:103680008588829795C0032304132244B240924454
:10369000970600209386C6AD4146C5451705002014
:1036A0001305059C41010283B24022449244014526
:1036B0004101828019C59707002023A9A71401455D
:1036C0008280454582801147636AA70A97D6010028
:1036D000938606870A0536951841411106C6369726
:1036E000AE87B2850287130700026145639DE7003C
:1036F000B7E70400FC471306000217050020130576
:1037000065F682970145B2404101828005476145D7
:10371000E39BE7FEB7E70400FC47054617050020DA
:10372000130545F6F9BF1307700F6145E39DE7FCEC
:10373000B7E70400FC471306700F170500201305B8
:10374000A5F4C1B7130700086145E39EE7FAB7E7A0
:103750000400FC4713060008170500201305450266
:103760004DB715476145E390E7FAB7E70400FC471A
:103770001546170500201305E50861B70945828045
:10378000411126C2B7E4040083A7C41322C44AC06F
:1037900006C62E8497050020938585062A89829780
:1037A000058905C5970700209387878B83D7A70BCB
:1037B000A28503A3440D2310F4002244B240924496
:1037C0004A850249014641010283B24022449244A3
:1037D000024949454101828097070020238A070258
:1037E0009707002023A80702B717004003A7070C7C
:1037F000B706C0FFFD16758F23A0E70C03A7070DC2
:10380000B7064000558F23A8E70C03A7070C3D9B84
:1038100023A0E70C03A7070D1367070123A8E70CF4
:103820008280B717004003A5470C83A7470C598136
:1038300013451500C18B058999E31365250097078A
:10384000002083C7E7FC6380A7029707002023813D
:10385000A7FC11C9970700209387C7FB03A30700A4
:103860006303030002838280114517F3FFFF6700A3
:1038700043C8411193962500AA852D4506C697F0A9
:10388000FF1FE780A0F2B240014541018280011193
:1038900022CC06CE3714004026CA4AC84EC652C4AF
:1038A00083447405034AB405834984050349940598
:1038B00097F0FFFFE780C09E8347A40593F4F40FC1
:1038C000137AFA0F93E71700230DF40493F9F90F15
:1038D0001379F90FB717004003C7A705058B6DFFD4
:1038E00003D5C705A38D4705238C3705A38C270572
:1038F000A38B9704F2406244D2444249B249224A1F
:103900000561828041119397050122C406C626C233
:10391000C1872E8463DC0700B7E40400FC5482975F
:1039200019C1BC5482972165218D15A893F7150004
:1039300013C515008DE793F725009DC7970000007C
:10394000E78060EEB7E70400BC4F1306000A894524
:1039500017050020034585EC829713452400B240EB
:1039600022449244410182809397250163D8070243
:10397000B7E4040083A7C41E829797000000E78085
:10398000E0EEBC4C37560700130606308965170574
:1039900000200345A5E88297096579B7939715013B
:1039A0000145E3DE07FA17C501001305256697B048
:1039B0000100E78000C7B7E70400BC4F13060064AE
:1039C000916517050020034565E582971165A9BF3C
:1039D0002D71232A9110FD74E98C232C811023284A
:1039E0002111232631112A84AE89328993060010D1
:1039F0000A86A6852D45232E111097F0FF1FE7801C
:103A0000E0DA13154401B7E70400FC4751810A05C9
:103A100013962900CA850A958297A6858566014670
:103A2000254597F0FF1FE78060D80A86A685930694
:103A30000010294597F0FF1FE78040D78320C11170
:103A40000324811183244111032901118329C11009
:103A500015618280B7F7070003C70701411106C649
:103A600022C426C24AC0A547631DF7009700000084
:103A7000E78040F6B24022449244024901454101A8
:103A8000828013942500AA843289A286AA850146E1
:103A9000254597F0FF1FE78060D1A2864A86A6855C
:103AA000294597F0FF1FE78060D0E9B71D71A2CCD0
:103AB00037E404005C5C485886CE494697C501004F
:103AC00093854550829711E917C501001305C5502C
:103AD00097B00100E780E0B401A0B7F600E07957A5
:103AE00098CAFD57DCCA0567B7E700E023A0E710D6
:103AF0001306F00290C223A0E71801000100370767
:103B0000002018471306000481459706002023A5CE
:103B1000E6D04157A38AE7403C44080882979707BC
:103B200000209387676C3EC8856713870740231A78
:103B3000E1001D673ACC37070105130707103ACE9D
:103B4000938757D11307B00F2310E1022312F1021C
:103B5000054797F7FFFF9387E7532301E1023ED81C
:103B600017070000130727D197070000938767D234
:103B7000B7F50700BAC23EDC170700001307C7ED10
:103B800097070000938787CE81463000E1051945ED
:103B9000BAC43EDE97F0FF1FE78040C11808814796
:103BA000994630003E960346060085070507A30B9D
:103BB000C700E398D7FEC24791C703574101856705
:103BC0006373F70001A0B7E7040083A7470A08085A
:103BD0008297AA8511C917C501001305254197B021
:103BE0000100E780208C01A0F640664425618280B8
:103BF000411126C2B7E4040083A7040806C622C404
:103C000017050000130545D0829717040020130400
:103C1000E4C02300A40097000000E7808002970022
:103C20000000E780A0BB03450400224403A38405F1
:103C3000B2409244130600328965410102837971D2
:103C400006D622D413078008F337078093F7870836
:103C50003EC201000100B7170040930570052380A4
:103C6000B704130680FA2380C7040100010083C64D
:103C7000F70293F6A60FA387D70223800704924684
:103C8000F3A60680010001007337078013778708C9
:103C90003AC4010001002380B7042380C704010057
:103CA000010003C7F70213672700A387E7022380F9
:103CB0000704A247F3A7078001000100054597E02C
:103CC000FFFFE780206197000000E78020BA0147EE
:103CD00081468147054685451305407E97E0FFFFF5
:103CE000E780206437E404003C4468005146814585
:103CF0008297B707C0A83EC8B787E803938707D065
:103D00003ECA97E7FF1F9387876B3EC67C586800C3
:103D10008297B250225445618280411197D50100AB
:103D20009385059517C501001305452506C697A07F
:103D30000100E780207717D50100130525AC97A077
:103D40000100E7802076B2402945410117A3010018
:103D50006700237A411197D501009385A59217C575
:103D600001001305A52106C697A00100E780807316
:103D700017D50100130545A797A00100E7808072C1
:103D8000B2402945410117A3010067008376411124
:103D900022C406C6834705002A849DC797D5010023
:103DA0009385059417C501001305451D97A00100D3
:103DB000E780406F4C4017D50100130565B297A00E
:103DC0000100E780206E3DA058410DEF97D501001E
:103DD0009385059117C501001305451A97A00100A9
:103DE000E780406C17D50100130505B197A00100CD
:103DF000E780406B2244B2402945410117A30100EE
:103E00006700236FA1679386D7036313D70297D503
:103E100001009385E58C17C501001305251697A0B1
:103E20000100E780206817D501001305E5AD7DBFCF
:103E3000ED0797D501009385A58A17C501001305E5
:103E4000E513631BF70097A00100E780A06517D575
:103E500001001305A5AC59BF97A00100E78080645D
:103E60004C4017D50100130565AD91BF411197D5A1
:103E700001009385658217C501001305251006C64C
:103E800097A00100E7800062B2402945410117A3D5
:103E9000010067000366797122D426D24AD02E84AD
:103EA0002A898145B2844800714606D697E0FFFF13
:103EB000E780A02297F7FF1F9387474CDC4783D703
:103EC0000700231421012313F10097500000E7801D
:103ED000A0859547A305F1009307401F3EC6FD57F7
:103EE0002305A100230AF10097500000E780009805
:103EF0002686A285480097500000E780C085B25012
:103F000022549254025945618280971700202390D1
:103F1000077E971700202389076CB7E70400BC478A
:103F2000411106C641468145170500201305451A73
:103F3000829797200000E780A05697200000E78036
:103F4000C031014597500000E780A02A17070020E4
:103F50000347071A9307F00A6315F7029307F0F86F
:103F60008945170500201305A51817070020230110
:103F7000F71897070020A38D071697500000E780D9
:103F8000E05197500000E780A05E814537050400AE
:103F90009707002023AC07129707002023960712EB
:103FA0009707002023830712970700202394070A0E
:103FB00097070020239207089707002023950710F2
:103FC00097070020239E071097300000E78040CE1F
:103FD000014597500000E780605597C50100938523
:103FE000256E17C50100130565F997A00100E7804C
:103FF000604B17D501001305A59A97A00100E78033
:10400000604AB2402945410117A301006700634E91
:10401000411122C406C626C293F715002E84638F71
:104020000710814617F6FF1F1306863285451705D0
:1040300000200355250097C00000E78060B815C92F
:1040400097C501009385856817C50100130505F321
:1040500097A00100E780004517C501001305C509B9
:1040600097A00100E7800044294597A00100E78060
:10407000404897C501009385656517C50100130584
:10408000E5EF97A00100E780E04117C501001305A7
:10409000E50797A00100E780E040294597A00100CF
:1040A000E780204517F5FF1F1305452D5C450547A3
:1040B0002390E70097300100E780E06897C5010092
:1040C0009385C56017C50100130545EB97A0010056
:1040D000E780403D17C501001305850497A0010046
:1040E000E780403C294597A00100E7808040930786
:1040F00010F817070020230DF7FE9707002083D73D
:1041000027F317070020A305F7FE17050020130566
:1041100025FEA183914517070020230CF7FC970784
:104120000020A38807FC97500000E7802037134544
:104130001400B240224492444101828093F725004A
:10414000E1C317070020035727F845CB9706002047
:104150009386C6F7944297D7010093876786170620
:104160000020034686F6814517050020130545F615
:1041700097700000E78020C4AA8441C197C5010060
:104180009385855B17C50100130545DF97A00100E6
:10419000E7804031A68517C501001305E5F997A012
:1041A0000100E7802030294597A00100E7806034B6
:1041B00097070020239A07F0930710F817070020AD
:1041C0002308F7F29707002083D787E61707002018
:1041D000A300F7F2A18317070020230CF7F0914505
:1041E0008D47170500201305A5F017070020A3022F
:1041F000F7F097500000E780602A1345240015BFB0
:1042000093F74500D1C397C501009385E55217C5C3
:1042100001001305A5D697A00100E780A02817C5C7
:104220000100130525F397A00100E780A027294589
:1042300097A00100E780E02B930720F817070020E4
:104240002308F7EA9707002083D7C7E01707002065
:10425000A300F7EAA18317070020230CF7E885479E
:1042600017070020A307F7E897400000E7800060E9
:10427000170500201305C5E7914597500000E7801A
:10428000E0211345440075B593F78500A9C797C58C
:1042900001009385654A17C50100130525CE97A037
:1042A0000100E780202017C501001305E5EB97A06A
:1042B0000100E780201F294597A00100E7806023C7
:1042C00097070020239207E097700000E78080BEE8
:1042D00013458400B9BD93F70501D1C38545170582
:1042E0000020035525D797500100E780A07097C59F
:1042F00001009385654417C50100130525C897A0E3
:104300000100E780201A17C50100130525E797A0D3
:104310000100E7802019294597A00100E780601D72
:10432000930730F8170700202304F7DC97070020D5
:1043300083D747D217070020A30CF7DA1705002010
:10434000130505DBA1838D45170700202303F7DA4A
:1043500097500000E780801413450401D9BB93F700
:104360000502D1C797C501009385053D17C501001A
:104370001305C5C097A00100E780C01217C5010052
:10438000130505E297A00100E780C011294597A019
:104390000100E7800016930740F817070020230963
:1043A000F7D49707002083D727C917070020A30158
:1043B000F7D4A18317070020230DF7D285471707ED
:1043C0000020A308F7D297070020239707C697403D
:1043D0000000E780A04917050020130565D191452D
:1043E00097500000E780800B1345040299B393F7C0
:1043F0000504FDC397C501009385053417C5010069
:104400001305C5B797A00100E780C00917C50100D3
:10441000130585DA97A00100E780C008294597A019
:104420000100E780000D9707002083C767CC1307C2
:10443000700A6386E7061307800A638CE708130790
:10444000600A6393E704930760F8170700202301CD
:10445000F7CA9707002083D707C717070020A309CB
:10446000F7C8A183170700202305F7C8854717075A
:104470000020A304F7C8B14517050020130545C760
:1044800097500000E780800197400000E780003EE1
:104490001345040497070020239707C259B99307CF
:1044A00070F8170700202305F7C49707002083D76B
:1044B00087C117070020A30DF7C2A18317070020AB
:1044C0002309F7C2854717070020A305F7C29945BE
:1044D00065B7930780F8F1B793F705080145E38ABC
:1044E00007C497C501009385252517C5010013054D
:1044F000E5A897A00100E780E0FA17C501001305C1
:1045000025CD97A00100E780E0F9294597A001009B
:10451000E78020FE9307A0F817070020230AF7BCC6
:104520009707002083D7C7BB17070020A302F7BC5B
:10453000A18317070020230EF7BA8547170700202D
:10454000A309F7BA97070020239C07B897400000FB
:10455000E780C03117050020130585B991459750B4
:104560000000E780A0F313450408E1B6411122C41E
:1045700097C50100938505182A8417C50100130506
:10458000E59F06C697A00100E780C0F14C4017C523
:1045900001001305653297A00100E780A0F02945CE
:1045A00097A00100E780E0F4034704009307F00FB1
:1045B000631FF70297C501009385C51317C5010056
:1045C0001305C59B97A00100E780C0ED4C4017C5BF
:1045D00001001305652F97A00100E780A0EC22449D
:1045E000B2402945410117A30100670083F0B240A2
:1045F000224441018280B1C1411122C417C501008A
:104600001305C5972E8497C501009385A50906C695
:1046100097A00100E78000E9A28517C501001305F6
:10462000E53597A00100E780E0E72244B240294544
:10463000410117A301006700C3EB8280411122C42E
:1046400026C22E84AA8497C501009385650617C5E6
:1046500001001305A59206C697A00100E78080E43B
:1046600017C501001305453297A00100E78080E3DC
:10467000294597A00100E780C0E797C50100938511
:104680002503970700202397979A17C50100130564
:10469000E58E854497070020239C87989707002084
:1046A00023999798971700202393870497A00100D8
:1046B000E78040DF9715002083D5650317C501000B
:1046C0001305052D97A00100E780C0DD294597A0BF
:1046D0000100E78000E297170020238797F09720DA
:1046E0000000E78080B7228597500000E78060B027
:1046F000054597500000E78060E397F7FF1F938719
:10470000E7C7DC4703D70700C167FD176312F7024D
:104710002244B7E70400B240924403A3870517F58B
:10472000FF1F034525101306000A8545410102833A
:10473000B2402244924441018280011122CC37E4EC
:1047400004005C5C06CE354697C501009385450C98
:1047500017D50100130505CC829711E917C5010093
:104760001305858797A00100E780A0EB01A097F7CC
:10477000FF1F9387E70B3EC4B7F507008567938754
:104780000780814617F6FF1F1306060AE105194543
:104790003EC697E0FF1FE78060017C44194697F50D
:1047A000FF1F93856508170500201305E58A82978A
:1047B000340017F6FF1F1306260797C501009385DF
:1047C000655617C501001305655797600000E7801F
:1047D00080332A841DCD97C501009385E5F417B574
:1047E00001001305A57997A00100E780A0CBA28561
:1047F00017C501001305C50297A00100E78080CA14
:10480000294597A00100E780C0CEF24062440561CF
:10481000828097E00000E780E09517C5010013054E
:1048200025F797500000E780C02797A00000E78099
:1048300020EA97500100E780A04E17F5FF1F1305EF
:1048400065B097500100E780403717C50100130598
:1048500025F597500100E780204F2A8497600000DB
:10486000E780008E97000100E78080269780010096
:10487000E780A0BF97700000E78040E697600000E7
:10488000E780000497300100E780E0E797C501006A
:10489000938585E917B501001305456E19C897A0E2
:1048A0000100E78020C0A28517C50100130585F926
:1048B000A1B797A00100E780E0BE17C5010013056E
:1048C000A5FA97A00100E780E0BD294597A0010067
:1048D000E78020C297300100E780C0C397F0000056
:1048E000E78080E255C98545370504009720000020
:1048F000E780003C97C50100938505E317B50100EB
:104900001305C56797A00100E780C0B917C501006E
:10491000130505F797A00100E780C0B8294597A0C7
:104920000100E78000BD97F7FF1F9387E79483D7C7
:10493000070017170020231CF7DA854717170020F8
:104940002304F7CA97200000E78000B097200000FA
:10495000E780A09017150020035565D997500000F7
:10496000E7802089054597500000E78020BC97C567
:104970000100938565DB17B501001305256097A03D
:104980000100E78020B217C501001305A5F197A02B
:104990000100E78020B1ADB597C501009385C5D86A
:1049A00017B501001305855D97A00100E78080AF72
:1049B00017C501001305C5FE97A00100E78080AE72
:1049C000294597A00100E780C0B2014569BF4111A8
:1049D00022C437E404008327041A06C6829797503E
:1049E0000000E780C0848327040817F5FFFF130544
:1049F0006562829797F7FF1F2386A7E217F5FF1FCF
:104A00001305C59797400000E780E0182244B240A4
:104A1000410117030000670083D2B7E70400FC4799
:104A20001171A2DDCAD986DFA6DBCED72E843289EA
:104A30002E86AA8517F5FF1F1305856B829717F73A
:104A4000FF1F1307E76A83470700930680029387D7
:104A5000E70793F7F70FE3ECF610BA898A0717B761
:104A600001001307E75ABA979C43BA9782878D478C
:104A700097C50100938585CD17B501001305055035
:104A8000630FF40097A00100E780C0A117C50100E3
:104A90001305858A97A00100E780C0A0BDA497A058
:104AA0000100E78020A017C501001305658A97A0C3
:104AB0000100E780209F294597A00100E78060A3BF
:104AC000930720F8114697F5FF1F938565624A8585
:104AD00017F7FF1F230EF76097F7FF1FA38B0760E1
:104AE00097F0FFFFE780603B2A841DC997C501004E
:104AF0009385C5C517B501001305454897A001006A
:104B0000E780409AA28517C501001305258897A064
:104B10000100E7802099294597A00100E780609D6A
:104B200097C50100938585C217B50100130505459A
:104B300097A00100E780009717C50100130545867F
:104B400097A00100E7800096294597A00100E78023
:104B5000409A4165930730FA054697F5FF1F938504
:104B600025597D1517F7FF1F2304F75897F0FFFF0E
:104B7000E780A0322A841DC997C50100938505BD31
:104B800017B501001305853F97A00100E7808091CC
:104B9000A28517B501001305657F97A00100E78086
:104BA0006090294597A00100E780A094B7E7040032
:104BB000BC4F0566130606C8A14517F5FF1F034540
:104BC00065C68297FE506E54DE544E59BE5911612F
:104BD000828091476303F40297C50100938505B76E
:104BE00017B501001305853997A00100E780808B78
:104BF00017B501001305057E71BDB7E70400FC4F32
:104C0000914517F5FF1F0345E5C1829797C5010040
:104C10009385C5B317B501001305453697A001006C
:104C2000E780408817B501001305857C97A0010037
:104C3000E7804087294597A00100E780808B974057
:104C40000000E780A0C2914535A485476303F402C4
:104C500097C50100938585AF17B50100130505328F
:104C600097A00100E780008417B501001305C579FE
:104C700015B597F7FF1F239F273DB7E7040005668B
:104C8000BC4F130606C8C1450DBF8D476303F40230
:104C900097C50100938585AB17B501001305052E57
:104CA00097A00100E780008017B501001305857704
:104CB000D5B3930740F8114697F5FF1F93854543F9
:104CC0004A8517F7FF1F2305F74297F7FF1FA382B7
:104CD000074297F0FFFFE780401C2A84E30405EEBB
:104CE00097C50100938585A617B501001305052911
:104CF00097900100E780007BA28517B5010013059E
:104D0000E56897900100E780E079294597900100D8
:104D1000E780207E45BD9147E31CF4F6B7E7040029
:104D2000FC4F9305000217F5FF1F0345A5AF8297BF
:104D300097C50100938585A117B5010013050524CA
:104D400097900100E780007617B501001305056F05
:104D5000F1BD894763E3870297C501009385059FED
:104D600017B501001305852197900100E780807336
:104D700017B501001305C56D31BB97F4FF1F83C440
:104D8000443797F7FF1F83C7B73697C50100938550
:104D9000E59BA20417B501001305451EDD8C979015
:104DA0000100E7802070A28517B501001305856B0F
:104DB00097900100E780006FC20429459790010099
:104DC000E7802073C1849305D4FF93960401C182C8
:104DD0004A8693F5F50F17F5FF1F130595319720B8
:104DE0000000E780A0F0E35F90DC930750F817F72E
:104DF000FF1F230FF72E83C73900228697F5FF1F69
:104E00009385052F85074A8517F7FF1FA303F72E04
:104E100097F0FFFFE78060082A84E30505DA97C56D
:104E200001009385A59217B50100130525159790EC
:104E30000100E7802067A28517C50100130505B3AF
:104E4000C9B5894763E3870297C50100938505903B
:104E500017B501001305851297900100E780806463
:104E600017B501001305C56135B197400000E78013
:104E7000E09FA28517F5FF1F1305852797400000C7
:104E8000E780C06181B38D476303F40297C50100D9
:104E90009385C58B17B501001305450E979001004A
:104EA000E780406017B501001305455FE5B6B766BA
:104EB00002000146B7750200054597E0FF1FE78035
:104EC000E08E930760F817F7FF1F2303F72297F789
:104ED000FF1FA38007229307000617F7FF1F230B6E
:104EE000F720894717F7FF1FA306F72097F7FF1F43
:104EF0002383072097F7FF1FA38F071EC14717F7CC
:104F0000FF1F230BF71E930720F917F7FF1FA305B9
:104F1000F71E314697F7FF1FA381A71E97F5FF1FC6
:104F20009385051D4A8597F7FF1F2388071C97F077
:104F3000FFFFE78080F62A84E30605C897C50100D5
:104F40009385C58017B501001305450397900100AF
:104F5000E7804055A28517B501001305A55555B347
:104F6000B1476303F40297B501009385257E17B519
:104F700001001305A50097900100E780A05217B526
:104F800001001305E55439B6B7E70400FC4F93055B
:104F9000000417F5FF1F0345E5888297974000003E
:104FA000E780C08CB145F9B5914763E3870297B5B7
:104FB00001009385A57917B50100130525FC97908D
:104FC0000100E780204E17B5010013052552D9B422
:104FD00097F4FF1F83C4041297F7FF1F83C777114D
:104FE000A204DD8C8E04B77702006D14BE94228675
:104FF000A68517B501001305A55097900100E7801D
:10500000604AB7E70400FC47228697F5FF1F9385A7
:10501000750E2800829793160401C1823000A68580
:10502000094597D0FF1FE78060782A8409C917B522
:1050300001001305A54E97900100E780805E93075D
:1050400070F8194697F5FF1F9385850A4A8517F76B
:10505000FF1F230FF70897F7FF1FA38D870897F00F
:10506000FFFFE78080E32A84E30E05B497B50100D3
:105070009385C56D17B50100130545F097900100A4
:10508000E7804042A28517B501001305254A95B96E
:105090009947630BF41297B501009385256B17B5FB
:1050A00001001305A5ED97900100E780A03F17B51B
:1050B000010013052549F9BA914763E3870297B5C3
:1050C00001009385A56817B50100130525EB97909E
:1050D0000100E780203D17B50100130525485DBAA2
:1050E00097F4FF1F83C4040197F7FF1F83C777005E
:1050F000A204DD8C8E04B77702006D14BE94228664
:10510000A68517B501001305A54697900100E78015
:105110006039B7E70400FC47228697F5FF1F9385A7
:1051200075FD2800829793160401C1823000A68580
:105130000D4597D0FF1FE78060672A8409C917B51E
:1051400001001305A54497900100E780804D930767
:1051500080F8194697F5FF1F938585F94A8517F75B
:10516000FF1F2307F7F897F7FF1FA38587F897F02E
:10517000FFFFE78080D22A84E30605A497B50100EB
:105180009385C55C17B50100130545DF97900100B5
:10519000E7804031A28517B501001305654095B63B
:1051A00099476303F40297B501009385255A17B513
:1051B00001001305A5DC97900100E780A02E17B52C
:1051C00001001305653FF9B0B7E70400FC4F9305F4
:1051D000000417E5FF1F0345E56482979730000040
:1051E000E780C068994579B18D476303F40297B5AC
:1051F00001009385A55517B50100130525D8979093
:105200000100E780202A17B501001305653C59B05D
:1052100017B501001305C53C97900100E780604079
:105220001305C01297D0FF1FE780A011014597E03A
:10523000FFFFE78020E30D4597100000E780009F07
:10524000294597D0FF1FE780C00F97D0FF1FE78049
:1052500020008DBA99476303F40297B50100938546
:10526000E54E17B50100130565D197900100E78061
:10527000602317B501001305653729B817F7FF1F1D
:10528000034757E797F7FF1F83C7C7E622075D8FDE
:105290009166BA96C2061166C1821306F6EF8D4773
:1052A0006365D60297E7FF1F9387470D9C4B17F660
:1052B000FF1F034616E49386C7002DC203D60700DE
:1052C00069CA8907E39CD7FE89471307A0F81146EE
:1052D00097F5FF1F9385C5E14A8597F6FF1F238940
:1052E000E6E017F7FF1FA306F7E097F0FFFFE78060
:1052F000C0BA2A84E308058C97B50100938505455B
:1053000017B50100130585C797900100E780801944
:10531000A28517B501001305A52EE5B203D6070037
:10532000630EE60A8907E39BF6FE8D4779BF914736
:105330006304F40297B501009385454117B5010058
:105340001305C5C397900100E780C01517B501008C
:105350001305852C6FF00FF4B7E70400FC4F93059D
:10536000000817E5FF1F0345E54B8297C9B897B5BD
:1053700001009385A53D17B50100130525C0979041
:105380000100E780201217B501001305652A6FF0B0
:105390006FF02390E70017E5FF1F130525FE972008
:1053A0000100E780A03C97B501009385253A17B529
:1053B00001001305A5BC97900100E780A00E17B56A
:1053C00001001305E52797900100E780A00D29450E
:1053D00097900100E780E0118147C5BD2390070049
:1053E00017E5FF1F130585F997200100E7800038B6
:1053F00097B501009385853517B50100130505B8EC
:1054000097900100E780000A17B501001305C52435
:105410005DBF411122C406C6834705002A849DC78B
:1054200097B501009385452E17B50100130505B505
:1054300097900100E78000074C4017B50100130565
:10544000255997900100E780E005E1A05841B70792
:10545000CF009387777D631DF70697B5010093858D
:10546000A52A17B50100130565B197900100E780E3
:1054700060031C448356E4008355C40003C6070040
:1054800017B501001305455697900100E78080018C
:10549000294597900100E780C0050357E40097076E
:1054A000002083D7C7246309F7008355C40008444C
:1054B00097E0FFFFE78080CF0356E4008355C400E8
:1054C00008442244B240410117F3FFFF670023550F
:1054D000B707CC009387777D6315F70497B5010074
:1054E0009385852217B50100130545A99790010002
:1054F000E78040FB1C448356E4008355C40003C688
:10550000070017B501001305254E97900100E780AD
:1055100060F92244B2402945410117930100670018
:1055200043FDB707CE009387777D6304F70297B5F5
:1055300001009385651D17B50100130525A49790FB
:105540000100E78020F64C4017B501001305053F28
:10555000CDBDB240224441018280B7E70400FC4740
:1055600041112E8606C622C426C24AC02E842A892C
:10557000AA8517F5FF1F1305A5B7829797B50100F8
:105580009385851E17B501001305459F979001006F
:10559000E78040F197F5FF1F83C585B517B501007A
:1055A000130585C497900100E780C0EF29459790C7
:1055B0000100E78000F497F4FF1F938464B383C76E
:1055C000040041479387070693F7F70F636AF75C78
:1055D00017B70100130707AE8A07BA979C43BA971B
:1055E00082879D476307F40297B501009385C5172D
:1055F00017B501001305859897900100E78080EAB0
:1056000017B501001305C5BE97900100E78080E93A
:10561000ADAC97F7FF1F83C7B7ADDDCB17F7FF1F03
:10562000034737AD97F7FF1F83C7A7AC22075D8FEE
:1056300097F7FF1F83C707ACC2075D8F97F7FF1F60
:1056400083C757ABE207D98F17F7FF1F2320F7A8AF
:1056500083C7640097B501009385051117B5010054
:105660001305C59117F7FF1F2301F7A697900100B7
:10567000E78040E397F7FF1F938747A58C4317F612
:10568000FF1F034686A417B50100130525B89790A0
:105690000100E78020E1294597900100E78060E55F
:1056A00097F7FF1FA38607A42244B2409244024901
:1056B000930700F817F7FF1F230CF7A29D4517F576
:1056C000FF1F1305E5A2410117430000670003DD3A
:1056D00097600000E780808D97F7FF1F238BA7A0BE
:1056E0009357850017F7FF1FA305F7A093570501F0
:1056F0002A8417F7FF1F230FF79E93578501014553
:1057000017F7FF1FA308F79E97600000E780C08A85
:1057100097F7FF1F2381A79E97B501009385C504C6
:1057200017B501001305858597900100E78080D7A4
:1057300017F6FF1F0346269CA28517B50100130527
:1057400065AEB1B7CD476303F40297B50100938509
:10575000A50117B501001305658297900100E78048
:1057600060D417B50100130565AD79BD37E40400B9
:105770007C44414697F5FF1F9385959717F5FF1FCA
:1057800013050595829717F5FF1F1305659497106C
:105790000000E78080C497100000E78000AC97F716
:1057A000FF1F83C7079617F7FF1F03477795A207C9
:1057B00003238405D98F17F7FF1F2317F7901306CC
:1057C000000A89452244B2409244024917E5FF1F6E
:1057D00003454505410102838D476303F40297B5F4
:1057E0000100938565F817A50100130525799790A9
:1057F0000100E78020CB17B501001305E5B329B5FB
:1058000017F4FF1F0344E48E97F7FF1F83C7578EDB
:1058100097B50100938545F5220417A501001305EE
:10582000E5755D8C97900100E780C0C7A28517B52C
:105830000100130525A297900100E780A0C6294525
:1058400097900100E780E0CA0D4697F5FF1F93850A
:10585000258A228597E0FFFFE7802064AA8421C182
:1058600097B50100938545F017A501001305057153
:1058700097900100E78000C3A68517B501001305C6
:10588000A59E97900100E780E0C12244B240924477
:1058900002492945410117930100670083C597E735
:1058A000FF1F2399877AB7E70400116603A38705D2
:1058B000130606E8914539B78D476303F40297B59F
:1058C0000100938565EA17A501001305256B9790E4
:1058D0000100E78020BD17B501001305A5B42DB365
:1058E00017F4FF1F0344E48097F7FF1F83C7578017
:1058F00097B50100938545E7220417A5010013051C
:10590000E5675D8C97900100E780C0B9A28517B567
:1059100001001305A59697900100E780A0B82945DE
:1059200097900100E780E0BC0D4697E5FF1F938547
:10593000257C228597E0FFFFE7802056AA841DC1C1
:1059400097B50100938545E217A50100130505638E
:1059500097900100E78000B5A68517B501001305F3
:10596000259305B797E7FF1F2398876CB7E70400D7
:10597000116603A38705130606E89305000299B58F
:10598000894763E3870297B501009385E5DD17A595
:1059900001001305A55E97900100E780A0B017B540
:1059A00001001305E5AA8DB197E4FF1F83C4647459
:1059B00097E7FF1F83C7D77397B501009385C5DAB3
:1059C000A20417A501001305655BDD8C979001000B
:1059D000E78040ADA68517B501001305E58C9790CB
:1059E0000100E78020AC294597900100E78060B076
:1059F000228697E5FF1F9385A56F268597E0FFFF19
:105A0000E780A0492A84630E051A97B501009385A3
:105A1000A5D517A501001305655697900100E780ED
:105A200060A8A28517B501001305458999BD854772
:105A300063F98718834519002244B2409244024911
:105A4000B335B00097E7FF1F2380B76217B5010099
:105A5000130505884101179301006700A3A4A285DF
:105A60002244B24092444A85024941011703000092
:105A70006700032299476303F40297B501009385F9
:105A8000A5CE17A501001305654F97900100E7808B
:105A900060A117B50100130565B5BDB617E4FF1F7A
:105AA0000344246597E7FF1F83C7976497B50100F8
:105AB000938585CB220417A501001305254C5D8C29
:105AC00097900100E780009EA28517B5010013059D
:105AD000A58197900100E780E09C294597900100FF
:105AE000E78020A1194697E5FF1F93856560228511
:105AF00097E0FFFFE780603AAA841DC197B50100D7
:105B0000938585C617A501001305454797900100A9
:105B1000E7804099A68517A501001305E57D95B39B
:105B200097E7FF1F239E875AB7E70400116603A378
:105B30008705130606E89305000869B1854797B500
:105B40000100938565C217A5010013052543630B6A
:105B5000F40097900100E780E09417A50100130579
:105B6000E57A5DB497900100E780C09317A5010026
:105B70001305457B97900100E780C09229459790D7
:105B80000100E78000972244B2409244024997E71F
:105B9000FF1F239B07524101175300006700833109
:105BA00097B50100938545BC17A501001305053D78
:105BB00097900100E780008F17B50100130545A7F6
:105BC000A1B4B24022449244024941018280411171
:105BD00006C622C497E0FFFFE780202C9377F50FDD
:105BE000A1C32A8497B50100938585B917A5010043
:105BF0001305C53897900100E780C08A9375F40FAC
:105C000017B50100130585D697900100E7808089BC
:105C10002244B24029454101179301006700638D7A
:105C2000B240224441018280411122C491462A841B
:105C300017E6FF1F1306065A9D652D4506C697D029
:105C4000FF1FE780A0B6B7F7070003C70701A54706
:105C50006313F70001A09306001001469D652545DA
:105C600097D0FF1FE78080B497E7FF1F23848756F4
:105C70002244B240914617E6FF1F1306A6559D65C4
:105C80002945410117D3FF1F670043B25171CAD1A3
:105C900037E904008327C904A2D52E8686D7A6D368
:105CA0002E84AA8517E5FF1F13058544829797E781
:105CB000FF1F83C7E7431307700A6387E710636C0E
:105CC000F7001307600A6384E704BE502E549E5405
:105CD0000E596D6182801307800A6388E7161307E7
:105CE000900AE394E7FE8D476309F41C97B5010021
:105CF000938505DB17A50100130545289780010052
:105D0000E780407A17B501001305C5D625A08D4759
:105D1000630CF40297B50100938585D817A501009F
:105D20001305C52597800100E780C07717B50100EE
:105D3000130585CD97800100E780C07629459780BF
:105D40000100E780007B51B7854717B501001305B7
:105D500065CD17E7FF1F2309F73097900100E78013
:105D6000408CB7750200B76602000146054597D022
:105D7000FF1FE780A0A3930760F817E7FF1F230921
:105D8000F73697E7FF1FA38607369307002617E726
:105D9000FF1F2321F736E5779387072117E7FF1FBA
:105DA000231CF734B14597E7FF1F2388073497E793
:105DB000FF1FA384A73417E5FF1F13056533973032
:105DC0000000E780A06D11B7914763E3870297B5A4
:105DD00001009385E5CC17A501001305251A9780CE
:105DE0000100E780206C17B501001305A5C599B720
:105DF00097E4FF1F83C4043097E7FF1F83C7772F03
:105E0000A204DD8C8327C9046D14228697E5FF1F49
:105E10009385552E280082978E0493160401B7753A
:105E20000200C1823000A695094597D0FF1FE78088
:105E3000E097930770F817E7FF1F230BF72A9945A0
:105E400097E7FF1FA388A72ABDB7914763E387029F
:105E500097B501009385C5C417A501001305051268
:105E600097800100E780006417B50100130505BFA6
:105E7000D1B597E4FF1F83C4E42797E7FF1F83C7CB
:105E80005727A204DD8C8327C9046D14228697E569
:105E9000FF1F93853526280082978E0493160401F0
:105EA000B7750200C1823000A6950D4597D0FF1F3F
:105EB000E780C08F930780F8BDBF17B501001305B9
:105EC000A5BC97800100E780C0751305C01297C07C
:105ED000FF1FE7800047014597D0FFFFE78080184C
:105EE0000D4597000000E78060D4294597C0FF1F4B
:105EF000E780204597C0FF1FE7808035F9B3411147
:105F00004AC097F6FF1F83D6867E328917D6FF1FB9
:105F10000356E64822C426C206C62A84AE849700E9
:105F20000000E780C05F35C12DC0994763FF97042B
:105F30008347140003470400A207D98F13978700F3
:105F4000A183D98FC2073167C1831307C755639EE9
:105F5000E70297D7FF1F83D78744A301F400A183EB
:105F60002302F40097F7FF1F83D7677891C7A30236
:105F7000F400A1832303F400A68517B501001305DF
:105F800025B697800100E780E05197F7FF1F83C790
:105F9000A765B9CF97D5FF1F83D5654017B5010019
:105FA0001305C5B597800100E780C04F2686A285FE
:105FB00017D5FF1F0355A53E97000000E78060C17D
:105FC0006301090497E7FF1F83C7C7219DCB95C8CD
:105FD00097E7FF1F83C747098DE722852244B24018
:105FE0000249A68592444101173300006700034B24
:105FF00017B50100130585B197800100E780606245
:10600000C1B7B24022449244024941018280834791
:1060100055008345450017B50100130525ABA207C0
:10602000DD8D178301006700E34717B501001305F5
:10603000E5A8178301006700C35E8D4763FBB70ABD
:10604000011126CA06CE22CC0344350097E4FF1F77
:1060500083C4541997B50100938505ACB33780000C
:1060600017E7FF1FA300F71809C497B50100938530
:1060700065AB17B50100130565AB97800100E7809C
:10608000604297E7FF1F83C7F71563869700970065
:106090000000E780802697E7FF1F83C7B7148DC7EE
:1060A00085472306F100B7E7040083A74717700070
:1060B000854513055030829717B50100130505A8D3
:1060C00097800100E780E0559967938757EE231684
:1060D000F100680085479145A30781002307F1007F
:1060E00097300000E780803BF2406244D244056173
:1060F00082808280894763F7B708011122CC06CEDF
:1061000026CA8344250085472A84639DF404914769
:1061100063F5B704034545008347340022055D8DD0
:1061200097D7FF1F239DA72697000000E780004810
:106130009967938767EE2314F100834734002305A2
:106140009100A305F10083474400954528002306EC
:10615000F10097300000E7806034F2406244D2449E
:1061600005618280FDF89967938767EE2314F1003B
:1061700097D7FF1F83D7A722A305F10023050100AE
:10618000A183E1B782800111996722CCD51717F45A
:10619000FF1F130464452314F1008347040026CA3B
:1061A00097F4FF1F9384A4542305F10083D70400C0
:1061B00028009545A305F100A18306CE2306F10032
:1061C00097300000E780802D03D60400834504004B
:1061D00017B501001305059897800100E780802C12
:1061E000F2406244D244056182809D677971D9177B
:1061F0002316F10097F7FF1F83C7073F06D6230733
:10620000F100A9C3B7E70400FC47414697E5FF1F2B
:10621000938505EC1305F10082976800CD45973012
:106220000000E780A02797F5FF1F83C5E53B17B562
:1062300001001305259597800100E780A026B25044
:1062400045618280B7E70400BC474146814513059C
:10625000F1008297D9B7B76702045D71938757AA97
:106260003EC08567938707302312F10097F7FF1F21
:106270009387873783C70700A2C4A30301002303C2
:10628000F10097F7FF1F9387874683D7070037E40E
:10629000040086C62314F10097D7FF1F93872710A9
:1062A00083D70700414668002315F1007C4497E539
:1062B000FF1F9385E5E18297F1450A85970000006D
:1062C000E780E021231EA1007C448A8508107946DE
:1062D00082973C441305E1030946814582971010DB
:1062E00093050002014597D0FFFFE780003EB640CE
:1062F000264461618280B7C7A55A01119387C733CD
:106300003EC497E7FF1F83C7F7ED3EC6B7F7070008
:1063100003C7070106CE22CCA5476313F70001A0EF
:106320001164930504F0930600100146254597C0BB
:10633000FF1FE780A0473000930504F0A1462945E0
:1063400097C0FF1FE780804697E5FF1F83C595E94B
:1063500017B501001305C59397800100E7808014ED
:10636000F24062440561828001119165A1463000CE
:10637000938505F02D4506CE97C0FF1FE7800043AB
:106380002247B7C7A55A9387C7336314F702B245AC
:1063900017B5010013050583B335B00097E7FF1F5C
:1063A000A382B7E497800100E780C00FF240056147
:1063B0008280814517B501001305058397E7FF1F0C
:1063C000A38207E297800100E780C00D97000000DC
:1063D000E780A0F2E1BFB7C7A55A79719387F73577
:1063E0003EC6B7E70400FC47AA8506D622D441463C
:1063F00008088297B7F7070003C70701A54763138B
:10640000F70001A01164930504E89306001001460B
:10641000254597C0FF1FE78060397000930504E8A9
:10642000D146294597C0FF1FE780403817B50100C6
:106430001305C58997800100E780A01EB250225441
:106440004561828079719165D1467000938505E838
:106450002D4506D697C0FF1FE78040353247B7C7A6
:10646000A55A9387F73517A501001305E57F63103B
:10647000F702B7E70400FC4717E5FF1F130545C502
:1064800041460C08829717A501001305E57B97800C
:106490000100E7800019B25045618280B7F707001C
:1064A00003C70701A5476313F70001A091654111D8
:1064B000930600100146938505E8254506C697C05A
:1064C000FF1FE780A02EB24017A501001305C56D80
:1064D0004101178301006700C314C16769768146D3
:1064E000FD1705061397060141836364B7003E85D7
:1064F00082803307D50003470700B98F214713F87F
:106500001700858363050800B18FC207C1837D171B
:106510001377F70F6DF78506F1B741C5A547054716
:1065200063F2B70883471500034705003168A207E7
:10653000D98F13978700A183D98FC207C18313080E
:10654000C855054763900707411106C622C426C2F5
:1065500003442500914763F087049307540063ECDC
:10656000F502A301C50021822302C5009304340073
:1065700091C6A302D500A1822303D5002A84A68553
:1065800097000000E780A0F526942300A400218155
:10659000A300A4000147B240224492443A8541013D
:1065A000828005473A858280B7C7A55A0111938733
:1065B000E7343EC42AC6B7F7070003C7070106CE73
:1065C00022CC26CAA5476313F70001A091642A8450
:1065D000938504EE930600100146254597C0FF1FE2
:1065E000E780C01C3000A146938504EE294597C082
:1065F000FF1FE780A01BA28517A501001305456BAF
:1066000097800100E78000EA97000000E780E0C47F
:10661000F2406244D2440561828001119165A14635
:106620003000938505EE2D4506CE97C0FF1FE7800D
:10663000E0172247B7C7A55A9387E7346318F702D4
:10664000B24517A501001305255C97D7FF1F2398B6
:10665000B7D4C205C18197800100E780A0E497000C
:106660000000E78080BFF24005618280D147D145BC
:1066700017A501001305455B17D7FF1F2311F7D29C
:1066800097800100E78000E217D5FF1F035525D151
:1066900097000000E78080F1F9B721C1411126C2BF
:1066A00006C622C4AE848DC52A8497200000E780E8
:1066B00040C097E7FF1F83C7E7B299CB22852244EA
:1066C000B240A6859244410117330000670003DD04
:1066D000B2402244924441018280828001114AC822
:1066E00006CE22CC26CA4EC693F715002E899DCB26
:1066F000AD67371700409387A7AA1CC3B7E704000C
:10670000BC4F13060019854517D5FF1F034505C962
:10671000829713451900F2406244D2444249B2497B
:106720000561828093F725006385071C97F6FF1F9C
:1067300083C6C6FB139706014183954763F9E70CAF
:10674000014417F5FF1F130565EA1306300513080A
:106750005004930810041303B004130E900593071C
:10676000640063F4F6043A84FD5997F4FF1F83C470
:10677000E4E797F7FF1F83C777E7A204DD8CAD67D7
:106780009387B7556383F41463E3970AA9679387E4
:10679000A7556386F414A28517F5FF1F130505E5B9
:1067A00097000000E780A0EFF5A8B307850083C538
:1067B0000700639AC50483C517006396050583C562
:1067C00027006392150583C53700639EC50283C504
:1067D0004700639A650283C757006396C703A2897F
:1067E0000DE897F5FF1F83C565F0B3853541C205F8
:1067F00017F5FF1F130585DFC1814E959700000037
:10680000E780E0E965A805044204418089BF3A8435
:10681000FD598547E3EB87F459CC854517F5FF1FF4
:106820001305C5DC97000000E78060E769A0B16749
:106830009387C7556380F404B5679387D755E39C66
:10684000F4F4A28517F5FF1F130545DA9730000011
:10685000E780C0C489476307F4049305E4FFC205D9
:10686000C18117F5FF1F130585D897200000E78029
:1068700040A40DA897000000E780603711C9A285E9
:1068800017F5FF1F130585D697200000E78060A24B
:106890000546A28517F5FF1F130545D597F0FFFFA5
:1068A000E7802066A68517A501001305254497807B
:1068B0000100E78020BFFD57E395F9F297F7FF1F2E
:1068C000238607E213452900B9B5A28517F5FF1FF6
:1068D0001305C5D197F0FFFFE780A073E1B7A2854C
:1068E00017F5FF1F130585D097F0FFFFE780207491
:1068F00055BF93F745000145E38F07E017A5010059
:106900001305054097800100E780A0D19730000073
:10691000E780C0C713454900FDBB411122C437E4DD
:1069200004005C5C06C6354697A50100938545EEDC
:1069300017B50100130505AE829711E917A50100EF
:106940001305C53C97800100E780A0CD01A08327F7
:10695000041C82972A84054597C00000E780E080E8
:1069600097600100E780000697600100E78000DB88
:1069700097B00000E78060922285B2402244410136
:1069800082801567B71700401307575598C3D8433F
:106990009D66558FD8C3D843FD76758FD8C3D8432D
:1069A0001367F70FD8C335671307C7CC98C3828026
:1069B0004111054506C622C426C297C0FFFFE780E5
:1069C00040541305800497B0FF1FE780406E757533
:1069D00085457D1597C0FFFFE780E03D7D758545C6
:1069E0001305F53697C0FFFFE78040473714004096
:1069F0008327840A8D451305002093E7072023246D
:106A0000F40A97C0FFFFE780003BB7E4040097D08B
:106A1000FFFFE7802080C85897800100E78060C0B2
:106A200017B501001305059F97800100E78060BF3F
:106A30008327840C8545414593E707082324F40CFC
:106A400097C0FFFFE78080418D451305000897C080
:106A5000FFFFE780A04097C0FFFFE780806D716572
:106A60001305052097C0FFFFE7804069014597C0E7
:106A7000FFFFE780606F85450545894717F7FF1FD2
:106A80002308F7C697C0FFFFE780A06F3707000411
:106A9000B7E700E023A0E71097D0FFFFE7804001B1
:106AA00097D0FFFFE780001597000000E78020E700
:106AB00097000000E780808B97000000E78020B6F9
:106AC00097E0FFFFE780E0F097000000E780C0124A
:106AD00097000000E780600B83A7040817050000FB
:106AE000130505C0829797D7FF1F2389A78ABC4C3F
:106AF000130600648545829797000000E780A0E8B0
:106B000097C0FF1FE780C08E01458280B7F707005E
:106B100003C70701A547AE866316F70093974501A3
:106B200091C301A0AA850146254517C3FF1F670031
:106B3000E3C74111B2862E86AA852D4506C697C0A9
:106B4000FF1FE780A0C6B240014541018280930744
:106B5000000463E8C7021D71A2CC2A84080886CE0F
:106B600032C697800100E7808088B2461008A2856F
:106B7000294597C0FF1FE78060C3F6406644256142
:106B800082803955828041110D658D4506C697C0BA
:106B9000FFFFE7804022B71700408D6623A6D70A83
:106BA00017F5FF1F130505B51387C70A9387870AD3
:106BB0001CC15CC5856689675CC958C114C518C904
:106BC000B7E70400B24003A3871E41010283814559
:106BD000B307B5008387070089E717130000670034
:106BE000436D8505C205C181E5B717F5FF1F034554
:106BF000E5B1828097F7FF1F83C757B199EF411125
:106C000006C697100000E780A062B240854717F7DC
:106C1000FF1FA30DF7AE41018280828059C5D1C507
:106C2000411122C426C206C6C1472A84AE8463F439
:106C3000B706414697A5010093850514977001009A
:106C4000E780807829E983470401130710036393E1
:106C5000E702854717F7FF1F230AF7AA17A50100C8
:106C60001305C5122244B2409244410117030000AB
:106C7000670023F61307000317A501001305051489
:106C8000E392E7FE97F7FF1F238207A817A50100ED
:106C900013054511C1BF22852244B240A685924406
:106CA000410117C3FFFF670063508280411126C274
:106CB000AE848D4522C406C62A8497C0FFFFE780B4
:106CC000E019B717004099C803A5C70C418D23A64A
:106CD000A70CB240224492444101828003A5870C54
:106CE000418D23A4A70CF5B7834705000347150082
:106CF000A207D98FC2076177C18713072720639A3C
:106D0000E7008345250037050400170300006700EE
:106D100023FA828017F6FF1F1306869F8147B286EB
:106D20001303F00FA9483308F6000348080013F7CF
:106D3000F70F6307A80C630668008507E39517FF44
:106D40002947B387E6002380A70097F7FF1F9387A3
:106D5000E79C5DA8411113D765001347170006C6CD
:106D600093F63500058B954791CA05469947638789
:106D7000C60009469D476383C600A14713F6450038
:106D80003336C00093F68503050685C2A145638BA3
:106D9000B604E145638AB604930580026388B604AD
:106DA000930580036393B600914697F5FF1F238CEC
:106DB000F5BC97F5FF1F2387C5BC97F5FF1FA3837D
:106DC000D5BCBE8517A501001305450497700100C9
:106DD000E780406DB240854717F7FF1FA305F7BA5C
:106DE000410182808546D1B78946C1B78D4675BFBE
:106DF00017A5010013050504177301006700836AD6
:106E000017F7FF1F13078791BA972380B700E14751
:106E1000E302F5F493077002E30CF5FC82802A8705
:106E200023800500814717F5FF1F1305658E1308A2
:106E3000F00F2946B306F50083C606006396E60206
:106E400097F6FF1F9386868DB69783C70700054583
:106E50002380F5009947636EF7029D4763FDE700C5
:106E6000E147630DF7008280638506018507E393A0
:106E7000C7FC0145C5B7238005008280B7370040B5
:106E800003C7370083C7050093F70704D98F238012
:106E9000F5008280797126D24AD097F4FF1F83C40F
:106EA00064C017F9FF1F130929BF06D622D44ECE9E
:106EB00052CC56CA5AC8B307990083C7070093F744
:106EC000F70FA5C79387140093F7F70F0D4763617A
:106ED000F70C17F7FF1F2307F7BC97F7FF1F9387E0
:106EE00027BCA69783C707001307100293F7F70381
:106EF0006389E7226363F70A054463808720E3829E
:106F0000076809476389E71413070002E387E7521C
:106F1000B7E700E03707400023A0E71801000100B1
:106F2000CA942380040023A0E710B787004003C75A
:106F30006700058BE308077297F6FF1F83C6A6B6A6
:106F40000547E393E67029472381E7020947238336
:106F5000E7022385E70297F7FF1FA38707A297F7AA
:106F6000FF1FA38207B4B7870040A381070017F76C
:106F7000FF1FA30D07A005472383E700B25022544B
:106F800092540259F249624AD24A424B4561828088
:106F900097F7FF1F238807B089B71307300263866E
:106FA000E70A63E6E71413074002638AE70813075A
:106FB0000003E39FE7F497F7FF1F938727AEA69799
:106FC00003C70700A1471377F70FE313F71617EA74
:106FD000FF1F130A6A7583476A0097F6FF1F238B0A
:106FE000F69897E7FF1F83C7977491C7FD5797F6E9
:106FF000FF1F2381F69897E5FF1F83C5F57297F76A
:10700000FF1FA389B79697E7FF1F83C7E77193F91F
:1070100007089306000493F70706639DD74A930772
:10702000A0096387F51463E4B7109307F005638440
:10703000F548930750096382F52801440DABFD57CD
:1070400017F7FF1F2307F792E1B5FD5717F7FF1F4B
:107050002300F79275BD17A50100130525EF977062
:107060000100E780005C97F7FF1F938727A3A6978F
:1070700003C40700814917FAFF1F130A6A831374B8
:10708000F40F97AA0100938AEAEC63C789042945A3
:1070900097700100E780E045854717F7FF1FA307BA
:1070A000F78017F7FF1F2304878017F7FF1F230DB3
:1070B000F78C37E700E0B70640002320D71801001F
:1070C0000100378600408347A60293F7370F230558
:1070D000F6022320D7102DBDB3073A0183C5070060
:1070E0005685850997700100E780C03B79BF8547C9
:1070F00017E7FF1F230CF77A21BD17F7FF1F1307B0
:10710000E79926970347070097E6FF1FA38EF66CC3
:1071100097E6FF1F238BE66C17F7FF1F2306F78602
:10712000C5BB854717E7FF1F2300F76CD5B393074F
:10713000400A638DF5349307200B6388F536930777
:10714000100AE39CF5EE83072A00014463D107424D
:1071500097E7FF1F83C7775D93F63700638E061AA4
:107160000546638EC62209466399C61A1D4775A255
:1071700017E5FF1F0345655BC94717EAFF1F034A71
:10718000DA5A97E5FF1F83C5655A17E4FF1F0344CA
:10719000F4596319F510CD476316FA109307700878
:1071A000639CF5021307300FB7170E006308E40065
:1071B0001307900DB7B704006314E40817E7FF1F27
:1071C0002320F77CBE8517A50100130525D99770EC
:1071D0000100E780202D95B593078008639DF50099
:1071E00033048040B77746001374F40F938787CD3C
:1071F000B3D78702E1B793079008639AF500330489
:10720000804091671374F40F9387C766D5B79307CF
:10721000A008639BF50033048040B7173D0013744A
:10722000F40F93870790E9B79307B008639AF500C6
:107230003304804091671374F40F938797D04DBF48
:1072400093F5F5078D47639BF50033048040B797AE
:107250005B001374F40F938707D859BF8947639B6A
:10726000F50033048040B7770B001374F40F938755
:10727000071BBDBF8547639AF50033048040DD6777
:107280001374F40F938767E3A5B789E9330480404B
:107290008D671374F40F938777DC99BFF167938739
:1072A000072029BF97000000E78000A7A28552852C
:1072B00097000000E78040A649B39305610017E5F9
:1072C000FF1F0345854617E4FF1F0344144697003C
:1072D0000000E78000B5930571002285970000004B
:1072E000E78020B43C0017E7FF1F2325F77A834788
:1072F00061002304F10083477100A304F100894772
:1073000017E7FF1F2308F7668357810017E7FF1F62
:10731000231CF7400944A1AC154793F64700B33648
:10732000D00093F78703850685C32146638BC70684
:107330006146638AC706130680026388C706130680
:1073400080036393C700914717E6FF1F230CD662A3
:1073500097E6FF1FA388F66297E7FF1F2385E76282
:1073600017E7FF1F0347873C9376070497E7FF1F44
:1073700083C7D73B8DEE1377770C93067008630CA9
:10738000D7021377F7078D46631ED70AB307F0407D
:10739000B7955B0093F7F70F938505D881A8194738
:1073A000ADBF854755B7894745B78D4771BF930630
:1073B00070086311D7021307300FB7150E006389E9
:1073C000E7021307900DB7B504006383E7021307C4
:1073D000700845BF9306800C6311D702B307F040D5
:1073E000B775460093F7F70F938585CDB3D5F502B2
:1073F00097E7FF1F23A6B758F9B39306900C631ABB
:10740000D700B307F040916593F7F70F9385C566F2
:10741000F1BF9306A00C631BD700B307F040B7156C
:107420003D0093F7F70F93850590C9B79306B00C0D
:10743000E319D7F4B307F040916593F7F70F9385FD
:1074400095D06DB78946631BD700B307F040B77579
:107450000B0093F7F70F9385051B49BF8546631A09
:10746000D700B307F040DD6593F7F70F938565E329
:10747000B5BF09EBB307F0408D6593F7F70F938520
:1074800075DCADB7F165938505209DB783472A006C
:10749000C18B99C7854717E7FF1F2300F74E71BEC1
:1074A00097E7FF1F238B074C49BE854717E7FF1F50
:1074B000A30BF74C59B63C0017E7FF1F232CF75CD2
:1074C0000947930700032314F10097E6FF1F238366
:1074D000E64A2DBD63990758A94763EBB74417A740
:1074E00001001307E78F8A05BA959C41BA978287F6
:1074F00017E4FF1F03447423094A630C440F636CB1
:107500008A0885476309F40A9307F00F17E7FF1FFE
:107510000347474663F6E70017E7FF1F230CF744CE
:1075200017EAFF1F034A0A45930700041374FA0F72
:1075300063F447011304000497E7FF1F93878755FF
:1075400083AA0700228617E5FF1F1305E51DD685D0
:10755000330A8A40A29A97700100E78040E997E7D2
:10756000FF1F2389474197E7FF1F23A5575397E73D
:10757000FF1F83C7374015476399E762B7E700E00D
:107580003707400023A0E71801000100B78600403C
:107590002380860285A58D47630CF40A9947E3157D
:1075A000F4F697A701009387278A17E7FF1F232385
:1075B000F74EA947A1BF17E7FF1F0347C74E97E73D
:1075C000FF1F9387273D494697A501009385C590E6
:1075D0006306870097A501009385058C3E8597700B
:1075E0000100E780C0E017E7FF1F2325A74AC9472E
:1075F00031BF97E6FF1F83C6064B054797E7FF1F7E
:10760000938747396394E6023E851306700297A577
:1076100001009385E58997700100E78040DD17E759
:10762000FF1F2329A74693077002CDB53E85130699
:10763000300497A501009385E58197700100E780EC
:1076400000DB17E7FF1F2327A744930730047DBD06
:1076500097E5FF1F83C5650D17A50100130545912B
:1076600097700100E78000E4854A17EBFF1F034B8A
:107670008B4397E5FF1F83C5450B17A50100130535
:10768000258F63185B0B97700100E780A0E197E7F7
:10769000FF1F83C78709B5CBE368F4E617A4010091
:1076A0001304C487638C670117A401001304848743
:1076B0006386470117A4010013044488228597704C
:1076C0000100E780C0FE1375F50F930715008607CC
:1076D00017E7FF1F2300F72C8D4717E7FF1FA30BAA
:1076E000F72A97E7FF1F9387E72A0147BE8613769D
:1076F000F70F89076365A60297E7FF1F23ACD7380A
:1077000097E7FF1F83C7072911B597970100938754
:10771000E77917E7FF1F232FF7369147C5BB3306DD
:10772000E40003460600A380070005072380C70086
:107730007DBF97700100E780E0D697E7FF1F83C702
:10774000C7FEE1D7E362F4DC179401001304047A66
:10775000638C5701179401001304C47963864701B1
:10776000179401001304847A228597700100E78042
:1077700000F41375F50F93071500860717E7FF1F31
:10778000230AF7208D4717E7FF1FA305F72097E788
:10779000FF1F938727200147BE861376F70F8907BF
:1077A000E37CA6F43306E40003460600A38007004A
:1077B00005072380C700D5B797E5FF1F83C5E5F60A
:1077C000179501001305857B97700100E78080CD38
:1077D00097E7FF1F83C7D71B93E7470017E7FF1FF4
:1077E000A308F71A83472A0017E7FF1FA300F71A19
:1077F000A9B0179501001305A57997700100E780DE
:1078000040E297E7FF1F9387671883C7070017E7D2
:10781000FF1F230BF7F017E4FF1F0344A4153334B5
:107820008000B1B3179501001305C577977001006B
:10783000E78020DF97E7FF1F83C7971593E70701CE
:1078400017E7FF1FA306F71483472A0017E7FF1F58
:10785000230EF7126FF06FFE179501001305C57523
:1078600097700100E780E0DB03470A007D8B51EF52
:10787000B787004003C767021377C70B136727005A
:107880002383E70203C7A7021377C70B13672700F9
:107890002385E70203C7E7021377C70B13672700A7
:1078A0002387E70203C727031377C70B1367270054
:1078B0002389E702854717E7FF1F2307F7F217E73A
:1078C000FF1F2305F7FE17E7FF1F2303F70A17E73C
:1078D000FF1F2300F70A97E7FF1FA38707F097E72B
:1078E000FF1FA38507FC97E7FF1FA383070897E700
:1078F000FF1FA380070897E7FF1FA387070897E7E5
:10790000FF1FA382071A6FF04FF389476312F70234
:1079100097E7FF1F83C787E19146638CD70863E031
:10792000F604638EE70C6369F70A05476380E70E88
:10793000FD5717E7FF1FA30FF70237074000B7E710
:1079400000E023A0E71801000100B78600401306FD
:10795000F0FC2381C60223A0E7106FF06FDB130752
:1079600020086382E7086362F70213071008E391B7
:10797000E7FC378700408347670293F7C70B93E71D
:1079800027002303F7026FF04FEB130730086389DA
:10799000E70213074008E39DE7F837870040834775
:1079A000270393F7C70B93E727002309F7026FF02C
:1079B000CFE8378700408347270393F73707F5B7AA
:1079C000378700408347E70293F7C70B93E7270009
:1079D0002307F7026FF06FE6378700408347E7021F
:1079E00093F73707F5B7378700408347A70293F728
:1079F000C70B93E727002305F7026FF00FE43787E3
:107A000000408347A70293F73707F5B73787004051
:107A10008347670293F73707ADB717950100130542
:107A2000A55A97700100E780C0BF97E7FF1F238D1D
:107A300007CED5B3179501001305055A97700100BD
:107A4000E78020BE97E7FF1F239007CE97E7FF1F31
:107A5000938747F203C40700894763F3870009440B
:107A60001374F40F29B613070002E393E7EC63994C
:107A7000090A638FF500930720026381F5081795C3
:107A800001001305E55897700100E780A0A14DB5EE
:107A9000179501001305055597700100E78060B840
:107AA0000144179B0100130B2B55A14AB3078A0011
:107AB00083C507005A85050497700100E780809E02
:107AC000E31654FF17950100130505B297700100E6
:107AD000E78020B517E4FF1F034444C511E497E78E
:107AE000FF1FA38607C261B48947E313F4E4854707
:107AF00017E7FF1FA30DF7C06FF02FD417E6FF1F86
:107B00000346B6C297E5FF1F83C525C2179501003E
:107B10001305054F97700100E780C0986FF0EFD113
:107B2000638FF50493071002E39BF5F497E5FF1FBD
:107B300083C5C5BF179501001305854E97700100D9
:107B4000E780409697E7FF1F23A647F597E7FF1FBB
:107B5000938707E3944383D7470017E7FF1F034743
:107B600087E217E6FF1F2321D6BC1D4497E6FF1FBF
:107B7000239EF6BA97E7FF1F238BE7BACDBA97E5A6
:107B8000FF1F83C5A5BA179501001305E54A977035
:107B90000100E780209197E7FF1FA38A07B697E7C8
:107BA000FF1F239307B86FF0EFF62547E388E79CA4
:107BB00019476391E702B786004023808602B7E742
:107BC00000E03707400023A0E7180100010013067A
:107BD00000FC41B31307100A6391E702B786004027
:107BE00023808602B7E700E03707400023A0E718AC
:107BF00001000100130680FCA9BB1307A009E38F55
:107C0000E7FC1307400AE38BE7FC13072002E38736
:107C1000E7960547E384E796B7E700E037074000BB
:107C200023A0E718E392099601000100B7860040FF
:107C300023808602130620FC29BB17E7FF1F03479A
:107C400077D36308F71E63E7E7029547630EF70EE5
:107C500099476308F704B786004023800602B7E718
:107C600000E03707400023A0E718010001001306D9
:107C7000A0FCC5B19307F005630AF700930750090C
:107C80006306F70093071002E317F7FCB7E700E07D
:107C90003707400023A0E71801000100B786004025
:107CA00051BF97E9FF1F83C9E9CC93070004CE8A2F
:107CB00063F43701930A000497E7FF1F938787DD7A
:107CC00003AA070013F4FA0F2286D28517E5FF1FD7
:107CD000130585A597600100E7806071B38789402F
:107CE000529417E7FF1F2307F7C897E7FF1F23A347
:107CF00087DA638E0902B787004023805703B7E60F
:107D000000E03706400023A0C6180100010003C7A9
:107D10002702134707042381E70203C727021377CB
:107D2000C70F2381E70223A0C6106FF06F9EB786AE
:107D3000004023800602B7E700E03707400023A099
:107D4000E71801000100FDB5378700408347370081
:107D500097E6FF1F83C696C393F70708D58FA30145
:107D6000F700B7064000B7E700E023A0D7180100EE
:107D700001001306A0FC2301C70223A0D7106FF057
:107D80002F9997E7FF1F938767D1A69783C70700AF
:107D900093F7F70FD9CF97E7FF1F83C7C7D0D1EB72
:107DA00017E7FF1F034717BD930700026313F70888
:107DB00097E7FF1F9387479703AB070097EAFF1FDB
:107DC00083CACA9617EAFF1F034A5A9697E9FF1F0C
:107DD00083C9E995D2875687CE865A8697E5FF1FD5
:107DE00083C5F5921795010013058526976001005C
:107DF000E780406B97E7FF1F23A467B997E7FF1F52
:107E0000238257B997E7FF1FA38E47B797E7FF1F56
:107E1000238B37B797E7FF1F238B878EB7E700E0E9
:107E20003707400023A0E71801000100B786004093
:107E3000D1B3B7E700E03707400023A0E7180100FF
:107E40000100B786004025B529472381E70209478D
:107E50002383E7022385E7022387E7022389E702DA
:107E60006FF06F8F03C76700118B6309079083C79B
:107E70005700918BB5CF17E7FF1F0347C7C2854750
:107E80006313F70697E7FF1FA38FE7AE97E7FF1F80
:107E9000238C079497E7FF1F238A07A097E7FF1F0C
:107EA000238807AC97E7FF1F238507AC97E7FF1FE1
:107EB000A38C079297E7FF1FA38A079E97E7FF1FF0
:107EC000A38807AA97E7FF1FA38507AA97E7FF1FC5
:107ED000A38C07AA97E7FF1FA38707BCB7870040BB
:107EE00011476FF06F8917E7FF1F2302F78279BFF1
:107EF000854717E7FF1F2309F78E17E7FF1F2307A3
:107F0000F79A17E7FF1F2305F7A617E7FF1F2302BE
:107F1000F7A669BF854717E7FF1F2307F78C17E709
:107F2000FF1F2305F79817E7FF1F2303F7A417E7A1
:107F3000FF1F2300F7A417E7FF1FA307078A17E710
:107F4000FF1FA305079617E7FF1FA30307A297E7E5
:107F5000FF1FA38007A28280411106C69700000080
:107F6000E78080FBB787004023800700130740FCB1
:107F70002386E7001307C004A386E70017D7FF1F77
:107F80001307877A2398E70017D7FF1F1307C77DCA
:107F9000239AE70017E7FF1F13074789239CE70091
:107FA00017E7FF1F1307C794239EE7002947238184
:107FB000E70209472383E7022385E7022387E702D5
:107FC0002389E702A3810700930600F8A380D70066
:107FD000930690022380D700FD562383D700238188
:107FE000E700B706400037E700E02320D71003C7BB
:107FF000170013671700A380E700B24097E7FF1F41
:108000002396079841018280411106C6970000001F
:10801000E78080F0B787004023800700130700FC4B
:108020002386E7003147A386E70017D7FF1F130712
:10803000A76F2398E70017D7FF1F1307E772239A4C
:10804000E70017D7FF1F1307677E239CE700294728
:108050002381E70209472383E7022385E702A381FF
:108060000700930600F8A380D700930690022380B0
:10807000D700FD562383D7002381E700B7064000D1
:1080800037E700E02320D71003C717001367170056
:10809000A380E700B24097E7FF1F2399078E4101B5
:1080A0008280F1679387072017E7FF1F232AF78C49
:1080B000854717E7FF1F2317F78CA14717E7FF1F17
:1080C0002303F78C97E7FF1FA38F078A97E7FF1F0C
:1080D000238C078A97D7FF1FA38B076297D7FF1FB1
:1080E00023870762814717D5FF1F13056562FD557A
:1080F00017D6FF1F130686622947B306F5002380B3
:10810000B600B306F600238006008507E397E7FE76
:1081100097E7FF1F2382079897E7FF1FA38E079615
:1081200097E7FF1F238B079697E7FF1FA385078419
:1081300097E7FF1FA383078497E7FF1F238E07821C
:1081400097E7FF1F2389078297E7FF1F238807828E
:1081500097E7FF1FA382078297E7FF1F238F078000
:1081600097E7FF1FA38B0792828017E7FF1F034744
:10817000879385476316F70017030000670003E93C
:1081800017030000670083DD411122C406C617E70C
:10819000FF1F0347479185472E8613F4F50FAA85E5
:1081A0006317F70417D5FF1F1305456C976001008F
:1081B000E780E02397D7FF1F238A076EB787004029
:1081C00023848702B7E600E03706400023A0C618E4
:1081D0000100010003C7A7021377C70F2385E70239
:1081E000B240224423A0C61001454101828017D528
:1081F000FF1F1305655B97600100E780401F97D75D
:10820000FF1F2383075EB787004023828702B7E6FC
:1082100000E03706400023A0C6180100010003C794
:1082200067021377C70F2383E7025DBF411106C6BC
:1082300097000000E78020E7B240410117030000EB
:108240006700E3F2411106C697F0FFFFE780C0C464
:1082500097D7FF1F83C75759A1CB97D5FF1F83C55A
:10826000C55889C917D5FF1F1305455897F0FFFF5B
:10827000E780009B97D7FF1FA388075697D7FF1F5C
:108280002384077037E700E0B70640002320D718A3
:1082900001000100378600408347660293F7370FDD
:1082A0002303F6022320D710B2404101828041C946
:1082B000D9C597D7FF1F83C7676DD1C3011122CCE2
:1082C0004AC84EC656C25AC006CE26CA52C42E89C5
:1082D000AA890144930A0004371B0300637724032F
:1082E000B3078940C207C183BE8463F4FA009304D4
:1082F0000004C204C180130A1BD497D7FF1F83C791
:10830000A74E9DE37D1A631C0A00F2406244D244EA
:108310004249B249224A924A024B0561828097F053
:10832000FFFFE78060B7D1BF338589002694A6851B
:10833000420497000000E78060E5418045B78280F5
:1083400097D7FF1F9387C77918429C4383D6450070
:108350000345070083C5C700035646006396A50082
:1083600083D5E700638DD502011106CE2386A700D1
:108370002397D700B705CF00DC4B9385757D0507A4
:108380007D162EC2230001003AC42316C100231714
:10839000D10099C30A858297F2400561828082806C
:1083A000DC4DDC4B81CFB7E70400904503A3870584
:1083B000914517D5FF1F0345E572028382806D71D9
:1083C0003C083EC6B707E500232291103EC8AA84A8
:1083D0003C083285232611103ECA23248110232015
:1083E00021112E8997300000E78020562A84979526
:1083F0000100938565C917850100130525B89760AD
:108400000100E780200AA28517950100130545D8D1
:1084100097600100E7800009294597600100E78027
:10842000400DB705CB009385757D6800971000005F
:10843000E780405FA285680097300000E7804043F6
:10844000014781467000CA85268597200000E78095
:10845000C08205CD2A84979501009385E5C21785D2
:1084600001001305A5B197600100E780A003A28574
:1084700017950100130585D297600100E7808002FF
:10848000294597600100E780C0068320C1100324BE
:10849000811083244110032901105161828097D7F4
:1084A000FF1F9387E76318429C43797122D406D655
:1084B0000348070083C807012A8483D64500035573
:1084C00046006396080183D82701638DD80223886C
:1084D000070105072399D7003708CC00DC4B1308A8
:1084E000787D3ACC1307F5FF42CA23080100231E0A
:1084F000E100231FD10099C7080832C62EC4829715
:108500003246A245228597000000E78080EBB250FA
:108510002254456182806D713C083EC0B707E5007A
:108520003EC23C083EC4232611102324811023227E
:108530009110231701002318010023190100231AA9
:108540000100231B010097B7FF1F83D7A7E799E31B
:10855000C167FD172316F10097B7FF1F83D7A7E662
:1085600091EB97D7FF1F9387A7579C439C43DC470A
:1085700083D7070017B4FF1F1304C4E4584C231714
:10858000F10083574400484B2318F10031E19795DF
:108590000100938565B6178501001305259E976038
:1085A0000100E78020F017950100130525B69760BC
:1085B0000100E78020EF294597600100E78060F324
:1085C0008320C110032481108324411051618280D3
:1085D00097B7FF1F83C777DF89EBB7E70400BC5766
:1085E00082975C4C23AA0700E1BFFD1797B6FF1FD7
:1085F000A38DF6DC03560701834704014C470A8527
:10860000230BF10097300000E780A02397D7FF1FCE
:108610009387074D9C430147814688430A866C0037
:1086200097100000E7806065AA8429C19795010032
:10863000938585AC1785010013054594976001006B
:10864000E78040E6A685179501001305E5AC976025
:108650000100E78020E5294597600100E78060E997
:10866000584CB7E70400BC57484B9DBF97B7FF1F56
:1086700083C7B7D5F5D7B7E70400BC4F104485458D
:1086800017D5FF1F0345054682971DBF5C4EDC4B87
:10869000B9CFB1CD411122C4178501001305058E54
:1086A0002E8497950100938565A306C69760010007
:1086B000E78040DFA285179501001305A5A8976004
:1086C0000100E78020DE294597600100E78060E235
:1086D000B7E704002244B24003A3870517D5FF1F64
:1086E00003454540130640069145410102838280BF
:1086F000411122C417B4FF1F130484CA1C4C06C6C0
:1087000089C7DC4399C34C488297584CB7E70400AB
:10871000BC57484B82975C4CB240224423AA0700C6
:108720004101828017B7FF1F130787C983470700DE
:108730009306F00B850793F7F70F63E9F60097B6FA
:10874000FF1F238FF6C6034507008280930700F8BA
:10875000FDB7835745006386071001114AC817B952
:10876000FF1F130929C652C4032AC90106CE22CC11
:1087700003274A0126CA4EC656C2F15735E31307EE
:10878000D00DFD57636EC704B7E9040083A709073E
:108790002A841305860042054181B284AE8A8297FD
:1087A000232AAA000325C9015C49A9E7979501007E
:1087B0009385C590177501001305457C97600100EE
:1087C000E78040CE17950100130505A097600100D2
:1087D000E78040CD294597600100E78080D1DD57D3
:1087E000F2406244D2444249B249224A924A3E850A
:1087F0000561828093874400B705CF002319F500F7
:108800009385757D310597100000E780A021032531
:10881000C90183456400310597300000E7804005B9
:108820000325C9012686D685310597300000E780EB
:1088300040017146A2854A8597600100E78020BB10
:10884000504419CA83A78905854517D5FF1F0345DD
:1088500065298297814769B797000000E780E0CBE0
:10886000D5BFFD573E858280411126C297B4FF1FB8
:10887000938444B5D84C22C437E404003C54484B9C
:1088800006C68297DC4C0323C4052244B2409244BE
:1088900023AA070017D5FF1F0345C52485454101BD
:1088A0000283411126C297D4FF1F938464239C4006
:1088B00006C622C44AC0D5C3DC43C5C35CC123007D
:1088C000B5002A84978501009385857A1775010084
:1088D0001305C56A97600100E780C0BC2945976011
:1088E0000100E78000C19C4023A4070023A20700E9
:1088F00097B7FF1F9387C7AADC4FDC4B91C7295559
:1089000097000000E78000DF97B7FF1F938787ABD2
:10891000DC4FDC4B89C797000000E78020F537E982
:1089200004008327C905894517D5FF1F0345851B0B
:1089300082978327C905914517D5FF1F0345851ADF
:1089400082979C4003A347016309030022852244C8
:10895000B2409244024941010283B240224492440F
:108960000249410182800111328506CE22CC26CAFD
:108970002E8497300000E78040FDAA84978501008F
:1089800093854572177501001305455F97600100D7
:10899000E78040B103078400035664008355440018
:1089A000A686178501001305E57B97600100E78027
:1089B00060AF294597600100E780A0B397B7FF1F1C
:1089C00083C7679E639D9700014597000000E7807D
:1089D00060D281450A8597000000E780C0ECF24034
:1089E0006244D244056182806D7123248110232664
:1089F00011102322911093F745002E8463870714EA
:108A00003C083EC0B707E5003EC23C083EC4231701
:108A100001002318010023190100231A0100231B60
:108A2000010097B7FF1F83D7A79799E3C167FD1789
:108A30002316F10097B7FF1F83D7A79691EB97D71F
:108A4000FF1F9387E7099C439C43DC4783D70700BC
:108A500017B7FF1F1307C7942317F100544F83570D
:108A600047002318F100DC4AA1E7978501009385B0
:108A7000A567177501001305655097600100E78031
:108A800060A2178501001305656897600100E78003
:108A900060A1294597600100E780A0A51345440027
:108AA0008320C110032481108324411051618280EE
:108AB00097B7FF1F83C7378F2555D9C3FD1717B643
:108AC000FF1FA302F68E03D6060183470701CC469B
:108AD0000A85230BF10097300000E78080D697D7F6
:108AE000FF1F9387E7FF9C4317B7FF1F1307478BB1
:108AF000978601009386866488430A866C009710E7
:108B00000000E7808017AA8451D9978501009385DA
:108B1000A55D177501001305654697600100E780A4
:108B20006098A685178501001305055F9760010011
:108B3000E7804097294597600100E780809B268564
:108B400097000000E78000BB91BF93F725009DC709
:108B5000B7E70400BC474146814528088297255560
:108B600097000000E78000B928089305F00F9700F0
:108B70000000E78040D3134524001DB793F715008C
:108B8000014599DF97000000E78020991345140004
:108B900001BF5C4D411106C688C317D7FF1F2321B3
:108BA000F7F4B7E7040083A70708170500001305CB
:108BB000E5E38297B24097D7FF1F2385A7F20145CF
:108BC0004101828001113335A000A307A100B7E75E
:108BD000040083A7471706CE1306F1008545130549
:108BE00050308297F240056182808280411122C418
:108BF00006C697D7FF1F83C767F0014489EF97B771
:108C0000FF1F83C7375E054499E717D4FF1F03444E
:108C1000A49D13441400228597000000E780C0FA49
:108C2000178501001305056609E417850100130582
:108C300065662244B24041011763010067008386E4
:108C4000797122D4A30F010037E40400832784172D
:108C500026D24AD006D6AA842E8913055030930511
:108C6000F10132C6829732468347F101931506011E
:108C7000C18185CB01452EC697000000E780C0F476
:108C800083274417B2454A86268582970545970073
:108C90000000E78060F3B2502254925402594561BB
:108CA0008280832744174A8626858297EDB7411133
:108CB0009397050122C406C626C2C1872E8463D4B9
:108CC0000702B7E40400FC5417A5FF1F0345857293
:108CD000829719C1BC5482972165218DB2402244EC
:108CE00092444101828093F715008DC7B7E70400D5
:108CF00083A7471A17A6FF1F1306C66E97D5FF1F37
:108D0000938505DF17A5FF1F0345C56E82971345A1
:108D10001400E9B793F7250099CFB7E70400BC4FDB
:108D200013060064894517A5FF1F0345A56C8297AC
:108D30001345240065B793F785009DC7B7E7040086
:108D400003A8871A1307401F97A7FF1F83C7876AC7
:108D5000814613064006994517D5FF1F035545DA8E
:108D60000298134584009DBF93F745000145BDD788
:108D7000B7E4040083A7041817D5FF1F035545D88F
:108D80008297BC4C13060064914517A5FF1F03454D
:108D9000656682971345440091B797D7FF1F83D725
:108DA00027D66398A70217D7FF1F231CB7D417D75E
:108DB000FF1F2319C7D417D7FF1F2316D7D42E861A
:108DC0001785010013054552BE8517530100670042
:108DD000636D178501001305A55217630100670035
:108DE00043840357450097D7FF1F83D767D1631A82
:108DF000F704C1674111F91722C417D7FF1F2321B8
:108E0000F7D037E4040097D7FF1F23AD07CE97D7DD
:108E1000FF1FA38507CE7C4C06C6894517A5FF1FFB
:108E20000345455D82977C4C914517A5FF1F03457F
:108E3000655C82972244B24041011703000067003D
:108E400023DB178501001305A54B175301006700AD
:108E5000437D7D15954763E2A71C17870100130723
:108E600027400A053A951C41011122CC06CEBA973B
:108E70002E8482871785010013050549975001004C
:108E8000E780207AA1A203C7250099476311F70262
:108E90002E8597000000E78000F583456400178564
:108EA00001001305654797500100E780A05F97B761
:108EB000FF1F23890732178501001305A5477DBFD2
:108EC00003C7250095476319F702C16717D7FF1F2E
:108ED000035707C3F91703D5A5006309F702B7E7DE
:108EE000040083A7C71782971785010013058545DE
:108EF00097500100E780E072854717B7FF1F2303F3
:108F0000F72E17850100130565468DBF97D7FF1F04
:108F10002398A7BE83D7E50097D6FF1F2393F6BEFD
:108F200083D7050197D6FF1F239EF6BC83D7250163
:108F300097D6FF1F2399F6BC97D7FF1FA38007BCC6
:108F4000631BE502B7E70400BC4F096613060690F1
:108F5000A14517A5FF1F0345E54982970356E40085
:108F60008355A400178501001305053F97500100A4
:108F7000E780405351B79307700F2316F100B7E70E
:108F8000040083A7870D17A6FF1F0346A6466C00A3
:108F900082974DF9854717D7FF1FA301F7B65DB735
:108FA000178501001305453DD1BD83C525009147B7
:108FB0006392F502178501001305853D9750010066
:108FC000E780206697000000E78080C2F24062449C
:108FD0000561828099476392F5022285970000001F
:108FE000E78060E083456400178501001305C53202
:108FF00097500100E780004BD1BF9547639AF50079
:1090000083471400E1F3178501001305A53ABDB5A8
:10901000178501001305853AE1BF82806D71232415
:1090200081102326111023229110328401CD89470B
:10903000630AF5028320C1100324811083244110A8
:10904000516182801785010013050538AE84975061
:109050000100E780005DA285268597C0FFFFE780BD
:109060000050C9BFB7E70400FC4728008297178566
:1090700001001305253697500100E780805A834789
:10908000810039C41307000B6380E7021387A7052B
:109090001377F70F8D4663EDE602A285280097D07F
:1090A000FFFFE780E0BE79B78547E3F587F88345A2
:1090B0009100177501001305A521B335B00097B7CE
:1090C000FF1F2383B7FA97500100E780A03D9DB7AB
:1090D00003479100A207D98F35671307D7556385DA
:1090E000E7086368F7022D671307B7556387E7063C
:1090F00031671307C755638AE70429671307A75524
:109100006394E702A285280097D0FFFFE78020F252
:1091100015B739679306E765638DD70663E9F600EF
:109120001307E7556380E706A28528003DB73D6732
:109130009306F7556386D7061307F766E396E7FEAF
:1091400097D0FFFFE780A00AF5B50146A285280069
:1091500097D0FFFFE780E0DAF1BDA285280097D025
:10916000FFFFE78000EBF9B58947E3F587EC93054E
:10917000E4FFC205C1811305A10097A0FFFFE780AE
:10918000E0024DBDA285280097D0FFFFE78020EBCD
:1091900055B5A285280097D0FFFFE780E0F559BDBF
:1091A00097D0FFFFE78060FE71B5411122C417A47C
:1091B000FF1F13046425AA86178601001306C60B39
:1091C0002285C14506C697500100E780C046035777
:1091D000440097A7FF1F938727242393E700035793
:1091E00064002394E700B24022444101828041118F
:1091F00006C697000000E78080FBB7E7040083A75E
:10920000871417A6FF1F13062620D5450145829710
:10921000B2404D4697A5FF1F93850520130570307A
:109220004101170300006700E3A161712324811A43
:1092300037E40400832704082326111A2322911AF5
:109240002320211B232E311917050000130565A6C5
:10925000829717A9FF1F1309E9199947854423002D
:10926000A900231CF100978501009385E50493076D
:10927000400617750100130565D0231CF10823086B
:10928000910097C9FF1F9389894697500100E78095
:10929000602183D50900178501001305E50097506B
:1092A0000100E7802020294597500100E7806024D5
:1092B00003D50900856997000000E78040EF832708
:1092C00044171008854513055030829783274417AB
:1092D00017A6FF1F13064614CD451305703082975D
:1092E0008327441717A6FF1F13060611B54513055C
:1092F0006030829783274417300889451305103161
:1093000082978327441730098945130520318297B6
:1093100083274415938509C80D45829783274415F3
:10932000938509C811458297A305910023069100F2
:109330002308910002CD230C0100832784163009F5
:109340009145130570408297832784161306B10058
:109350008545130500408297832784167000854554
:10936000130510408297832784163008854513051E
:1093700020408297832784161008854513055040A6
:109380008297832704157D558297832744137D5543
:1093900082977D5597A0FFFFE780002C8327440C20
:1093A000829797A0FFFFE78040078327841417A6C2
:1093B000FF1F13066605D5450145829789471306A9
:1093C000700F814528092306F1009790FFFFE78081
:1093D000C0D08D471306000881452808230CF108EA
:1093E0009790FFFFE78060CF9147230CF1009777BC
:1093F0000100938727AA984383C747003AC8230AE6
:10940000F10097D0FFFFE78040E5700085450545F6
:1094100097A0FFFFE780602B30099305700F094587
:1094200097A0FFFFE780602A3008930500080D45EC
:1094300097A0FFFFE780602910089545114597A088
:10944000FFFFE7808028C16717C7FF1F1307476B1F
:10945000F9171CC32322070017A5FF1F130545F9A1
:1094600097A0FFFFE78040258327C41D17C5FF1F76
:109470001305856782973C48034509008545829717
:109480008320C11A0324811A8324411A0329011A53
:109490008329C1195D618280C16717C8FF1F035806
:1094A0002866F9176301F8083DCDB5CD011126CA2C
:1094B000B7E4040083A7841222CC2E862315B100C2
:1094C00006CE2A8401478146ED45428582972AC609
:1094D00011ED17850100130525DF97500100E78086
:1094E0004014F2406244D24405618280FC44035639
:1094F000A100A28582972C0017C5FF1F0355456068
:1095000097A0FFFFE780002869DD1785010013059C
:10951000E5DC97500100E780C01083A7C412ED4539
:10952000280082977DBF8280411106C61DC98547EC
:1095300017A7FF1FA307F7EC354697A5FF1F9385D5
:10954000A5EB1305603097A7FF1F238D07EA97F05F
:10955000FFFFE780206FB240410117F3FFFF670074
:10956000236997A7FF1FA38E07E8F9B7C16717C53F
:10957000FF1F0355E558F9176307F500B7E7040027
:1095800003A3C71702838280854717C7FF1F2307DE
:10959000F756014517F3FFFF670003631793FFFFBB
:1095A000E70203AF2A8408452E89B28919C900C190
:1095B000971500009385A586610597300100E78027
:1095C000800181447D5A97100000E780E03963C72D
:1095D000A404814497100000E780003A63C8A40403
:1095E00097C7FF1F938747529C43DC47B307F94057
:1095F00091872302F400638309048327C900B3071A
:10960000F4409587A302F4001C4C89C79C4799C37A
:10961000228582971793FFFF6700C3AA5C441397C4
:1096200014008504BA972390470171BF1C48139713
:1096300014008504BA972390070069BF8327890027
:109640000547B307F4409587A302F400835704004D
:10965000638EE7028DC309476384E7040D47E395F2
:10966000E7FA978701009387A7291CCC9787010009
:109670009387072A11A8978701009387E7EF1CCCEF
:1096800097870100938747F05CC8BDBF97870100AB
:10969000938787DB1CCC978701009387E7DBEDB7C7
:1096A000978701009387872A1CCC978701009387AF
:1096B000E72AD9BF95E51793FFFFE702039F00460E
:1096C00018448347940075839D8B6317F7009710A8
:1096D0000000E78060B448C41793FFFF6700239F32
:1096E00082801793FFFFE702A39A13893500C164B4
:1096F00042094111AA890144F11413590901054A8B
:109700002EC697100000E7802026B2456348A400CB
:10971000014541011793FFFF6700C39A83A7090022
:1097200013171400BA9783D707006388B7006394B0
:10973000970063742A010504E1B70545D9BF179363
:10974000FFFFE7020394AA892E89328BB6843A8AF6
:10975000BE8A97A00000E78020FB71C9268597206C
:109760000000E78020098D4763E7A7007D55179328
:10977000FFFF6700839483DB440097100000E780BD
:10978000A0242A8497100000E780402593077400E6
:1097900031443305850263CDA70297100000E780AE
:1097A000A02297100000E78020222A849710000052
:1097B000E780C0229307740031443305850263C3F8
:1097C000A70497100000E78020209307450029A8F0
:1097D00097100000E7808020330585021307F017FB
:1097E0009307C017E35FA7FA2D55E3C277F9630427
:1097F0000B02D6865286A6854A8597200100E7800F
:1098000020BAB5B797100000E780401D33058502E8
:109810009307C5FFD1BF832749001385C90083D5AE
:10982000270097000000E78000EC61F581B76955DB
:109830003DBF97C7FF1F239BA72C97C7FF1F938789
:10984000A72C904381470C463307F500420741831C
:109850006393B70082805446139847008507C296E9
:109860002390E600D5B797C7FF1F9387E7299C434E
:1098700003C58700828017C5FF1F035525298280F5
:109880001793FFFFE7026382C1671387D7FF630B5C
:10989000E502636AA700F1176300F502014517931B
:1098A000FFFF6700C3821387E7FF6302E502FD172E
:1098B0001D8D13351500E5B797500000E780C026D1
:1098C0007D15C5BF97500000E78040FBD5BF97507E
:1098D0000000E78060F9EDB71783FFFFE702E37C44
:1098E0004111AA8401442EC697100000E780C008E9
:1098F000B2456348A400014541011783FFFF67009B
:10990000037D9C48131514003E9583570500E3859D
:10991000B7FE0504C9BF03485500814693F7F60F0B
:1099200063E5070181473E8582805845939756003D
:10993000BA9703D727006316B70003D70700E304DD
:10994000C7FE8506E1BF8346450001479377F70FC1
:1099500063E4D700814711A81C451316570005077B
:10996000B29703D60700E313B6FE3E8582801783C5
:10997000FFFFE702E37193170501C18797CAFF1F35
:10998000938A8A18635BF00883A70A00C0479C4744
:1099900003570400198D420541816368F5000144B5
:1099A00022851783FFFF6700E37112052A94CDBF5C
:1099B000DC4713944900014A3E94834744006341C5
:1099C000FA02014A834754006349FA028509C20931
:1099D00093D9090183A70A009847E3EBE9FCC1B7D3
:1099E0001C4413195A00A6853E994A859700000029
:1099F000E780C0EE05E1050AC9B75C4413195A00B7
:109A0000A6853E994A8597000000E78020ED19E180
:109A1000050A4DBFE30C09FA61B7AA8481495DBF0D
:109A20001783FFFFE70263681C452A8481E79307D9
:109A3000C5001CC51C44231204001CC09307F00F72
:109A400063EDB70093F5F50F228597200000E780BE
:109A500020E21783FFFF6700836793940501C167C6
:109A6000C18063F9F500A685228597200000E78074
:109A700040E5C5B7C18193F5F50F22859720000019
:109A8000E78000DFA685228597200000E78040E080
:109A9000C9B797C7FF1F93872707884382801C4554
:109AA00099C797C7FF1F23A1A706014582807D554F
:109AB000828097C7FF1F93872705984383474500F8
:109AC000484792073E9582801783FFFFE702E35DD8
:109AD000617100451C183EC6B70780013EC81C18BE
:109AE0003ECA8357440002CE02D002CC231EF100AE
:109AF000834784002A8902D22301F1023C083ED424
:109B000002D697000000E78000FB8357050023166C
:109B1000F10297500000E78060C42307A1025C4077
:109B200003556400F18313F717008347F1025205D0
:109B30005181F99BD98FA307F10297100100E780AB
:109B4000807539CDAA840355050097A00000E780F1
:109B500080BC83D704002AD26800231CF10083D77D
:109B60002400231DF1001C4803D647008C43972096
:109B70000000E78000CD8347B400CA861786010045
:109B8000130606868117A305F4006C004810972081
:109B90000100E780E0805D611783FFFF67002353CA
:109BA0002155D5BF1C45B1CF03C5A7008946135722
:109BB0006500630BD7028D46630ED70285466300AE
:109BC000D702130740063305E50203C7B700418BF0
:109BD00015CB83C7B700BD8B3355F5408280137515
:109BE000F5031307803EC5B709671375F50313071F
:109BF0000771D1BF372709001375F5031307077CD9
:109C0000D9B7014582801783FFFFE702034A03A902
:109C10008500630C09048347B900AE8493F7070EEF
:109C200085C303459900930520030D810505B30500
:109C3000B5028844610597300100E780E0A935A0AE
:109C40002E8597000000E78020F62A8419CD970022
:109C50000000E780605C8325C900B307B54063FA64
:109C600087002E94B305A440E9F51783FFFF670032
:109C7000034685457DBF1783FFFFE70203432A8420
:109C800003D50500011132C636C43AC22EC002CA3D
:109C900002CC02CE97A00000E780E0A782452ACA46
:109CA00022852ECC97000000E780E0E003570500F6
:109CB000231EE10097500000E78040AAA2463246EA
:109CC0009247230FA10036874C08B28622850146B1
:109CD00097000000E780E0A605611783FFFF67009B
:109CE000033F1783FFFFE702433C61711C183EC628
:109CF000B70780013EC81C183ECA3C0800453ED448
:109D0000AA8402CC02CE02D002D202D69700000072
:109D1000E78060DA8357050035592316F102975022
:109D20000000E780A0A32307A10209C483574400D1
:109D300081EB21594A855D611783FFFF6700233955
:109D4000035564005205518197100100E780A0542B
:109D50002A8965D18347B40093F7070E99C7130585
:109D6000840197300100E780609983574400231EE7
:109D7000F100834784002301F1025C400355090090
:109D8000D98313F7070883471102231CA10093F717
:109D9000F707D98FA300F10283572900231DF10093
:109DA0005C40F18313F717008347F102F99BD98FC9
:109DB000A307F10297A00000E780E0952AD235D9E9
:109DC000834794006800139757008347B400FD8BC6
:109DD000D98FA305F4001C4803D647008C43972075
:109DE0000000E78000A6A687177701001307475FEA
:109DF000740005464C10268597000000E7806094AB
:109E00002A890DD98347B400A685FD8BA305F400EC
:109E100097000000E78060DF31BF1783FFFFE70294
:109E2000C328832485FE2A844111268597000000DB
:109E3000E78080D7834734FF93F7070E8DCB2AC680
:109E4000268597000000E78060C809CD834734FF6E
:109E5000B245FD8BA309F4FE91C522859730010020
:109E6000E780808741011783FFFF670043267DD984
:109E70008327C4FF2685829775F5834734FF93F7C0
:109E8000070E91C7228597300100E78020870325C0
:109E900084FE97000000E78000E5E9B71783FFFF25
:109EA000E702A31D9C4141112A8903C70700894786
:109EB0002E84935667006380F6040D466388C604BB
:109EC0009307F0076304F7022E8597200000E780D0
:109ED000C0A7AA848149C16B130C490097C7FF1F13
:109EE000938787C29C43984763E4E9044101178341
:109EF000FFFF6700431C03D745008547E3F8E7FEF3
:109F00002E8597200000E780A0A9E1B703D7450080
:109F1000E3FEE7FC2E8597200000E78000A3AA84DB
:109F2000228597200000E78060A4C204C98C5DB739
:109F3000DC470355A900139A49003E9A931705017F
:109F4000C187635DF00083570A006397A70263E748
:109F500074038327CA00034D5A002DA0A16721670F
:109F6000A98F1307F7EFE374F7FE639709009700D3
:109F70000000E780209161FD85098DB783278A0065
:109F8000034D4A00835DA90003576900216A138BC2
:109F9000C7003AC6814A33CA4D01631E5D0197C7A7
:109FA000FF1F9387E7B69C43E1DBA286628681456B
:109FB00026858297D1B7A1679387F7EF930C4BFF64
:109FC00063F24703B2455A8597F0FFFFE780A0711F
:109FD0000DC103278B00104709CE10436382C402D2
:109FE0003107D5BFEE85668597000000E780008FBA
:109FF00071F993861A0093FAF60F130B0B0271BFD7
:10A00000835644005C43E3E9F6F622853AC697108E
:10A010000000E780807DA1679387D7042A8A035DCB
:10A020004400324763E897008347D90093E707F875
:10A03000A306F9001C4766852286E2858297C167E0
:10A040000844FD17337AFA00529508C02312A40180
:10A0500025B797C7FF1F938727AB9843814715C341
:10A060001447814763FFD500939745004C47BE9541
:10A0700019C903C7550081476375E600DC4516061C
:10A08000B2973E85828003C745008147E37BE6FEA9
:10A0900016069C45F5B71783FFFFE70263FFAA8901
:10A0A0002E8A814497CAFF1F938A0AA683A70A00B3
:10A0B000984763E6E4001783FFFF6700A300DC47CF
:10A0C0001394440001493E9413BB14008347440099
:10A0D000634BF900014913BB140083475400634FDD
:10A0E000F9008504E1B70844931759005287DA86CE
:10A0F0000146A2853E9582990509C9BF4844931738
:10A1000059005287DA860546A2853E95829905094F
:10A11000E9B71783FFFFE70243F9814517F5FFFF12
:10A120001305054897C7FF1F2392079E970000005D
:10A13000E780A0F61783FFFF670063F997C7FF1F4B
:10A140009387879C9C4395C31783FFFFE702E3F542
:10A15000814517F5FFFF1305A54497000000E78030
:10A16000C0F31783FFFF670083F682801783FFFF2A
:10A17000E70203F237E40400832784124111231518
:10A18000E100AE893289368A3A8681460147ED453B
:10A19000AA8482972AC621C90356A100D285974076
:10A1A0000100E780C0248327C413CE8526858297CB
:10A1B000058905C98327440D2314210101462C007C
:10A1C000268582972A8401C9B7E7040083A7C712AE
:10A1D000ED4528008297228541011783FFFF670024
:10A1E00063EE4944D5B76554FDB75C41FD175CC1CA
:10A1F00082801783FFFFE70243EBB7E70400FC5FB1
:10A20000829795473305F50281450D811783FFFF3E
:10A210006700E3EB1783FFFFE70223E9B7E70400DA
:10A22000FC5F829795473305F5020D811783FFFF89
:10A230006700E3E91783FFFFE70223E7B7E70400BE
:10A2400083A7870B0355050082971783FFFF6700DD
:10A2500003E81783FFFFE70243E503550500328754
:10A26000AE861796FF1F0356462197C5FF1F93859D
:10A27000658A97000000E780A0EF1783FFFF670063
:10A2800003E51783FFFFE70243E2B7E7040083A774
:10A29000C71782971783FFFF670063E31783FFFFEA
:10A2A000E702A3E0B7E7040083A7871397C5FF1F62
:10A2B00093854586829701451783FFFF670023E159
:10A2C0001783FFFFE70263DEB7E7040083A7C71F1A
:10A2D00081451795FF1F0355451682971783FFFF8A
:10A2E0006700E3DE1783FFFFE70223DCB7E7040024
:10A2F00083A7871397C5FF1F9385C5828297014562
:10A300001783FFFF6700A3DC1783FFFFE702E3D992
:10A31000B7E7040083A7C71F81451795FF1F0355A3
:10A32000C51782971783FFFF670063DA1783FFFF64
:10A33000E702A3D72E8597800000E780E0AF9780E3
:10A340000000E780E0EC1783FFFF670043D8178326
:10A35000FFFFE70283D597800000E780E0F61783D0
:10A36000FFFF6700C3D65C49E1175CC95CC5835732
:10A370002501A1072319F50083570501A10723181B
:10A38000F5008280F1473305F50297B7FF1F9387E9
:10A39000677B9C433E9582808D476315F60803D703
:10A3A0004600854763F0E7081783FFFFE702E3CF26
:10A3B000368536842E8997100000E780005929C918
:10A3C0008357440093140501C18063E397042285F9
:10A3D00097100000E7806057FD1423129400930744
:10A3E000A0026300F5029307B0026307F50293072A
:10A3F0009002631FF500228597000100E780C08569
:10A4000001A80146CA85228597A00000E78060B0B8
:10A410001783FFFF6700A3CB228597100000E7801A
:10A42000C003FDB7828097B6FF1F9386E6719C42FA
:10A43000014599CF9843D44217B6FF1F2326E670F3
:10A440006396D70097B6FF1F23A2E6701385C7FE59
:10A4500082801783FFFFE70243C597000000E78073
:10A46000A04B714433058502914597900000E78029
:10A4700020E911E565551783FFFF670043C597B7CE
:10A48000FF1F23AFA76A97000000E780E04833056D
:10A490008502914597900000E78080E661DD97B7DF
:10A4A000FF1F23A1A76A97000000E780E04697B747
:10A4B000FF1F2391A76897000000E780E04597B74A
:10A4C000FF1F239AA766977701009387A7F617B710
:10A4D000FF1F2325F76697070000938707E917B743
:10A4E000FF1F232BF764014579B71783FFFFE702AE
:10A4F000C3BBAA8517B5FF1F1305C56397100000DE
:10A50000E780C05B1783FFFF670063BC1783FFFF13
:10A51000E702A3B997000000E78060FD97100000F4
:10A52000E780405B97B7FF1F938707629C4391CFFB
:10A530001387C7FE19CB83D5C7FF17B5FF1F1305B8
:10A54000256197200100E78020191783FFFF67002E
:10A5500003B81783FFFFE70243B597000000E780C9
:10A56000C0EC09CD834785002A8493F7070499EB53
:10A570000355E50097000000E78080F91783FFFF8F
:10A580006700E3B48347C5009304450117B9FF1F73
:10A590001309895B85E3832709005CC997B7FF1F0F
:10A5A00023A4975A83274900F1FB97B7FF1F23AFD6
:10A5B0009758E9B7FD172306F5006105978000005D
:10A5C000E780C0D68307840063CB070483478400F9
:10A5D00093E707F82304F400B7E704009C5F829731
:10A5E0004205A94741813375F5028347840093F7FB
:10A5F00007FCC98F2304F4008347D4003E951C4018
:10A600002318A40089CF984319CB8347C400504036
:10A61000814585073305F50242054181029783276D
:10A6200009005CC897B7FF1F23A0975283274900F2
:10A6300089E797B7FF1F23AB97508347C4009DDF7F
:10A640008355040117B5FF1F13058550972001009E
:10A65000E780800825B71783FFFFE70203A597B7B8
:10A66000FF1F938727749C4701448583858B85E36F
:10A67000AE84B2853A8697100000E780804B2A842A
:10A6800019C597100000E780C041829408CC22854C
:10A690001783FFFF6700A3A31783FFFFE702439F12
:10A6A00041112E8932C6AA8997000000E780C03187
:10A6B000324713060502CA86970500009385C5CC6C
:10A6C00017B5FF1F1305054797000000E780E0F866
:10A6D0002A8425C99304C50097000000E780E04163
:10A6E0001946AA85268597100000E78080158545C4
:10A6F000268597100000E78060111775010013058B
:10A7000025D14E9583450500268597100000E780EA
:10A7100020165C4831468145A1075CC85CC483575C
:10A720002401E1172319F40083570401E1172318CA
:10A73000F4001C4C3E859780FFFFE780009AA3043D
:10A740002501228541011783FFFF6700A397178327
:10A75000FFFFE70283954111AA842EC632C49710E9
:10A760000000E7806036004DB245224683478400F2
:10A770000CC050C093F7F70393E707042304F400D9
:10A7800023180400268597100000E7808031834756
:10A790009400A9462317A40013D7370005073307F1
:10A7A000D7029D8B85072306F400A306E40083C728
:10A7B0000401D8488507230FF7FE17B7FF1F1307BB
:10A7C000A7385843232A04009307440129E317B705
:10A7D000FF1F232DF73617B7FF1F2327F73617B4B0
:10A7E000FF1F1304E436228597200100E78000E173
:10A7F0001C44858B5D8D19E58145228597200100DC
:10A80000E78080ED41011783FFFF6700438C1CC385
:10A8100017B7FF1F232CF732D9B71783FFFFE702C3
:10A82000C38897050000938565B701459700000030
:10A83000E78000B001451783FFFF67004389178356
:10A84000FFFFE702838697000000E78080B0178350
:10A85000FFFF6700C3878347C500A5E31783FFFF9A
:10A86000E702A3842A840355E50097000000E780EF
:10A8700000C821C18347840093F7F7FB2304F40049
:10A880001C4091C7DC4381C74C400145829797002B
:10A890000000E78080B917B5FF1F1305652B9720CF
:10A8A0000100E780A0E50355E40097000000E78081
:10A8B00020C61783FFFF6700838182801773FFFF25
:10A8C000E702A37E97B7FF1F93870728970500002D
:10A8D000938565C817B5FF1F1305852723A00700BB
:10A8E00023A2070097200100E780E0CE1773FFFF47
:10A8F0006700E37D1C4D91CFDC4381CF1773FFFFD1
:10A90000E702A37A8345070082971773FFFF67006A
:10A91000037C828097B7FF1F9387C7259C4303C59D
:10A920000700828097B7FF1F9387C7249C4303C506
:10A930001700828097B7FF1F9387C7239C4303C5E7
:10A940002700828097B7FF1F9387C7229C4303C5C8
:10A950004700828097B7FF1F9387C7219C4303C599
:10A960003700828097B7FF1F9387C7209C4303C59A
:10A970005700828097B7FF1F9387C71F9C4303C56B
:10A980006700828097B7FF1F9387C71E9C4303C54C
:10A990007700828097B7FF1F9387C71D9C4303C52D
:10A9A0008700828097B7FF1F9387C71C9C4303C50E
:10A9B0009700828097B7FF1F9387C71B9C4303C5EF
:10A9C000A700828097B7FF1F9387C71A9C4303C5D0
:10A9D000B70011E11D45828097B7FF1F9387871944
:10A9E0009C4303C5C700828097B7FF1F93878718D2
:10A9F0009C4303C5D700828097B7FF1F93878717B3
:10AA00009C4303C5E700828097B7FF1F9387871693
:10AA10009C4303D50701828097B7FF1F9387871553
:10AA20009C4303C52701828097B7FF1F9387871434
:10AA30009C4303D54701828097B7FF1F93878713F5
:10AA40009C4303D56701828097B7FF1F93878712C6
:10AA50009C4303D58701828097B7FF1F9387871197
:10AA60009C4303C5A701828097B7FF1F9387871078
:10AA70009C4303C5B701828097B7FF1F9387870F59
:10AA80009C4303C5C701828097B7FF1F9387870E3A
:10AA90009C4303C5D701828097B7FF1F9387870D1B
:10AAA0009C438857828097B7FF1F9387A70C9C43CE
:10AAB00003D5C702828097B7FF1F9387A70B9C43DC
:10AAC00003D5E70219E11305800C828097B7FF1FB9
:10AAD0009387470A9C4303C50703828097B7FF1FEC
:10AAE000938747099C43C85B828097B7FF1F938772
:10AAF000E7078843828097B7FF1F938767078843DC
:10AB0000828019E17D558280F5DE984265DFFDD9AE
:10AB100017B7FF1F130707291847AA877155058B19
:10AB2000631D072403C507001547E37DA7FC03C782
:10AB300037001305F0057D171377F70FE364E5FC85
:10AB400003C35700E30003FC83C86700E38C08FAE3
:10AB500003C77700494579171377F70FE364E5FAE0
:10AB600003C7A70011481305F7FF1375F50FE36B33
:10AB7000A8F803CE97000D481305FEFF1375F50FD7
:10AB8000E362A8F803C8B7006309080065181378E2
:10AB9000F80F1305600DE36705F703C5C700794893
:10ABA00079151375F50FE36FA8F403C8D7000D45A9
:10ABB0007D181378F80FE36705F503D80701930EA6
:10ABC00040175118420813580801E3ED0EF303C86B
:10ABD000E7007D181378F80FE36605F303C8270133
:10ABE0007D181378F80FE36F05F103C88700C54E91
:10ABF00075181378F80FE3E70EF103D86701856E37
:10AC0000938EBEE06D18420813580801E3EC0EEF76
:10AC100003D847016D18420813580801E3E40EEF0A
:10AC200003D887017918420813580801E36C05ED31
:10AC300003C8A7017D181378F80FE36505ED03C578
:10AC4000B7011D487D151375F50FE36DA8EA03C51F
:10AC5000D701714879151375F50FE365A8EA03D597
:10AC6000E7011308E00F7D1542054181E36CA8E878
:10AC700003C50702494879151375F50FE364A8E881
:10AC8000C85301C937C834005915130858BFE36BBE
:10AC9000A8E603A8870237C53400130555BF591825
:10ACA000E36205E717B5FF1F2324C5EC03C60501C2
:10ACB00017B5FF1F2320F5EC0545E375C5E403D860
:10ACC0002501D04933760603E31E06E203C61501CB
:10ACD000E30A06E217B6FF1F232AB6E883C527005A
:10ACE00001466387A50003C61700F1453306B60287
:10ACF00083C707039305C00272971A071307C70596
:10AD000016031A9796084697B387B70241553E97A0
:10AD10003297420741836362E8061773FFFFE70239
:10AD2000C338368597800000E780A068970001004F
:10AD3000E78020482A8497A00000E780805A2A9460
:10AD400097F00000E78060262A9497900000E78043
:10AD5000A0812A9497F0FFFFE780E06F2A94974044
:10AD60000000E78060932A9497700000E780A09C21
:10AD700022951773FFFF6700833582801773FFFFEB
:10AD8000E702A3324111A307A10097A00000E780CA
:10AD9000A0C59305F100170500001305E5B597F070
:10ADA000FFFFE780802F014541011773FFFF670018
:10ADB00003321773FFFFE702C32C17B4FF1F1304FE
:10ADC00064FE0328840079599368180097B4FF1F24
:10ADD00023AE14FD1378180063100802BA84BE89EC
:10ADE000368B328A2E89AA8A97F0FFFFE780E0A788
:10ADF0007D15269519E531594A851773FFFF6700C0
:10AE0000C32B97F0FFFFE78040A67D152695A1672D
:10AE1000E353F5FE97B7FF1F9387C72F98433E8CE8
:10AE2000814B01CB014597F00000E7802044933B24
:10AE300015004A85DA865686D28597900000E7800D
:10AE4000C04D2A8911CD1C44F99B17B7FF1F232F32
:10AE5000F7F483270C00CDD3E3800BFA829769BF08
:10AE6000268597B7FF1F23A107F497F0FFFFE78020
:10AE7000809C4146CE8517B5FF1F130525FC9730F2
:10AE80000100E780C05697D00000E7804099032575
:10AE9000040B97D00000E780009D054597D0000087
:10AEA000E78000A4054597000000E78060EDA9B7A2
:10AEB00097B7FF1F938707EF9C47858BEDC71773E5
:10AEC000FFFFE702831E17B5FF1F130565F597B750
:10AED000FF1F23A907EC97B7FF1F23A707EC97B71E
:10AEE000FF1F23A507EC97200100E78020819750E2
:10AEF0000000E780E0F597100100E780A04C971074
:10AF00000100E780A05297B7FF1F938727E89C4373
:10AF100091C7054597800000E780402097B7FF1F45
:10AF2000938787D09C4399C741657D159770000032
:10AF3000E78040A297F00000E780E03D97D0000056
:10AF4000E780808F97B7FF1F9387C7FA9C431397BB
:10AF500017016356070097F00000E78000AD97B730
:10AF6000FF1F23AD07EC97B7FF1F23AB07EC97B785
:10AF7000FF1F23A907EC97B7FF1F23A707EC970034
:10AF80000000E780008C97000000E780007297F0D7
:10AF9000FFFFE780401897F00000E78040D6177366
:10AFA000FFFF6700C312828097B7FF1F938787DF79
:10AFB000884382801773FFFFE702230F978000000A
:10AFC000E780607597800000E780C0771773FFFF08
:10AFD0006700E30F1773FFFFE702830B2A849304D4
:10AFE000140201112E85B289A685214636C63A89FA
:10AFF00097300100E780403D0DE9B24638082686CB
:10B00000CE851305940497500000E78060412146E7
:10B010002C084A8597300100E780003B1335150066
:10B0200005611773FFFF6700E3090145D5BF17737B
:10B03000FFFFE70283079305450617B5FF1F1305BA
:10B04000A5B397100100E78020691773FFFF670021
:10B0500003081773FFFFE702430541112EC697F05F
:10B06000FFFFE780601BB24588C141011773FFFFF6
:10B070006700E3051773FFFFE7028301AA842E84AC
:10B0800097800000E780006CAA898545228597009B
:10B090000000E780E07D83C7E4011389940899E309
:10B0A00013890403CE85228597000000E780407C49
:10B0B000214693051902228597000000E7806078F9
:10B0C00097B7FF1F938707CE8C4322859710000008
:10B0D000E780C08221469385840222859700000084
:10B0E000E78020761773FFFF6700C3FD1773FFFF2C
:10B0F000E70223F9397197F00000E780E0B4930587
:10B10000400661E997800000E78000606302051453
:10B1100097B7FF1F83C707A813B7170097B6FF1F7E
:10B12000238AE6A6014499CFC16417B9FF1F13090A
:10B1300069C79309400EFD1497000000E780C086A0
:10B140006342A40A97F0FFFFE780000D4169B72929
:10B150000900096AFD7A2A8B81447D199389F97B5C
:10B16000130A0A71938A8AC797000000E780C08398
:10B1700063D7A4041304400EB387840217B7FF1FDC
:10B18000130747C20324070B3E948357C40163820D
:10B19000270B18403307EB4063EAE900834744007C
:10B1A0008507B3874703D6976365F708014681454E
:10B1B000094597F0FFFFE780604EAA8B29E597408D
:10B1C0000000E780808385476317F50689659385CE
:10B1D000057117B5FF1F1305259A97100100E78029
:10B1E000A04F95A0B30734030327090BBA9703D7E1
:10B1F000C7016308970003C75700A3820700238293
:10B20000E700050415BF9305C500228597000000DF
:10B21000E78080E65E85228697650100938585201C
:10B2200097F0FFFFE780E0525E8597100000E7800F
:10B23000608A850415BF97B7FF1F9387A7B69C4701
:10B240008D83858BC1F721611773FFFF6700E3E6EC
:10B2500001468545094502D002D202D402D697F0B4
:10B26000FFFFE780A043AA8479DD97F00000E78024
:10B27000E09C1389C4002A8481454A859700000018
:10B28000E780005F0C4041464A8597000000E78058
:10B29000405B832944006385090C4E8502D802DA9D
:10B2A00002DC02DE97300100E78060402ACE1410F5
:10B2B00005462C0808184ECC97500000E780E00A9D
:10B2C0001375F50F51ED8355840093E525004A85EC
:10B2D00097000000E780E05E11460C104A85970059
:10B2E0000000E7800056014697650100938505142C
:10B2F000268597F0FFFFE780C04526859700000070
:10B30000E780407D5C40A1D3014685450D4597F01F
:10B31000FFFFE780A038AA841DD548401389C400E8
:10B3200097300100E780A0382AC64A8597000000C0
:10B33000E780404C3246636FC5004C404A85970019
:10B340000000E780005001468145268597F0FFFF09
:10B35000E7802040268597000000E780A077E5B5CC
:10B3600083558400ADB71773FFFFE70203D497B787
:10B37000FF1F938727A39C471DC193E7870017A54D
:10B38000FF1F1305657F17B7FF1F2321F7A2971033
:10B390000100E78040321773FFFF670043D3DD9B56
:10B3A00017B7FF1F2324F7A097300000E780E06461
:10B3B0007DF117A5FF1F1305257C97100100E7807D
:10B3C000E033D1BF1773FFFFE702A3CB4169AA891E
:10B3D0002E8AB28A368BBA8B814417BCFF1F130C9E
:10B3E0006C9C930C400E7D1997F0FFFFE780C05BCB
:10B3F00063C4A40001443DA03384940383270C0B51
:10B400003E948357C401638627055A87D6865286A1
:10B41000CE851305040397000000E780E0BB01C957
:10B4200023800B0022851773FFFF670003C9834742
:10B43000F40185C35A87D6865286CE8513059408B3
:10B4400097000000E78040B909C585472380FB00CD
:10B45000D1BF850451BF835745006380071E177312
:10B46000FFFFE702E3C201112A8497000000E78092
:10B47000C04D09C985476309F50605611773FFFFCC
:10B48000670043C497E00000E780007C7DF58357A8
:10B4900044004947ED9BE392E7FEC14522859700B2
:10B4A0000000E7804033AA84228597000000E780EF
:10B4B000204F0357440002CE91472A89631AF700B0
:10B4C000228597000000E780A0513C082ACC3ECEA0
:10B4D00097E00000E78080765C55C5D374084A8603
:10B4E000A6850545829751BF03574400D147E3F62F
:10B4F000E7F8032A0400C169014997BAFF1F938A3C
:10B500006A8A130B400EFD1997F0FFFFE780C049D0
:10B51000634FA90E2285032A040097000000E780EC
:10B52000C042A1452A89228597000000E780A02A11
:10B53000AA84228597000000E780804A14402A866A
:10B54000AA8978082685CA8597000000E780C0E7A9
:10B55000AA8405D503C7F40189476315F70083471B
:10B56000C10181DF5546D285138564009730010003
:10B57000E780E0E7014597800000E780C01901C53A
:10B5800083D7C401A5E797B7FF1F9387A7819C477F
:10B5900093551900858913D73700058B01CF89830F
:10B5A000858B6399B70001452EC697000000E780A0
:10B5B000C0DBB2454E8597800000E780601F0346E0
:10B5C000C1012A8493751900268597900000E780B1
:10B5D000E03935C1268597800000E780E018268590
:10B5E00011C0014597800000E780004C97300000B3
:10B5F000E780A0408547E312F5E883C754001307AE
:10B60000F00FE38CE7E68507A382F400BDB5B30431
:10B61000690383A70A0BBE9483D7C401638B3701E8
:10B620005546D2851385640097300100E780C0D964
:10B6300055DD0509D1BD5DD86DB782801773FFFF59
:10B64000E70203A597800000E780000C05C1C164F4
:10B65000014417A9FF1F1309E9749309400EFD1453
:10B6600097F0FFFFE7804034634EA40017A5FF1F4B
:10B670001305855097100100E780E0031773FFFF63
:10B68000670043A4330534038327090B3E95835792
:10B69000C501638897002312050097800000E780AA
:10B6A000A00C050475BF97A7FF1F9387A76F9C4742
:10B6B0008D83858B8DE31773FFFFE702039F17A52B
:10B6C000FF1F1305654B97100100E78020031773D8
:10B6D000FFFF6700C39F82801773FFFFE702E39CB1
:10B6E000970500009385C5A017A5FF1F1305C54842
:10B6F00097100100E78020EE1773FFFF6700239D7E
:10B700001773FFFFE702639A8841B7E70400BC5B49
:10B71000050542054181829709C585472300F5004B
:10B7200005051773FFFF6700839A83C7F5FF2E8512
:10B730008507A38FF5FE828083C7F5FFFD1793F77A
:10B74000F70FA38FF5FE99EF1773FFFFE702E3955D
:10B75000B7E70400BC571385F5FF82971773FFFF07
:10B760006700E39682801C41035745008D8FBA9590
:10B770001CC12312B5003E85828093D78500A205A7
:10B780001441DD8D835745001387E6FF18C18907F3
:10B790002312F50013D685004111238FB6FEA38F27
:10B7A000C6FE4101828018419307F7FF1CC18357F1
:10B7B000450085072312F500A30FB7FE828083574B
:10B7C00045008D8F2312F5001C41BE950CC12E85BE
:10B7D0008280AA8703D7470008410D8FAA9523923C
:10B7E000E7008CC38280184108453305A74082805A
:10B7F00083574500035765001D8F1C41084533855D
:10B80000A7403305A74082801773FFFFE702E38953
:10B8100041112EC62A8497000000E780A0FDB245A2
:10B820006373B50001A0835744000840BE952312FE
:10B83000B4003E9541011773FFFF670043891773FA
:10B84000FFFFE702838641112E84B28532C697003E
:10B850000000E780A0FB3246A28597300100E78018
:10B8600000B941011773FFFF670063861773FFFF7D
:10B87000E702A3832E84854597000000E78000F946
:10B88000230085001773FFFF670063841773FFFFB2
:10B89000E702A38141112317B100894597000000F9
:10B8A000E780C0F68347E1002300F5008347F100FD
:10B8B000A300F50041011773FFFF67004381176381
:10B8C000FFFFE702837E93D78500A2054111DD8D3E
:10B8D0002317B100894597000000E78020F38347D4
:10B8E000E1002300F5008347F100A300F5004101CA
:10B8F0001763FFFF6700A37D1763FFFFE702E37A8B
:10B900001397850193D78501C166938606F0D98F79
:10B9100013D78500758FD98FA2053707FF00F98DE2
:10B920004111DD8D2EC6914597000000E78000EEA5
:10B930006C00114697300100E78060AB410117634E
:10B94000FFFF6700C3781763FFFFE70203761C4120
:10B95000854503C4070097000000E78080E6228544
:10B960001763FFFF6700A3761763FFFFE702E37328
:10B970001C414111894503C7070083C717002307EE
:10B98000E100A307F10097000000E78080E3035582
:10B99000E10041011763FFFF670063731763FFFF57
:10B9A000E702A3701C414111894503C7070083C703
:10B9B00017002307E100A307F10097000000E780CC
:10B9C00040E08357E100410113D58700A2075D8D58
:10B9D000420541811763FFFF6700636F1763FFFF35
:10B9E000E702A36C0C4141112A841146680097308C
:10B9F0000100E780C09F9145228597000000E78005
:10BA000040DCB247C166938606F01397870113D5D1
:10BA10008701598D13D78700758F598DA207370776
:10BA2000FF00F98F5D8D41011763FFFF6700236AF7
:10BA30001C45BE950CC18280AE87944391E6584167
:10BA400001EF0CC15CC1828003C757001367170068
:10BA5000A382E700B687D5B70CC3EDB7AA87084124
:10BA600019CD1841D44398C36313D500D8C32A878E
:10BA7000034657009376160081E623200700828054
:10BA8000944381CA8C4203A847008CC36393060188
:10BA9000CCC3799A14C3A302C7003687D1BF1C4513
:10BAA000DC471D8DB777DBB6938777DB09853305D8
:10BAB000F502420541818280F147B385F502484590
:10BAC0002E9582808347450085072302F5008280FA
:10BAD0001763FFFFE702635D2A8409E41763FFFF32
:10BAE0006700E35E83474400F5DBFD1793F7F70F2C
:10BAF0002302F400E5F71C4403D727000507239130
:10BB0000E700DC4399C3228582974C4889CD83475F
:10BB10005400898B99E71C4422859C479C439C4791
:10BB20008297232A04000040232004007DB7176376
:10BB3000FFFFE70283578357250041112EC681EB93
:10BB40000144228541011763FFFF670043580357F3
:10BB500005008147F146E305F7FEB385D70240456E
:10BB600085072E948345440008C4F5F5B247AA849E
:10BB700081E7232A040009A81C456C0022859C4308
:10BB80009C43829748C84DDD85472312F400B24795
:10BB900023200400231804002319F4005C485CC42B
:10BBA00083D72400FD172391F40061BF1763FFFFC3
:10BBB000E702A34F97A7FF1F938707FE884323261B
:10BBC000050023240500410597100100E78000B31C
:10BBD0001763FFFF6700A34F1763FFFFE702E34C04
:10BBE00017A4FF1F130444FB1C40411199CF9C472D
:10BBF0002300B5002AC65CC197000000E78040FB27
:10BC00001C40DC4399C33245829741011763FFFF13
:10BC10006700E34B0347450029E3584DAA877D554C
:10BC20001DCF1763FFFFE70243481CC3DC4797A6FD
:10BC3000FF1F23A3E6F6F156130507012390D70053
:10BC4000970500009385050297100100E780A098F2
:10BC500001451763FFFF670083477D55828082801F
:10BC60001763FFFFE7026344011161468145280025
:10BC70009760FFFFE780604697A7FF1F9387C7F194
:10BC80009C4328009305F00FDC473EC69700000058
:10BC9000E780C0F405611763FFFF6700434397A780
:10BCA000FF1F938767EF9C43D847A1679387C7021D
:10BCB000631EF70A397106DE22DC26DA80004AD8D4
:10BCC0004ED652D456D23285B28497000000E78017
:10BCD000C0C7AA89268597000000E78020C92318DD
:10BCE000A4FC268597000000E78040C82319A4FC27
:10BCF000268597000000E78060C783D744000A8A42
:10BD0000231AA4FC858393F7F70F230EF4FC860710
:10BD1000BD0793F7073F3301F1408A8A0149834702
:10BD2000C4FD6367F902CE85130584FC232C54FD02
:10BD300097000000E78080EA5281130104FCF25072
:10BD40006254D2544259B259225A925A2161828085
:10BD5000268597000000E78060C193171900D697E9
:10BD600005092390A7001379F90F55BF828097A783
:10BD7000FF1F938767E29C43D847A1679387A70279
:10BD8000631AF70A397106DE22DC26DA80004AD807
:10BD90004ED652D456D23285B28497000000E78046
:10BDA000C0BAAA89268597000000E78020BCFD570D
:10BDB0002318A4FC26852319F4FC97000000E780D3
:10BDC000E0BA83D744000A8A231AA4FC858393F738
:10BDD000F70F230EF4FC8607BD0793F7073F3301E7
:10BDE000F1408A8A01498347C4FD6367F902CE8521
:10BDF000130584FC232C54FD97000000E78000DE2F
:10BE00005281130104FCF2506254D2544259B25987
:10BE1000225A925A21618280268597000000E7808D
:10BE2000E0B493171900D69705092390A70013795A
:10BE3000F90F55BF828097A7FF1F9387E7D59C43D3
:10BE4000D847A16789076310F70A397106DE22DC3B
:10BE500026DA80004AD84ED652D456D2328532895C
:10BE600097000000E78060AEAA894A85970000002D
:10BE7000E780C0AF835749000A8A2318A4FC858352
:10BE800093F7F70F230CF4FC8607BD0793F7073FE2
:10BE90003301F1408A8A8144834784FD63E7F402D9
:10BEA000CE85130584FC232A54FD97000000E7800B
:10BEB000E0D25281130104FCF2506254D254425930
:10BEC000B259225A925A216182804A859700000015
:10BED000E780C0A993971400D69785042390A70004
:10BEE00093F4F40F55BF828097A7FF1F9387C7CAAB
:10BEF0009C43D847A1679387E704631EF70A39710B
:10BF000006DE22DC26DA80004AD84ED652D456D23B
:10BF10003285B28497000000E78020A3AA89268595
:10BF200097000000E78080A42318A4FC26859700D2
:10BF30000000E780A0A3231AA4FC26859700000038
:10BF4000E780C0A283D744000A8A2319A4FC858312
:10BF500093F7F70F230EF4FC8607BD0793F7073F0F
:10BF60003301F1408A8A01498347C4FD6367F902BE
:10BF7000CE85130584FC232C54FD97000000E78038
:10BF8000E0C55281130104FCF2506254D25442596C
:10BF9000B259225A925A2161828026859700000068
:10BFA000E780C09C93171900D69705092390A70036
:10BFB0001379F90F55BF828097A7FF1F9387C7BDDD
:10BFC0009C43D847A1679387C704631AF70A39715E
:10BFD00006DE22DC26DA80004AD84ED652D456D26B
:10BFE0003285B28497000000E7802096AA892685D2
:10BFF00097000000E7808097FD572318A4FC268552
:10C00000231AF4FC97000000E780409683D7440091
:10C010000A8A2319A4FC858393F7F70F230EF4FCF7
:10C020008607BD0793F7073F3301F1408A8A01492C
:10C030008347C4FD6367F902CE85130584FC232C76
:10C0400054FD97000000E78060B95281130104FCA1
:10C05000F2506254D2544259B259225A925A216132
:10C060008280268597000000E78040909317190092
:10C07000D69705092390A7001379F90F55BF828041
:10C0800097A7FF1F938747B19C43D847A167DD0758
:10C090006317F7041763FFFFE70223017971328505
:10C0A000328497000000E780408A2AC622859700E4
:10C0B0000000E780A08B2311A102228597000000D9
:10C0C000E780A088B2452300A1022808970000005D
:10C0D000E780C0B045611763FFFF670043FF8280C0
:10C0E00097A7FF1F938747AB9C43D847A1679387C8
:10C0F00087046317F7041763FFFFE70203FB7971F7
:10C100003285328497000000E78020842AC6228589
:10C1100097000000E78080852311A1022285970007
:10C120000000E7808082B2452300A1022808970022
:10C130000000E780A0AA45611763FFFF670023F9AD
:10C14000828097A7FF1F938727A59C43D847A167A5
:10C150009387A7046312F7021763FFFFE702E3F474
:10C1600001112800814597000000E78020A70561A4
:10C170001763FFFF6700A3F5828097A7FF1F9387D0
:10C18000A7A19C43D847A167938757026319F70279
:10C190001763FFFFE70263F10111328597F0FFFF9C
:10C1A000E780A07A2308A1008145280097000000BD
:10C1B000E780C0A205611763FFFF670043F182803B
:10C1C00097A7FF1F9387479D9C43D847A1679387F5
:10C1D000E702631BF7041763FFFFE70203ED01119A
:10C1E0003285328497F0FFFFE7804078AA84228569
:10C1F00097F0FFFFE7808077854709E9228597F070
:10C20000FFFFE78080744205B337A0002800814516
:10C21000231891003ECA97000000E780209C05612A
:10C220001763FFFF6700A3EA828097A7FF1F93872A
:10C23000A7969C43D84799476313F7081763FFFFF6
:10C24000E702A3E679713285328497F0FFFFE78039
:10C25000C06F2AC6228597F0FFFFE7802071231068
:10C26000A102228597F0FFFFE780206E2301A10243
:10C27000228597F0FFFFE780406DA301A102228590
:10C2800097F0FFFFE780606C2302A102228597F000
:10C29000FFFFE780806B2313A102228597F0FFFF49
:10C2A000E780A06AB2452314A10228089700000085
:10C2B000E780C09245611763FFFF670043E182801A
:10C2C00097A7FF1F9387478D9C43D847A167938704
:10C2D000C7036313F7081763FFFFE70203DD7971F4
:10C2E0003285328497F0FFFFE78020662AC62285D8
:10C2F00097F0FFFFE78080672310A102228597F067
:10C30000FFFFE780A0662311A102228597F0FFFFBF
:10C31000E780A0632302A102228597F0FFFFE78058
:10C32000C062A302A102228597F0FFFFE780E061CF
:10C330002303A102228597F0FFFFE7800061B24549
:10C34000A303A102280897000000E7802089456127
:10C350001763FFFF6700A3D782801763FFFFE70221
:10C36000C3D401112A8497F0FFFFE780005EAA84FE
:10C37000228597F0FFFFE780605F228597F0FFFF3F
:10C38000E780C05E035744008D4763F7E7002285CE
:10C3900097F0FFFFE780805D228597F0FFFFE78041
:10C3A000E05C2800A68597000000E78020830561F7
:10C3B0001763FFFF6700A3D19797FF1F9387C77D80
:10C3C0009C43D847A167FD07631FF7001763FFFF72
:10C3D000E702A3CD328597000000E78040F817639D
:10C3E000FFFF6700C3CE82809797FF1F9387C77AAE
:10C3F0009C43D847A167E5076315F7081763FFFF5C
:10C40000E702A3CA79713285328497F0FFFFE78093
:10C41000C0532AC6228597F0FFFFE780205522856A
:10C4200097F0FFFFE78080542310A102228597F048
:10C43000FFFFE780A053520551812311A1022285FD
:10C440002302010297F0FFFFE7802050A302A10220
:10C45000228597F0FFFFE780404F2303A10222854A
:10C4600097F0FFFFE780604EB245A303A1022808C2
:10C4700097F0FFFFE780807645611763FFFF670055
:10C4800003C582809797FF1F938707719C43D84706
:10C49000A1679387E703631FF7001763FFFFE702B6
:10C4A000C3C0328597000000E78060EB1763FFFF91
:10C4B0006700E3C182809797FF1F9387E76D9C43D6
:10C4C000D847A16793874704631EF7021763FFFFEE
:10C4D000E702A3BD79713285328497F0FFFFE780D0
:10C4E000C0462AC6228597F0FFFFE7802048B24564
:10C4F000280897F0FFFFE780606E45611763FFFF34
:10C500006700E3BC82809797FF1F9387E7689C438F
:10C51000D847A167938787026310F7041763FFFF6B
:10C52000E702A3B879713285328497F0FFFFE78084
:10C53000C0412AC6228597F0FFFFE7800041B2453F
:10C540002300A102280897F0FFFFE78020694561DA
:10C550001763FFFF6700A3B782801763FFFFE7023F
:10C56000C3B4011197F0FFFFE780203EAA852800A1
:10C5700097F0FFFFE780806605611763FFFF6700A4
:10C5800003B59797FF1F938727619C43D847A167FF
:10C59000D107631FF7001763FFFFE70203B132857E
:10C5A00097000000E780A0FB1763FFFF670023B23E
:10C5B00082809797FF1F9387275E9C43D847A16788
:10C5C000C507631FF7001763FFFFE70203AE32855D
:10C5D00097000000E780A0F81763FFFF670023AF14
:10C5E00082809797FF1F9387275B9C43D847A1675B
:10C5F000B907631FF7001763FFFFE70203AB32853C
:10C6000097000000E780A0F51763FFFF670023ACE9
:10C6100082809797FF1F938727589C43D847A1672D
:10C62000AD07631FF7001763FFFFE70203A832851A
:10C6300097000000E780A0F21763FFFF670023A9BF
:10C6400082809797FF1F938727559C43D847894738
:10C650006318F7021763FFFFE70223A50111328574
:10C6600032C897F0FFFFE780402EAA85280097F098
:10C67000FFFFE780A05605611763FFFF670023A552
:10C6800082809797FF1F938727519C43D847A167C4
:10C690008D076311F7041763FFFFE70203A1011180
:10C6A0003285328497F0FFFFE780202A130661006D
:10C6B000AA844C00228597300000E780C023280020
:10C6C000A68597F0FFFFE780605105611763FFFFC4
:10C6D0006700E39F82809797FF1F9387274C9C43B7
:10C6E00081CFDC4391CB1763FFFFE702039C829766
:10C6F0001763FFFF6700A39D82801763FFFFE702B8
:10C70000C39A79713C08AE843ED2A165B7070A008E
:10C710002A843ED448103C08DD053ED636C432C6D5
:10C720003AC297D0FFFFE780E02F12474810BA8542
:10C7300097F0FFFFE780C01332464810B28597F0AC
:10C74000FFFFE780E014A2464810B68597F0FFFF90
:10C75000E7800012501001478146A685228597D0B8
:10C76000FFFFE780805145611763FFFF6700239655
:10C770001763FFFFE702639301117C000329C501E2
:10C78000AE843ECAA165B70707002A843ECC48089C
:10C790007C00C5053ECE97D0FFFFE780A0288345EB
:10C7A000D900480897F0FFFFE780800C5008014748
:10C7B0008146A685228597D0FFFFE780004C056162
:10C7C0001763FFFF6700A3901763FFFFE702E38D86
:10C7D00083C7950093F7F707A384F500970000003F
:10C7E000E78040F91763FFFF6700638E1763FFFF61
:10C7F000E702A38B79713C08AE843ED2A165B707EE
:10C8000009002A843ED448103C08938545043ED64E
:10C8100032C636C497D0FFFFE780C020A24648103A
:10C82000B68597F0FFFFE780A00432464810B28536
:10C8300097F0FFFFE780C005501001478146A685AD
:10C84000228597D0FFFFE780404345611763FFFFD4
:10C850006700E3871763FFFFE702238583C795001F
:10C8600041112A8493F7F707A384F50032852EC679
:10C8700097F0FFFFE780800F85672AC46370F50299
:10C8800097700000E78020E92246B24509ED114784
:10C890008146228597000000E78060E6410117632A
:10C8A000FFFF6700C38201478346F501DDB71753D9
:10C8B000FFFFE702E37D01113C003ECAB7070A0013
:10C8C0003ECC3C003ECE83C79500AA89328593F7C3
:10C8D000F707A384F5002E8497F0FFFFE780000997
:10C8E0008567637DF504A165AA849385850448085E
:10C8F00097D0FFFFE7800013268597700000E78040
:10C9000080E12A8929E19145480897F0FFFFE780F7
:10C9100020F6A685480897F0FFFFE78060F7CA85F4
:10C92000480897F0FFFFE780A0F4014781465008D0
:10C93000A2854E8597D0FFFFE7802034056117530D
:10C94000FFFF670023788145480897F0FFFFE780E5
:10C9500020F20349090275BF1753FFFFE702437333
:10C9600079711C103ECAB7070F003ECC404D1C1019
:10C97000AA84AE894808994532C636893ECE97D0FA
:10C98000FFFFE780200A32464808B28597F0FFFF94
:10C99000E78000EE630C0902A545480897F0FFFF09
:10C9A000E780C0E62546CA8597200100E78020A4DD
:10C9B000500801478146CE85268597D0FFFFE78046
:10C9C000C02B45611753FFFF6700C36F8355C40237
:10C9D000480897F0FFFFE780A0EB0355E40281458C
:10C9E00005C5854785456301F502C167FD179305B8
:10C9F000F00F630BF5007D1597700000E780208E27
:10CA00009305150093F5F50F480897F0FFFFE780B1
:10CA100020E683450403480897F0FFFFE78040E5E0
:10CA200083451403480897F0FFFFE78060E48355CF
:10CA30002403480897F0FFFFE78080E5835544030F
:10CA4000480897F0FFFFE780A0E49DB71753FFFF6A
:10CA5000E702A36583C795008146014693F7F70770
:10CA6000A384F50097000000E78040EF1753FFFF15
:10CA70006700E3651753FFFFE702236379713E8484
:10CA80001C103ECA2E89B7070F00A1653ECCFD05DC
:10CA90001C10AA84480842C03AC23ECE36C432C6F0
:10CAA00097D0FFFFE78000F832464808B28597F03C
:10CAB000FFFFE780E0DBA2464808B68597F0FFFF5E
:10CAC000E78000DD12474808BA8597F0FFFFE7804E
:10CAD00020DC0248630C08029145480897F0FFFFEC
:10CAE000E780C0D21146A28597200100E780209000
:10CAF000500801478146CA85268597D0FFFFE78009
:10CB0000C01745611753FFFF6700635C89454808FC
:10CB100097F0FFFFE78080CF834704002300F500F4
:10CB200083471400A300F500E1B71753FFFFE702A6
:10CB3000235683C7950001112A8A93F7F707A38428
:10CB4000F5003285AE8432C697F0FFFFE78000E241
:10CB500032462A89328597F0FFFFE78000DF85673C
:10CB60006373F902AA894A8597700000E780A0BA2A
:10CB70002A8419ED114781464A86A6855285970079
:10CB80000000E780C0B705611753FFFF67008353BC
:10CB90009387E9FF93F7F70F0547E366F7FE8347AF
:10CBA000F50195EB8947E380F9FE8346F401528550
:10CBB00001474A86A68597000000E78040B4A16738
:10CBC000D90748083ECC230A010002CE9700000096
:10CBD000E780A0B04DBF639EE7008947639EF900E0
:10CBE00093071020231FF50097700000E780C0B75F
:10CBF0006DBF0947E39BE7FA8D47E398F9FA228571
:10CC000097700000E78080DF9797FF1F93870718D2
:10CC10009C4399E79797FF1F938707019C4399C708
:10CC200003D5040097800000E780A0CE231F0400F6
:10CC300022855DBF1753FFFFE702234701113C0028
:10CC40003ECAB7070B003ECC3C003ECE83C79500E2
:10CC50002A89328593F7F707A384F500AE8497F00D
:10CC6000FFFFE780A0D093170501C187635AF00644
:10CC7000A1652A849385E502480897D0FFFFE780E5
:10CC800060DAA285480897F0FFFFE78060C09797B9
:10CC9000FF1F938767F99C43A9EB01449375F40F39
:10CCA000480897F0FFFFE780A0BC9355844093F5B8
:10CCB000F50F480897F0FFFFE78080BB93550441CC
:10CCC00093F5F50F480897F0FFFFE78060BA01473A
:10CCD00081465008A6854A8597D0FFFFE780E0F996
:10CCE00005611753FFFF6700833E41658546054692
:10CCF000A2857D1597500000E78060BD59DD510584
:10CD000097000100E780808F1304400633448502BA
:10CD100071B71753FFFFE70243390111B707060048
:10CD20003EC683C7950021642A8993F7F707A38439
:10CD3000F500AE8428009305A4040AC40AC897D05D
:10CD4000FFFFE78020CE300001478146A6854A8557
:10CD500097D0FFFFE78060F297E0FFFFE780801544
:10CD600013049404480822CC230A010002CE970041
:10CD70000000E780809605611753FFFF67002335A9
:10CD80001753FFFFE702C330C1642A890144979912
:10CD9000FF1F93892901130A8002FD1497E0FFFF0A
:10CDA000E78080C16347A40001451753FFFF670078
:10CDB0006331B307440303A7C90ABA9703D707002F
:10CDC0006306970083D72700638427010504F9B71A
:10CDD0000545E1BF1753FFFFE702832B2A8A2E89FF
:10CDE00099C123A0050081498144979AFF1F938A26
:10CDF0002ADB614B97E0FFFFE78040C263C7A400D6
:10CE00004E851753FFFF6700E32B3384640383A72A
:10CE10000A003E948357040099E763040900232025
:10CE200089008504C1BF4146D2851305440097108F
:10CE30000100E780605975F5A289E5B71753FFFF38
:10CE4000E702032539717C083ED4B7070A003ED6B5
:10CE50007C083ED883C795002A8A328593F7F70766
:10CE6000A384F5002E8932C697F0FFFFE78000B05B
:10CE700085676373F5083246AA84328597F0FFFF11
:10CE8000E780A0AC8547AA8963E8A706A1659385DA
:10CE90008504281097D0FFFFE780C0B826859770DB
:10CEA0000000E78040872A8429ED9145281097F0FB
:10CEB000FFFFE780E09BA685281097F0FFFFE78043
:10CEC000209DCE85281097F0FFFFE780609A0147EC
:10CED00081463010CA85528597D0FFFFE780E0D9A0
:10CEE000A1679387770448183EDC230A010202DE1B
:10CEF00097F0FFFFE780607E21611753FFFF670017
:10CF0000631C8145281097F0FFFFE7806096A68597
:10CF1000281097F0FFFFE780A0979797FF1F938750
:10CF2000271F9C4381CB22856389090097D000008D
:10CF3000E78040248345040271B797D00000E78062
:10CF4000C022CDBF1753FFFFE702831483C79500AC
:10CF50004111AA8993F7F707A384F5003285AE84BF
:10CF6000328A97F0FFFFE78060A08567637FF50254
:10CF70002A8997600000E780007A2A84914631C5AB
:10CF80008347F50105476387E70291C70D4763664D
:10CF9000F704AD461DA89305050303250A00414685
:10CFA00097100100E78040420DE941011753FFFF50
:10CFB000670043119305950803250A004146971021
:10CFC0000100E7806040814669F54A86A6854E8566
:10CFD00097000000E780C081C9BF83250A001305C0
:10CFE000940897700000E780A02919C1C146F1BFDD
:10CFF0009797FF1F938787D99C4399E79797FF1FC0
:10D00000938787C29C4399C7228597800000E78059
:10D01000208A69FD8547A30FF400228597B00000A0
:10D02000E7806084228597600000E780E0734E858A
:10D0300081464A86A68597F0FFFFE780607BA1675F
:10D040009387570448003EC42302010002C697F0AC
:10D05000FFFFE780806891BF1753FFFFE70263027D
:10D0600083C795004111AA8993F7F707A384F500B8
:10D0700032852E89B28A97F0FFFFE780208F85677F
:10D080006374F50EAA8497600000E780C0682A8464
:10D090000DED416B014A979BFF1F938BABD0130C97
:10D0A000400E7D1B19A833048A0383A70B0B3E9403
:10D0B0008357C40163836705050A97E0FFFFE78094
:10D0C000A08EE342AAFE95460DA08357C501639644
:10D0D00097029305050303A50A0041469710010036
:10D0E000E780802E994611E181462686CA854E85C5
:10D0F00097F0FFFFE780C06F85A883A50A0013059E
:10D10000040397700000E780A017C14679FD2285CF
:10D11000231E940097A00000E780E07422859760AA
:10D120000000E78060649797FF1F938767FE9C432A
:10D13000A9C323000402228597D00000E78040F0B5
:10D140004E8581462686CA8597F0FFFFE780406AB4
:10D15000A1679387070448003EC42302010002C66A
:10D1600097F0FFFFE780605741011753FFFF67000B
:10D17000C3F489472300F402E1B7397106DE22DCEB
:10D180004AD8800052D456D25AD026DA4ED65ECE35
:10D190002E8A32892A8B97D0FFFFE780E07D060533
:10D1A000710541998A8A3301A140232224FC23146A
:10D1B00004FC97D0FFFFE780207C83479A00060598
:10D1C000350593F7F7072315A4FCA304FA004A8555
:10D1D000232624FC97E0FFFFE780407993170501A1
:10D1E000C1876340F0025681130104FCF25062547F
:10D1F000D2544259B259225A925A025BF24B2161DF
:10D200008280AA844A8597E0FFFFE7802076AA897A
:10D210004A8597E0FFFFE7806075A1659385C502A9
:10D220002A89130544FC97C0FFFFE780A07F26856D
:10D2300097C0FFFFE780E073854511C94A86CE8518
:10D2400097C0FFFFE780606DAA8B21E98945130530
:10D2500044FC97E0FFFFE780A061A685130544FC2E
:10D2600097E0FFFFE780C062CE85130544FC97E09E
:10D27000FFFFE780E061CA85130544FC97E0FFFFEC
:10D28000E780006101478146130644FCD2855A8538
:10D2900097D0FFFFE780609EB9B78145130544FC36
:10D2A00097E0FFFFE780C05CA685130544FC97E08C
:10D2B000FFFFE780E05DCE85130544FC97E0FFFFAC
:10D2C000E780005DCA85130544FC97E0FFFFE78017
:10D2D000205C814497D0FFFFE780006AE3D4A4FA82
:10D2E00083A70B0113971400BA9783D5070099C53C
:10D2F000130544FC97E0FFFFE78080598504D9BF00
:10D30000797106D622D44AD000184ECE52CC56CAD5
:10D3100026D25AC8AE893289AA8A97D0FFFFE78001
:10D32000A0650605690541990A8A3301A140232AAF
:10D3300024FC231C04FC97D0FFFFE780E06383C735
:10D34000990006052D0593F7F707231DA4FCA38478
:10D35000F9004A85232E24FC97E0FFFFE780006157
:10D3600093170501C187634FF0005281130104FD3B
:10D37000B250225492540259F249624AD24A424B64
:10D3800045618280AA844A8597E0FFFFE780005EBE
:10D39000A1659385A5022A89130544FD97C0FFFF67
:10D3A000E7804068268597C0FFFFE780805C854561
:10D3B00009C9CA8597C0FFFFE78020592A8B29E158
:10D3C0008945130544FD97E0FFFFE780604AA68585
:10D3D000130544FD97E0FFFFE780804BCA851305E6
:10D3E00044FD97E0FFFFE780A04A0147814613060E
:10D3F00044FDCE85568597D0FFFFE7800088B5B7FE
:10D400008145130544FD97E0FFFFE7806046A68550
:10D41000130544FD97E0FFFFE7808047CA851305A9
:10D4200044FD97E0FFFFE780A046814497D0FFFFCF
:10D43000E7808054E3DBA4FA83270B0113971400E1
:10D44000BA9783D5070099C5130544FD97E0FFFF00
:10D45000E78000448504D9BF1753FFFFE702E3C408
:10D4600083474500404DD5EFFD575DC4834694008A
:10D4700009476363D70A0346B400854663EEC608CE
:10D480008306E40063CA06085C45F9562390D7007A
:10D490009787FF1F83C7077199E3A304E400978769
:10D4A000FF1F938767789C4381E78947A306F400B1
:10D4B0009797FF1F9387C7C59C4381E7894723063A
:10D4C000F4009705000093854506AA84130504011E
:10D4D00097F00000E7802010FD57231AF4028147DF
:10D4E0001CDC01489787FF1F23AA876A9787FF1FC5
:10D4F0009387076B232E040304C0804397D0FFFF5C
:10D50000E780C05161463306C502814522859750A8
:10D51000FFFFE78080BC81473E851753FFFF670010
:10D5200003BBFD57D5BF1753FFFFE70203B82A849B
:10D530000355450297600000E780E01D19E5231EB2
:10D5400004001753FFFF670083B88357E401F5DB3E
:10D55000930504FF174501001305052797E0000018
:10D56000E780E014F9BF1753FFFFE70203B42E89E9
:10D57000A16541119385E5032A8436C432C6BE8471
:10D580003AC297C0FFFFE780E04912472285BA857B
:10D5900097E0FFFFE780C02D32462285B28597E0F5
:10D5A000FFFFE780E02EA2462285B68597E0FFFFC9
:10D5B000E780002E630309029145228597E0FFFF73
:10D5C000E780C0241146A68597100100E78020E27D
:10D5D00041011753FFFF670083AF8945228597E01C
:10D5E000FFFFE780A02283C704002300F50083C764
:10D5F0001400A300F500E9BF1753FFFFE702E3AAF9
:10D6000083C79500444D054793F7F707A384F500BA
:10D610001C42411183C707006367F7062E842A89DD
:10D62000B1C003C7D400630FF7021787FF1F1307AA
:10D63000A75F184305C3A386F40097A00000E78006
:10D64000404A83C7D40099E741657D1597400000A3
:10D65000E780403083D72403918B89C797E000008F
:10D66000E780C0134A85A28597F0FFFFE78080100E
:10D67000A167C10748003EC42302010002C697F01B
:10D68000FFFFE780800541011753FFFF670023A4D8
:10D690001753FFFFE70263A103D745008D47AA8414
:10D6A00041112E8432892E8563E3E70297E0FFFF64
:10D6B000E780C02BAA8523000900268597C0FFFFBD
:10D6C000E780A02841011753FFFF670043A097E0C0
:10D6D000FFFFE780A0292AC6228597E0FFFFE780A9
:10D6E000E028B24585472A862300F900268597C0A1
:10D6F000FFFFE7808022F9B7397106DE22DC26DAE7
:10D7000080004ED652D456D24AD85AD05ECEAE8978
:10D71000B284AA8A97D0FFFFE7800025060513058B
:10D72000250241990A8A3301A140232224FC2314B3
:10D7300004FC97D0FFFFE780202383C799000605EC
:10D740004D0593F7F7072315A4FCA384F90026855C
:10D75000232624FC97E0FFFFE78040219317050173
:10D76000C1876340F0025281130104FCF2506254FD
:10D77000D2544259B259225A925A025BF24B216159
:10D780008280AA8B03AB040097C0FFFFE780601E76
:10D7900051E583D7440001498544F11793B7170039
:10D7A000A301F4FC834734FCA165C9C79385E50454
:10D7B000130544FC97C0FFFFE780C026A68513052C
:10D7C00044FC97E0FFFFE780A00ADE85130544FCD8
:10D7D00097E0FFFFE780C00B834734FC114691E3DD
:10D7E0000946DA85130544FC97E0FFFFE7806005F2
:10D7F0008144630A0900416B7D1B97D0FFFFE780DE
:10D80000A01663CCA40201478146130644FCCE85D2
:10D81000568597C0FFFFE7804046B1B7A68513063F
:10D8200034FC97000000E780E0E6933415002A8975
:10D8300086048DBF9385C504A5BF8327C9001397B0
:10D840001400BA9783D5070063886501130544FC6B
:10D8500097E0FFFFE780C003850445B71753FFFF3C
:10D86000E702238279711C103EC4B7070F003EC641
:10D870001C103EC883C79500AA8A328593F7F70724
:10D88000A384F500AE89328497E0FFFFE780000EA5
:10D8900093170501C187635AF0062A8A228597E00B
:10D8A000FFFFE780A00C2A895285032B040097C054
:10D8B000FFFFE780000C39ED8357440081440544A5
:10D8C000F11793B71700A303F10083457100DA87BE
:10D8D0002287CA865286280097000000E780E0C8A9
:10D8E000014781463000CE85568597C0FFFFE7800F
:10D8F000C038A1679387D70348083ECC230A81002C
:10D9000026CE97F0FFFFE78040DD45611743FFFF1C
:10D910006700A37AA2851306710097000000E780D4
:10D9200060D7AA84094455D13544E30055FB4A85A4
:10D9300097F0FFFFE78000450D4441D9014497D09F
:10D94000FFFFE7806002634DA400C16B0144FD1B33
:10D9500097D0FFFFE7804001634EA4001544B5B7A0
:10D96000DC4413171400BA9783D707006383270397
:10D970000504F1B7D84493171400BA9703D70700EA
:10D98000631B770123902701268597A00000E7807D
:10D9900080DB01441DBF050465BF1743FFFFE7029D
:10D9A000236F83C7950041112A8A93F7F707A38451
:10D9B000F50032852E89328497E0FFFFE78000FB77
:10D9C00093170501C1876353F006AA89228597E062
:10D9D000FFFFE780A0F92311A1004E85832A0400F0
:10D9E00097C0FFFFE780E0F839E58357440085449E
:10D9F0000144F11793B71700A300F1000348110089
:10DA000003572100D6875285CE862686CA8597F091
:10DA1000FFFFE7806006A167F10748003EC42302CC
:10DA2000910022C697F0FFFFE78020CB410117430A
:10DA3000FFFF67002369A28513061100970000000D
:10DA4000E78040C52A84894455D98357210011674E
:10DA50008544BA97C2071167C1831307F7EFE36FD5
:10DA6000F7F89787FF1F938767329C4381CB8545E3
:10DA70001305210097500000E78020758355210091
:10DA80002285814497C0FFFFE78040E525D9231018
:10DA90000500228597A00000E78040CD85B7174399
:10DAA000FFFFE702035E83C7950041112A8B93F7BE
:10DAB000F707A384F50032852E8A328497E0FFFFB2
:10DAC000E780C0EA93170501C1876351F006AA8A6F
:10DAD000228597E0FFFFE78060E92A895685832B3E
:10DAE000040097C0FFFFE780C0E831E5835744009A
:10DAF00081440544F11793B71700A301F1000348CF
:10DB00003100DE875A854A87D6862286D28597F0ED
:10DB1000FFFFE78060F6A167ED0748003EC42302DF
:10DB2000810026C697F0FFFFE78020BB4101174325
:10DB3000FFFF67008358A28513063100970000009D
:10DB4000E78040B5AA8409445DD99167CA97C207A6
:10DB50001167C1831307F7EF0544E362F7FACA853B
:10DB600097C0FFFFE78080D7014451F9814997D0E2
:10DB7000FFFFE78060E063DBA900984893971900F6
:10DB8000BA9703D7070005EF2390270197D0FFFF2F
:10DB9000E78080DE1544E384A9F6268597A000007F
:10DBA000E780C0BC9787FF1F9387471E9C430144B3
:10DBB000B9D74A8597500000E780C05889B78509D2
:10DBC0007DB71743FFFFE702A34C79713E847C08C1
:10DBD0003EC82E8AB7071400A1653ECAE5057C0839
:10DBE000AA89080836C4428932C6BA8AC6843ECC9D
:10DBF00097C0FFFFE78000E3CA85080897E0FFFFB2
:10DC0000E78000C732460808B28597E0FFFFE7804B
:10DC100020C8A246630A09049D45080897E0FFFF53
:10DC2000E780C0BE1D4681459740FFFFE780E04A80
:10DC300063890A089145080897E0FFFFE78000BD67
:10DC40001146A68597000100E780607A1008014719
:10DC50008146D2854E8597C0FFFFE780000245616F
:10DC60001743FFFF67000346B685080897E0FFFFEC
:10DC7000E78000C21C400808D8439355C701858936
:10DC800012075183B205D98D97E0FFFFE78040C0AE
:10DC90001C40080883C5870097E0FFFFE78040BD70
:10DCA0001C40080883C5A70097E0FFFFE78040BC41
:10DCB0001C40080883C5970097E0FFFFE78040BB42
:10DCC00085BF8945080897E0FFFFE78020B483C738
:10DCD00004002300F50083C71400A300F500BDB7BE
:10DCE0001743FFFFE702C33A83C795004111AA8992
:10DCF00093F7F707A384F5003285AE84328497E06A
:10DD0000FFFFE780A0C693170501C187635DF0049C
:10DD10002A89032A040097C0FFFFE78080C519E91C
:10DD2000835744000548F11793B71700A307F10084
:10DD3000814631A81306F100A28597000000E78014
:10DD400060951DC51C459DC783D647000148034704
:10DD5000F10093078500D2884A86A6854E859700F4
:10DD60000000E78040E641011743FFFF670083356D
:10DD700009487DBF1D486DBF1743FFFFE7024331D0
:10DD800065715C083EC4B7077B013EC65C083EC8AF
:10DD900083C795002A8A328593F7F707A384F50095
:10DDA000AE8997E0FFFFE78040BA8357E100E1C703
:10DDB0008945280097C0FFFFE780C0C6814528003D
:10DDC00097E0FFFFE780C0AA97C0FFFFE780A0CCE5
:10DDD0009787FF1F9387C7339C431784FF1F034414
:10DDE00064DCAA843334800099C3136424009787C9
:10DDF000FF1F938767E39C4399C31364440097878D
:10DE0000FF1F9387A7F89C4399C31364840083D5AD
:10DE100004002800014997E0FFFFE78060A783D551
:10DE20002400280097E0FFFFE78080A683D5440008
:10DE3000280097E0FFFFE780A0A597D0FFFFE780CD
:10DE4000A0AE93150501C181280097E0FFFFE78090
:10DE500020A4A285280097E0FFFFE78060A39C44F0
:10DE60006360F902014781463000CE85528597C034
:10DE7000FFFFE78080E059611743FFFF67008324BD
:10DE8000DC441314490028003E9497E0FFFFE7802C
:10DE90006096834744000347540089070607BA97F2
:10DEA0008607E36AF5FC835524002800814A97E041
:10DEB000FFFFE780E09D83454400280097E0FFFFD7
:10DEC000E780009B83455400280097E0FFFFE78030
:10DED000209A8347440063C9FA00814A834754006B
:10DEE00063C1FA020509A5BF1C4413975A00280014
:10DEF000BA9783D50700850A97E0FFFFE78040992E
:10DF0000C9BF032BC40093975A0028003E9B83553A
:10DF10002B00850A97E0FFFFE780809783550B0071
:10DF2000280097E0FFFFE780A0964DBF1743FFFF53
:10DF3000E702A3175C4993E717005CC997A00000AC
:10DF4000E78020B61743FFFF670063181743FFFF02
:10DF5000E702A3152E84814597F0FFFFE780C0E715
:10DF600005C583570500FD172310F50009C4835725
:10DF700025002310F40097000000E78060FB0145B6
:10DF80001743FFFF6700A31431457DD82310040019
:10DF9000C5BF1743FFFFE702A30F83C795004111D9
:10DFA0002A8A93F7F707A384F50032852E893284F5
:10DFB00097E0FFFFE780809B93170501C1876356B9
:10DFC000F006AA89C145228597E0FFFFE780A0807F
:10DFD0002A8B4E85832A040097C0FFFFE780609953
:10DFE00031E983574400231101000544F11793B729
:10DFF0001700A300F10081440348110003572100DA
:10E00000D6875285CE862286CA8597F0FFFFE780A5
:10E01000A0A6A1679387170248003EC4230281008F
:10E0200026C697E0FFFFE780406B41011743FFFFE3
:10E030006700430913061100A28597F0FFFFE780F0
:10E040006065AA8409E523110100094475B79305A9
:10E0500021005A8597000000E78080EF8357210058
:10E060002A84D9DB9787FF1F938747D29C4381CBB4
:10E0700085451305210097500000E7800015835562
:10E0800021002685314497C0FFFFE78020852DD5EC
:10E0900023100500268597900000E780206D01443D
:10E0A000A1BF1743FFFFE702430041112E896C0017
:10E0B000AA8402C697F0FFFFE78000D20DC1035784
:10E0C000050005072310E50097000000E78040E603
:10E0D00081473E8541011743FFFF670043FF3247F9
:10E0E000954765DBCA85268597300000E780400D9F
:10E0F000C147E34005FE3244854741462310F40002
:10E1000083570900A685130544002311F4009700E6
:10E110000100E780C02D228545BF1743FFFFE702BE
:10E1200023F783C795004111AA8A93F7F707A384C1
:10E13000F5003285AE89328497E0FFFFE7800083E7
:10E1400093170501C1876356F0062A8AC1452285C7
:10E1500097D0FFFFE7802068AA845285032B040034
:10E1600097C0FFFFE780E08031E983574400231127
:10E1700001008544F11793B71700A300F100014493
:10E180000348110003572100DA875685D286268678
:10E19000CE8597F0FFFFE780208EA1679387070267
:10E1A00048003EC42302910022C697E0FFFFE780AB
:10E1B000C05241011743FFFF6700C3F0A285130659
:10E1C000110097F0FFFFE780E04C2A8409E5231156
:10E1D0000100894475B7268593052100970000004A
:10E1E000E78060ECAA8449FD83552100228597B021
:10E1F000FFFFE780A06E49F5014997C0FFFFE78068
:10E20000A077635DA900184893171900BA9703D740
:10E2100007000DEF035721002390E70097C0FFFF91
:10E22000E7808075630625039787FF1F938707B6EE
:10E230009C4399C70355210097500000E78080F068
:10E24000228597900000E78060521DBF050975B7D1
:10E2500095443DB705C19307F00F630FF500C5471F
:10E26000630CF5009307F5FF05453315F5004205EE
:10E27000418182800145828041657D158280B9E9B6
:10E280001743FFFFE70263E203450603328497006A
:10E290000000E78060FC9305803EB305B502C2052F
:10E2A000C18181CD0357E402854763F8E700130578
:10E2B000040197E00000E78020428357E4024167B1
:10E2C0007D176385E700FD172317F4021743FFFF4F
:10E2D0006700E3DF82801743FFFFE70283DA004233
:10E2E00083C79500444D0349140093F7F707A384AF
:10E2F000F50083470400220911673369F900A1671B
:10E30000B347F90041112A8BAE8A63ECE70E8347CD
:10E3100024001307C00EB91793F7F70F6373F710B4
:10E3200003473400C14763EEE70E834744001307F9
:10E33000E00793C707086371F70C8349840083479C
:10E340007400A209B3E9F900856763F7F90A034A83
:10E350006400834754004E85220A336AFA009750BE
:10E360000000E780403B61C123962403834B3400C7
:10E37000137AFA00239A34032388740323994403FD
:10E3800093890401631C090023A604022398040254
:10E390004E8597E00000E78060363DA003492400E9
:10E3A0004A8597000000E78020EB2397A40283476B
:10E3B00044004E85A388F402E38D0BFCE30B09FCBB
:10E3C00097E00000E780202F97900000E78000731F
:10E3D00081460146D6855A8597E0FFFFE7800058C1
:10E3E000A167938797033EC423020100480002C639
:10E3F00097E0FFFFE780602E41011743FFFF6700B2
:10E40000C3CB8544A2862686D6855A8597E0FFFF32
:10E41000E780C054A167938797033EC4230291000D
:10E42000F1B7BD44C5B79144F1BF1743FFFFE70201
:10E4300023C601111C08404D3EC2B7070F003EC461
:10E440001C083EC62A89AE8997C0FFFFE780A0DA84
:10E45000585C1C5C6346B70E6394E50063E2A70E4C
:10E460003385A740B3B7A700B305B7401306803E76
:10E4700081469D8D97000100E78080B793140501C8
:10E48000C180A1659385C503480097B0FFFFE78071
:10E4900060598145480097D0FFFFE780603D835574
:10E4A0000404480097D0FFFFE780803E8355240492
:10E4B000480097D0FFFFE780A03D814589CCC16728
:10E4C000FD179305F00F6388F40026859750000030
:10E4D000E780E0E0AA85480097D0FFFFE780403959
:10E4E00003554404814501CDC167FD179305F00F25
:10E4F0006307F50097500000E78060DEAA854800BA
:10E5000097D0FFFFE780C03683456404480097D06A
:10E51000FFFFE780E03583457404480097D0FFFF94
:10E52000E7800035500001478146CE854A8597B087
:10E53000FFFFE780807405611743FFFF670083B822
:10E54000814481B71743FFFFE70223B683C79500D5
:10E5500093F7F707A384F50097000000E78020ED0C
:10E560001743FFFF6700A3B61743FFFFE70243B25D
:10E5700083C795004111404D93F7F707A384F50039
:10E580002A8A3285B284AE8997D0FFFFE780003EA9
:10E590002A8B268597D0FFFFE780403D2A89268574
:10E5A00097D0FFFFE780603A93170B0163CA070219
:10E5B000E177CA97C207C183116763E3E702930754
:10E5C0000910C207C1831307B00F637BF7009317CD
:10E5D0000901C187AA8A634AF000C54763FE570153
:10E5E00041011743FFFF6700E3AD97B0FFFFE780EE
:10E5F000C028E31725FFD5B763080B02630609029D
:10E60000814463890A02B7077F0023106405231140
:10E6100024057CC0568597000000E780E0C3930482
:10E62000803EB304950239A0B7077F00232004047D
:10E630007CC081440355240497E00000E780A0A338
:10E64000A1C497C0FFFFE78000BB269593D7F44194
:10E6500033379500AE97BA9708DC5CDCCE855285DF
:10E6600097000000E780A0DC99E023220404A16762
:10E670009387B70348003EC42302010002C697E017
:10E68000FFFFE7808005A9BF814701481CDC232EDE
:10E690000403E9B71743FFFFE70223A197C0FFFF79
:10E6A000E780C037E1473305F502914597500000F8
:10E6B000E78000C5E55711C59777FF1F23A2A74E36
:10E6C00081473E851743FFFF670063A085471777A3
:10E6D000FF1F2309F74C82801743FFFFE702E39CEB
:10E6E0009777FF1F9387874B80433DC08357040470
:10E6F0006390A70683572404639CB7043689B284C9
:10E7000097C0FFFFE78020AF5C5C63C3B7046395ED
:10E71000B7001C5C63EEA7028347640463F3F40054
:10E72000A6872303F4048347740463F39700A68742
:10E73000A303F4048357440441677D176385E7000E
:10E7400085072312F4043C4481C7CA852685829735
:10E750001743FFFF6700A3979777FF1F938707442F
:10E760009C43014599C303C5870082801743FFFF7F
:10E77000E702A3930111B70707003EC683C79500C0
:10E78000584D0AC493F7F7070AC8A384F5002A89ED
:10E79000AE8411CB1C4283C707002304F700979077
:10E7A0000000E7800034216493055402280097B0EC
:10E7B000FFFFE780202797000000E78020FAAA8566
:10E7C000280097D0FFFFE780A00A3000014781466C
:10E7D000A6854A8597B0FFFFE780204A13044402CC
:10E7E000480822CC230A010002CE97E0FFFFE78011
:10E7F000C0EE05611743FFFF6700638D1743FFFFFE
:10E80000E702A38A01117C003ECAB70707003ECC8D
:10E810007C003ECE83C795002E84AA8493F7F70729
:10E82000A384F500A16593855502480897B0FFFFC2
:10E83000E780401F97000000E78040F2AA85480863
:10E8400097D0FFFFE780C002500801478146A285AC
:10E85000268597B0FFFFE780404205611743FFFF21
:10E860006700E3869777FF1F938747339C430945EB
:10E8700099C303C5970082809777FF1F938707325C
:10E880009C43094599C303C5D70082809777FF1F32
:10E890009387C7309C43014599C303C5A700828075
:10E8A0001733FFFFE702C37E0111B70708003EC61A
:10E8B00083C79500404D0AC493F7F7070AC8A3849D
:10E8C000F5002A89AE8429C41442854703C706008F
:10E8D00063E0E70A83479400094681496380C702E1
:10E8E000B307F740A304E400B339F00083C7160070
:10E8F0002305F40097900000E780A01E035724032F
:10E90000058B19C76386090097D00000E78000E9EE
:10E91000216493058402280097B0FFFFE7808010F0
:10E9200097000000E78040F4AA85280097D0FFFFF9
:10E93000E78000F497000000E78080F5AA852800B2
:10E9400097D0FFFFE780C0F2014781463000A685DF
:10E950004A8597B0FFFFE7804032130474024808ED
:10E9600022CC230A010002CE97E0FFFFE780E0D629
:10E9700005611733FFFF6700E3741733FFFFE702FA
:10E98000C37201117C003ECAB70708003ECC7C0070
:10E990003ECE83C795002E84AA8493F7F707A384FD
:10E9A000F500A16593858502480897B0FFFFE780D1
:10E9B000600797000000E78020EBAA85480897D001
:10E9C000FFFFE780E0EA97000000E78060ECAA859F
:10E9D000480897D0FFFFE780A0E95008014781462B
:10E9E000A285268597B0FFFFE780202905611733B0
:10E9F000FFFF6700C36D9777FF1F9387271A9C431C
:10EA0000014599C303C5B70082801733FFFFE702B2
:10EA1000C3690111B70707003EC683C79500404D83
:10EA20000AC493F7F7070AC8A384F5002A89AE84BD
:10EA300005C81C42054783C707006368F7060347FC
:10EA4000B400630FF700A305F40097900000E7807F
:10EA500040098347B400B9CF97D0FFFFE78040BE9D
:10EA600021649305B400280097B0FFFFE78080FB86
:10EA700097000000E78060F8AA85280097D0FFFF84
:10EA8000E78000DF014781463000A6854A8597B0C0
:10EA9000FFFFE780801E2904480822CC230A0100DA
:10EAA00002CE97E0FFFFE78040C305611733FFFF09
:10EAB0006700E36197D0FFFFE78020BF55B71733AA
:10EAC000FFFFE702835E01117C003ECAB707070023
:10EAD0003ECC7C003ECE83C795002E84AA8493F75B
:10EAE000F707A384F500A165AD05480897B0FFFFBF
:10EAF000E78040F397000000E78020F0AA854808EF
:10EB000097D0FFFFE780C0D6500801478146A28515
:10EB1000268597B0FFFFE780401605611733FFFF9A
:10EB20006700E35A9777FF1F938747079C43094580
:10EB300099C303C5C70082801733FFFFE702E3567E
:10EB400001117C00AE843ECAA165B70707002A8484
:10EB50003ECCD1057C0048083ECE97B0FFFFE78051
:10EB600060EC97000000E78020FCAA85480897D059
:10EB7000FFFFE780E0CF500801478146A685228548
:10EB800097B0FFFFE780600F05611733FFFF670055
:10EB900003541733FFFFE702435183C7950093F7F0
:10EBA000F707A384F50097000000E78020F91733EA
:10EBB000FFFF6700C3511733FFFFE702634D83C7B1
:10EBC00095000329C501411193F7F707A384F500C8
:10EBD0001C4283C90700854763E637079777FF1F05
:10EBE000938707539C432E84AA8485CF9700000007
:10EBF000E78080F389476306F502630409028347CF
:10EC0000C900638037032306390197900000E7802D
:10EC100040ED83572903898B89C797D00000E7808F
:10EC2000E0B72685A28597000000E78020F1A16764
:10EC3000CD0748003EC42302010002C697E0FFFF53
:10EC4000E780A0A941011733FFFF6700A34797772B
:10EC5000FF1F9387A7F49C431D4599C303C5E70095
:10EC600082801733FFFFE70243440111B707070013
:10EC70003EC683C79500584D0AC493F7F7070AC8E4
:10EC8000A384F5002A89AE8415C71C4283C70700F8
:10EC900093968701E18663C4060685466381D7069D
:10ECA0008346E7006388F6002307F700979000008B
:10ECB000E78020E321649305E400280097B0FFFF7C
:10ECC000E78040D697000000E780A0F8AA852800DA
:10ECD00097D0FFFFE780C0B9014781463000A68585
:10ECE0004A8597B0FFFFE78040F93504480822CCF9
:10ECF000230A010002CE97E0FFFFE780009E056136
:10ED00001733FFFF6700A33C1733FFFFE702E33928
:10ED100001117C003ECAB70707003ECC7C003ECE06
:10ED200083C795002E84AA8493F7F707A384F50080
:10ED3000A165B905480897B0FFFFE780A0CE97000E
:10ED40000000E78000F1AA85480897D0FFFFE78020
:10ED500020B2500801478146A285268597B0FFFF63
:10ED6000E780A0F105611733FFFF670043361733D3
:10ED7000FFFFE702E331AA8401441779FF1F13095B
:10ED800029E2E14997C0FFFFE78040C96344A4003E
:10ED9000014519A833053403832709003E9583579D
:10EDA00025006397970011051733FFFF6700833134
:10EDB0000504C9BF032E8500630A0E121773FF1FD7
:10EDC0001303C3FC0323030063150300294363906B
:10EDD000061203234E01631503001D4363990710B8
:10EDE0001733FFFFE702E329C689428A3E89BA8AC0
:10EDF000B684328BAE8B2A84B5E103554E0019E5FB
:10EE000001431A851733FFFF6700232BA167A98FE2
:10EE1000116763FBE70097000000E78080F58145FC
:10EE200097F0FFFFE780C0120844B70700E05841A1
:10EE3000F98F18455CC1B707001FF98F1CC55C49E5
:10EE400091C7610597E00000E780408BE38A09FAEB
:10EE5000228597900000E78060C65DB7328597C035
:10EE60000000E78040430D4349DD1C44116703D592
:10EE70004700A167A98F63FBE70097000000E780C8
:10EE800040EF814597F0FFFFE780800C032384006B
:10EE900093164B01D1828347B300035663008588E4
:10EEA000FD8BA305F300FD777D8E558EFD76FD1657
:10EEB000B204F18E83274301C58E231273012313FD
:10EEC000D3002304530123052301A3044301BDDF21
:10EED000228597B0FFFFE78020CDAA850844B5D1F1
:10EEE000610597D00000E780207F8DB71D431A850C
:10EEF00082801733FFFFE702A3190569AA84AE8950
:10EF0000328A0144FD5A7D1997C0FFFFE780C0A5F2
:10EF10006347A40001451733FFFF6700A31AD844D5
:10EF200093171400BA9703D70700631F3703239082
:10EF3000570163070A00268597900000E780A080AC
:10EF40009C449DC383D76700B3F72701639E3701B5
:10EF5000D28801488147014781460146814526857F
:10EF600097000000E78040E5050479BF1733FFFFF5
:10EF7000E702031279711C103EC4B7070F003EC6AA
:10EF80001C103EC883C79500AA8A328593F7F707FD
:10EF9000A384F5002E89328497D0FFFFE780009D7F
:10EFA00093170501C187635AF006AA89228597D075
:10EFB000FFFFE780A09B2A8A4E85032B040097B0B1
:10EFC000FFFFE780009B39ED8357440081440544EF
:10EFD000F11793B71700A303F10083457100DA8797
:10EFE0002287D2864E86280097E0FFFFE780E05711
:10EFF000014781463000CA85568597B0FFFFE780FC
:10F00000C0C7A1679387F70348083ECC230A810055
:10F0100026CE97D0FFFFE780406C45611733FFFF96
:10F020006700430AA2851306710097E0FFFFE7809F
:10F030006066AA84094455D1528597E0FFFFE780B6
:10F0400060D40D4459D90546D28526859700000025
:10F05000E78060EA2A8451B71733FFFFE702E30431
:10F06000835507000346270041112A842E8532C6A6
:10F070002EC497E0FFFFE780E0D001C93246A245E9
:10F08000228597000000E78000E741011733FFFF6A
:10F090006700E3031733FFFFE702A3FE83C7950072
:10F0A0004111AA8A93F7F707A384F5003285AE8948
:10F0B000328497D0FFFFE780608B93170501C187EB
:10F0C0006357F00AC1452A8A228597C0FFFFE7806F
:10F0D00080702A8D228597D0FFFFE78020892A89BA
:10F0E000228597D0FFFFE7804086930705F893F7C6
:10F0F000F70F1307E007AA8B637BF706228597D0EB
:10F10000FFFFE78080842A8C228597D0FFFFE7806D
:10F11000C083AA8C5285032B040097B0FFFFE780C1
:10F12000408539E983574400231101008144F117D8
:10F1300093B71700A300F10005440347110083565D
:10F140002100938784005685DA8822885286CE85EE
:10F1500097F0FFFFE78020A7A167E90748003EC4BA
:10F160002302810026C697D0FFFFE78000574101A8
:10F170001733FFFF670063F413061100A28597E0C1
:10F18000FFFFE7802051AA8409E52311010009440B
:10F190006DB7930521006A8597F0FFFFE780A0F027
:10F1A0002A8441FD835521009356C9001316490155
:10F1B00085486688E2875E87858A51822685970022
:10F1C0000000E78060BF2A848DBF1733FFFFE7028E
:10F1D00043EB83C7950041112A8B93F7F707A3846C
:10F1E000F5003285AE89328497C0FFFFE780007852
:10F1F00093170501C1876352F00A2A8A228597C0B6
:10F20000FFFFE780A076AA8A228597C0FFFFE780EC
:10F21000E0752A89228597C0FFFFE7800073930776
:10F2200005F893F7F70F1307E0072A8C6377F706C3
:10F23000228597C0FFFFE7804071AA8C228597C086
:10F24000FFFFE78080702A8D5285832B040097A0F2
:10F25000FFFFE780007239E583574400854401448D
:10F26000F11793B71700A301F1000347310093078B
:10F2700084005A85DE882688D6865286CE8597F009
:10F28000FFFFE78040948D4748003EC42302910071
:10F2900022C697D0FFFFE780404441011733FFFFAC
:10F2A0006700A3E1A2851306310097E0FFFFE78026
:10F2B000603E2A84894455D99356C90013164901E2
:10F2C00085486A88E6876287858A5182D685970055
:10F2D0000000E78060AEAA8449BF1733FFFFE70252
:10F2E00023DB2A8981440144617A916A177BFF1FDD
:10F2F000130BCBA997B0FFFFE780006863C7A4009A
:10F3000022851733FFFF6700E3DB8327090093990A
:10F310001400CE9703D50700330745014207418308
:10F320006364570305C103270B0019C785453E8554
:10F3300097400000E78060E9832709000504CE9725
:10F340002390070085047DB797000000E78060A246
:10F35000832709000504CE972390070065D58145D2
:10F3600097F0FFFFE780C0BEF1BF1733FFFFE70252
:10F3700023D283C7950041112A8A93F7F707A38404
:10F38000F50032852E89328497C0FFFFE780005E4A
:10F3900093170501C187635AF004AA89832A0400E0
:10F3A00097A0FFFFE780E05C31E583574400854488
:10F3B0000144F11793B71700A301F100034831008E
:10F3C000D68752850147CE862686CA8597D0FFFF0D
:10F3D000E780806AA167F50748003EC423029100D8
:10F3E00022C697D0FFFFE780402F41011733FFFF70
:10F3F000670043CDA2851306310097E0FFFFE78049
:10F4000060292A8489445DD99777FF1F93870798DD
:10F410009C4381CF044997B0FFFFE780E055AA8560
:10F42000268597400000E78040DA13050401970025
:10F430000000E780C0EA228597800000E780003363
:10F440008144ADBF1733FFFFE702A3C383C7950015
:10F450004111AA8A93F7F707A384F5003285AE8994
:10F4600032842311010097C0FFFFE78020509317DB
:10F470000501C1876354F0062A8AC145228597C0D9
:10F48000FFFFE7804035AA8B5285032B040097A02D
:10F49000FFFFE780004E21E9835744008544014483
:10F4A000F11793B71700A300F100034811000357A9
:10F4B0002100DA875685D2862686CE8597D0FFFF33
:10F4C000E780805BA1679387270248003EC4230240
:10F4D000910022C697D0FFFFE7802020410117331B
:10F4E000FFFF670083BDA2851306110097E0FFFFB1
:10F4F000E780401A2A8489444DD99777FF1F938764
:10F50000E78898433E8901CF044997B0FFFFE78021
:10F51000A046AA85268597400000E78000CB13050A
:10F52000040197000000E78080DB97B0FFFFE780D1
:10F53000A04495443DD9930521005E8597F0FFFFD7
:10F54000E78060B6AA8435F11C4803572100228564
:10F550002390E70097800000E7804021832709007F
:10F56000A9D70355210097400000E780A0BD35BF13
:10F570001733FFFFE702E3B083C795004111AA8A62
:10F5800093F7F707A384F5003285AE89328497C0DC
:10F59000FFFFE780A03D93170501C1876351F00687
:10F5A0002A8A228597C0FFFFE780403C2A8952853E
:10F5B000032B040097A0FFFFE780A03B31E58357B2
:10F5C000440085440144F11793B71700A301F100EB
:10F5D00003483100DA8756854A87D2862686CE854B
:10F5E00097D0FFFFE7804049A167F90748003EC474
:10F5F0002302910022C697D0FFFFE780000E410151
:10F600001733FFFF670063ABA2851306310097E055
:10F61000FFFFE78020082A8489445DD99167CA9753
:10F62000C2071167C1831307F7EF8544E362F7FA56
:10F630009767FF1F938787759843BE8B01CF044957
:10F6400097B0FFFFE7804033AA85268597400000EA
:10F65000E780A0B71305040197000000E78020C8E9
:10F6600097B0FFFFE780403195443DD11C4822858B
:10F6700081442390270197800000E780200F83A713
:10F680000B00B9D74A8597400000E780A0AB89B747
:10F690001733FFFFE70263A12A844105B284970074
:10F6A0000000E780C0C311C5228597800000E78075
:10F6B000E00B81460146A685228597800000E78001
:10F6C000C04E1C4C89C7DC4799C3228582971733EB
:10F6D000FFFF6700C39F9767FF1F9387274C9C43DB
:10F6E000014599C31385070182809767FF1F9387A0
:10F6F000E74A884382801733FFFFE702039B931793
:10F70000C600DD8DC2054111C1812A8432C697C071
:10F71000FFFFE780E0173246228511829375F60FCE
:10F7200097C0FFFFE780C01441011733FFFF670058
:10F73000039A1733FFFFE702A39579713C083ED285
:10F74000B7070C003ED43C083ED683C79500AE8474
:10F750002A8993F7F707A384F500A16593853504FB
:10F76000481097A0FFFFE780E02BC165FD1501441D
:10F77000176AFF1F130A0A63930A400EAE892E8B85
:10F780002EC697B0FFFFE7802022420593170401A1
:10F790004181C183B24563E9A702C167FD17638751
:10F7A000F500481097C0FFFFE780800E501001471A
:10F7B0008146A6854A8597A0FFFFE780004C4561FA
:10F7C0001733FFFF670003903307540383270A0BA7
:10F7D000BA9703D6C701630A3601638A3501481018
:10F7E00097000000E78060F1DA85050451BFB2851B
:10F7F000EDBF1733FFFFE702C38879717C083EC86D
:10F80000B70711003ECA7C083ECC83C79500AA8981
:10F81000328593F7F707A384F5002E8997C0FFFF81
:10F82000E780C01485676378F504A165AA8489051B
:10F83000080897A0FFFFE780E01E2685974000009C
:10F84000E78060ED133415000A04A285080897C00C
:10F85000FFFFE780E001A685080897C0FFFFE7806B
:10F86000200325CC014781461008CA854E8597A004
:10F87000FFFFE780804045611733FFFF6700E383A8
:10F88000B30754030327CA0ABA9703D70700631CB8
:10F89000970003D6270063806505080897000000DD
:10F8A000E780A0E5DE8505042EC697B0FFFFE78060
:10F8B000A0104205931704014181C183B245E3E1E1
:10F8C000A7FCC167FD17E38FF5F8080897C0FFFF95
:10F8D000E78000FC41BFB285F9B7C165FD15014461
:10F8E000176AFF1F130A0A4C930A80022E8BAE8BF5
:10F8F00065BF1723FFFFE702437B184183471700CB
:10F9000083460700A207D58FD207D1832390F50045
:10F9100083472700034717008D45A207D98F91839E
:10F920002310F60097C0FFFFE780A0E91723FFFF31
:10F930006700E3791723FFFFE7028375C164014481
:10F940001769FF1F1309094693098002FD1497B038
:10F95000FFFFE78060066347A40001451723FFFF10
:10F9600067004376330534038327C90A3E958357DE
:10F970000500E38597FE0504D9BF1723FFFFE702C3
:10F9800023712A8AAE89B284B68A97400000E78044
:10F9900080D819E591473E851723FFFF67008372E2
:10F9A0002A894E8597C00000E780E08E2A84638E06
:10F9B0000A048D476DD103570500C547E31D47FD78
:10F9C0000347F9018546AD47E317D7FC8347450058
:10F9D00081CF4146A6855D0597F00000E780C09E77
:10F9E000814755D9AD4745BF130965012302E5009D
:10F9F000CA85268597100000E780606231C1A5475F
:10FA0000E38B0AF82302040079B705C18357050088
:10FA1000E39247F94146A685190597F00000E78073
:10FA2000A09A81472DD99947BDB74E859700000010
:10FA3000E78080F02A84954739DD130955004DBFD2
:10FA40004146A685231044012311340113051900F2
:10FA500097F00000E780A099228597800000E7805A
:10FA6000A0EA81470DBF1723FFFFE7020364797106
:10FA70007C003ECCB7070A003ECE7C003ED083C758
:10FA80009500B2842E8493F7F707A384F50013063C
:10FA9000A1002A892C00268597000000E780A0E5B8
:10FAA000A16528088D0597A0FFFFE780A0F790408B
:10FAB0008355A10003558100854697000000E7802B
:10FAC00000ECAA84AA85280897C0FFFFE78040DAE7
:10FAD0000356A10083558100280897000000E780A5
:10FAE000C0C1300801478146A2854A8597A0FFFF23
:10FAF000E780A018854748103ED42302910202D621
:10FB000097D0FFFFE78060BD45611723FFFF6700C7
:10FB1000035C1723FFFFE702435979717C003ECC59
:10FB2000B7070A003ECE7C003ED083C79500B28462
:10FB30002E8493F7F707A384F5001306A1002A8902
:10FB40002C00268597000000E780E0DAA1652808F0
:10FB50008D0597A0FFFFE780E0EC90408355A10062
:10FB600003558100814697000000E78040E1AA84A8
:10FB7000AA85280897C0FFFFE78080CF0356A10021
:10FB800083558100280897000000E78000B73008FF
:10FB900001478146A2854A8597A0FFFFE780E00DD7
:10FBA00048102302910202D402D697D0FFFFE780CB
:10FBB000C0B245611723FFFF670063511723FFFFA2
:10FBC000E702A34E97000000E78060DB1723FFFFEA
:10FBD0006700E34F9767FF1F938787FC8843828006
:10FBE0001723FFFFE702634C835725004111AE84C2
:10FBF0002A842307B10017F5FFFF130525466C0083
:10FC00002316F10097A0FFFFE780204991C42285C9
:10FC100097800000E780E0D6FD572310F40013061C
:10FC200020028145130554009720FFFFE780E04A3A
:10FC300041011723FFFF670083491723FFFFE702F6
:10FC4000234579717C003ECCB7070A003ECE7C008C
:10FC50003ED083C79500AA89AE8493F7F707328513
:10FC6000A384F5001306A1002C0097000000E78094
:10FC700080C803558100114497400000E780A0A987
:10FC800015C50355A100014497B00000E780A060AE
:10FC900011CD035705008357810045446318F700D1
:10FCA000854597000000E780E0F301442169930552
:10FCB0003900280897A0FFFFE780C0D6A285280852
:10FCC00097C0FFFFE780C0BA0356A10083558100AB
:10FCD000280897000000E78040A2300801478146CD
:10FCE000A6854E8597A0FFFFE78020F948104AD4EB
:10FCF0002302810202D697D0FFFFE780009E456174
:10FD00001723FFFF6700033C1723FFFFE702433879
:10FD10009767FF1F938787E82A8488432E8915C534
:10FD2000035745038357C4016311F70223260502D5
:10FD300023180502410597D00000E780209C630648
:10FD4000090097800000E78060DB81449769FF1F0E
:10FD500093894905130A800297B0FFFFE780C0C569
:10FD600063C4A4049767FF1F938707EC9C4399C75C
:10FD70000355C40197200000E780C0BD6307090058
:10FD8000228597800000E780C0A01306400E8145C1
:10FD900022859720FFFFE7804034FD57231EF400A3
:10FDA0001723FFFF670003323385440383A7C90A83
:10FDB0003E95035705008357C4016317F700CA85B2
:10FDC00097000000E78000E2850479B71723FFFF62
:10FDD000E702032C83C795004111AA8993F7F7071F
:10FDE000A384F5003285AE8497C0FFFFE78000B89A
:10FDF00085676378F5042A8997400000E780A09121
:10FE0000014401CD83D7040031446388270185452F
:10FE100097000000E78080EF01444E85A2864A8665
:10FE2000A68597D0FFFFE780A09CA1679387170462
:10FE300048003EC42302810002C697D0FFFFE7803E
:10FE4000C08941011723FFFF6700C3271723FFFF66
:10FE5000E70203249767FF1F938747D4804329C491
:10FE6000014597C00000E780002181470148C16437
:10FE70001CDC232E0403232004041769FF1F13092D
:10FE800069F201449309400EFD1497B0FFFFE7802B
:10FE9000A0B1634FA400814517F5FFFF1305857FCF
:10FEA00097A0FFFFE780601F1723FFFF67008321F4
:10FEB000330534038327090B3E958357C5016387B8
:10FEC0009700854597000000E78040E4050475BF72
:10FED0009357050113D78700A380F50093170501F9
:10FEE000C183A1832380E5002381F500A381A500C0
:10FEF00082801723FFFFE702431B2300050083C70F
:10FF00001500A300F50083C725002301F50083C772
:10FF10003500A301F50083C745002302F50083C720
:10FF20005500A302F50083C7650093059500A30360
:10FF300005002303F5002304050032859700000027
:10FF4000E78040F91723FFFF670063181723FFFFBF
:10FF5000E70203144111E9540DCD85CD93F9C5FF96
:10FF60002E842A89AA84338AA900B7EA0400631878
:10FF70009A020D88854411CCB7E704009C5F8297F4
:10FF80002AC622866C003305390197E00000E7801D
:10FF90000046268541011723FFFF6700A31283A7B0
:10FFA0008A039104829793170501C183A183A38ECD
:10FFB000F4FE93570501238FF4FEA183238EA4FE44
:10FFC000A38FF4FE6DB763E6D5021723FFFFE702A8
:10FFD000C30DB28741113686BE8536C697E0000054
:10FFE000E780E040B246410136851723FFFF6700F6
:10FFF000030E814636858280838705001387F500CE
:020000040001F9
:100000003D05FD8793F77708834607007D15860633
:10001000B58FA300F5006307B7007D17834717006E
:100020009D83DDB782801723FFFFE7020308B7E750
:10003000040083A7070932872A863A8582971335F9
:1000400015001723FFFF6700830815C181478DC185
:100050001723FFFFE7026305414697E00000E780B2
:10006000003985473E851723FFFF67004306814718
:100070003E8582801DCD1723FFFFE7020303414623
:1000800081452A849720FFFFE7802005414681456E
:10009000130504039720FFFFE78020040147C16791
:1000A0002322040438C87CC805451723FFFF6700D6
:1000B00003020145828081473DCDB5CD1723FFFF67
:1000C000E702A3FEB2842E891306800581452A84A7
:1000D0009720FFFFE7806000CA8524C4268597002B
:1000E0000000E780C0F64146814522859720FFFF4A
:1000F000E780A0FE3044A285228597000000E780BB
:10010000C0F293040401A285268597000000E780D1
:10011000E0EEA6851305040297000000E78000EEDC
:10012000228597000000E78020F585473E8517234C
:10013000FFFF6700C3F93E8582801723FFFFE702B8
:1001400023F54111E9540DCD85CD93F9C5FF2E84DA
:100150002A89AA84338AA900B7EA04006398440371
:100160000D88814411CCB7E704009C5F82972AC6B2
:1001700022866C003305390197E00000E7802027D4
:10018000268541011723FFFF6700C3F383A78A0376
:100190009104829793170501C183A183A38EF4FE76
:1001A00093570501238FF4FEA183238EA4FEA38F12
:1001B000F4FE6DB765CD1723FFFFE70263EDB28450
:1001C00011E605451723FFFF6700C3EF2A842E8938
:1001D0000145EDD93C487848B3E6E700E5D693867B
:1001E000F7FFB3B7F6007D17032A4404BA9734C863
:1001F0007CC863050A06C14913050A03B38949414E
:100200002295637D3601B2862E86A6859700000072
:10021000E780A0DB7C40BE9464C065B7CE862E86A6
:10022000CE8597000000E78040DAC114D2944E9941
:1002300023220404A2879306040103C7070003C610
:1002400007038507318FA38FE7FEE398F6FE30445E
:10025000A285228597000000E78020DD2699C1490C
:100260003306994063EC9900A9DCA686A6851305A0
:10027000040397000000E78040D579BF8147B306AB
:10028000F4003307F6000347070083C5060085071F
:100290002D8F2380E600E39437FF3044A28522852A
:1002A00097000000E78060D8C1145DBF01458280DF
:1002B0000DC11723FFFFE70243DF130680058145C9
:1002C0009720FFFFE78060E105451723FFFF6700E8
:1002D00003E001458280814749C5C1C51723FFFF5F
:1002E000E702A3DCFC4141462E84AA846399C7043B
:1002F00013860501A2878146C14503C7070003C5D0
:1003000007038507298F3305D600034505008506B9
:10031000298FA38FE7FEE392B6FE3044A28526859F
:1003200097000000E78060D0228597000000E780FA
:1003300060F885473E851723FFFF670043D9138583
:1003400007031D8E814522959720FFFFE780E0D8A7
:100350007C40130700F813060402A2972388E702E3
:1003600051BF3E8582801723FFFFE70203D46D71E2
:100370002E84B284AA859010280036899700000048
:10038000E780A0D309EDD55725A050400C402800A8
:1003900097000000E78040E27DD5FD142104F5F4CC
:1003A0002C004A8597000000E78020F3814761DD3B
:1003B0003E8551611723FFFF670063D11723FFFFBD
:1003C000E702A3CE41112EC432C62C000546970089
:1003D0000000E78080F941011723FFFF670023CF6A
:1003E0001723FFFFE70263CC01112A842EC602C83F
:1003F00002CA02CC02CE97E00000E780402BB24652
:100400002A86A285080897000000E78060FB137524
:10041000F50F05611723FFFF670063CB1723FFFF6D
:10042000E702A3C87971B2872A8421462308B10064
:1004300013051101BE853AC436C697E00000E78077
:1004400000FBB24693059101368597000000E780D6
:1004500060A82285141035460C0897000000E7803C
:1004600020F62A84224701E921460C103A8597E0BC
:100470000000E780C0F7228545611723FFFF670072
:1004800003C51723FFFFE70243C27171AE84AA853B
:100490000A85328497000000E78060BB11C90A8694
:1004A000A685228597000000E78020B8814711E1EA
:1004B000C5473E854D611723FFFF670043C11723E2
:1004C000FFFFE70283BB1D712A8AB289BE843546CD
:1004D0008547130511012E8CB68A3A8BC28C468D46
:1004E0002308F10097E00000E78060F010100C088E
:1004F0005285231F010097000000E780C0F82A847E
:100500003DEDA1476313FD089307900591E0E54792
:100510003546E2851305110113990A012308F100FC
:100520001359090197E00000E78060EC1357890038
:1005300093978A00D98F90080C085285231FF100E9
:1005400097000000E78020F42A8415E9A1E493874E
:10055000FA0091831379F9003EC6631309004149FB
:10056000668B8144C14B854DB247639F970C6A8669
:100570008C0033855C0197E00000E78040E722852E
:1005800025611723FFFF670003B393079004C9F0A9
:10059000A547BDBF834701050947C14B2308F100AB
:1005A00083471105A58FA308F10093872400814498
:1005B00063E1FB04014714083386E6008C08B38628
:1005C000E400BA95DA9683C6060083C505000507E0
:1005D000AD8E2300D600E390E7FE4147639CE7041D
:1005E00090080C08528597000000E780C0E925D1EB
:1005F00081A0B3069B00BA871008B305F6009008E7
:100600003E9603C506000346060085078506298E2B
:100610002380C500E39277FF998F90080C085285DC
:10062000BE9497000000E78000E68947014749D162
:100630002A84B1B790083E96034606001408BE9679
:100640002380C600850759BFB24785046387971486
:1006500081471808B306F70098083E973386F900DB
:1006600003470700034606008507318F2380E60015
:10067000E39177FF90080C08528597000000E7800F
:1006800080E05DF53546E285130511012308B101CF
:1006900097E00000E780A0D513970401418393976A
:1006A00084002183D98F10180C085285231FF10074
:1006B00097000000E78020DD25FD81471018338773
:1006C000F9003E960347070003460600B306FB0009
:1006D0008507318F2380E600E39277FF65A818082D
:1006E000B306F70098083E973386F90003470700E2
:1006F000034606008507318F2380E600E3E127FFEC
:10070000CA87639E770990080C08528597000000FD
:10071000E78060D711FD81479800B306F700900885
:1007200018103E973E9603470700034606008507CC
:10073000318F2380E600E39177FF3546E28513058C
:1007400011012308B10197E00000E78040CA139728
:1007500004014183939784002183D98F10180C08DA
:100760005285231FF10097000000E780C0D1E311FC
:1007700005EC814710183387F9003E9603470700C0
:1007800003460600B306FB008507318F2380E60091
:10079000E3E227FFC109410BC1BB814785B794083C
:1007A000BE9683C6060018083E972300D70085072B
:1007B00089BF638006321723FFFFE702038C59715C
:1007C0002A84BE89B28B85473546130511022E8BCC
:1007D000468C4289BA8A368A2300F10297E00000EB
:1007E000E780E0C010180C10228523170102970043
:1007F0000000E78040C963180512A147631FFC068B
:100800009307900563930900E5473546DA8513059C
:10081000110293140A012300F102C18097E0000045
:10082000E780E0BC93178A0013D78400D98F900823
:100830000C1022852317F10297000000E780A0C466
:100840007DE1639209049307FA00BD88918391E0EA
:10085000C144C207C183DE8C814A3EC6414DB247C6
:1008600063E2FA0E6286B3854B01881097E00000C0
:10087000E78080B54DC93D557DA093079004E39670
:1008800009F8A54759B7834701050947C14C23001B
:10089000F10283471105B3C7F900A300F102938762
:1008A0002900814963E1FC04814618103306D70012
:1008B0008C083387D900B69556970347070083C540
:1008C000050085062D8F2300E600E390D7FE414703
:1008D0006390E70690080C10228597000000E780DF
:1008E00080BA35D189A0B3863A01BA871010B30512
:1008F000F60090083E9603C50600034606008507ED
:100900008506298E2380C500E39297FF3387EC404C
:1009100090080C102285BA9997000000E780A0B6D5
:100920008947014741D165611713FFFF6700A3782D
:1009300090083E96034606001410BE962380C6001B
:10094000850779B7B247850A93990A01939D8A0072
:1009500093D909016391570F85473546DA85130509
:1009600011022300F10293D9890097E00000E7808B
:1009700000A8B3ED3D0190000C1022852317B103B0
:1009800097000000E78020B059FD8147A68963EAFF
:10099000970626860C084A8597E00000E78020A588
:1009A00081471810B306F700100898083E973E9646
:1009B00003470700034606008507318F2380E600C2
:1009C000E3E197FE639FA90590080C10228597002C
:1009D0000000E78040AB21F981479810B306F7008B
:1009E000900818183E973E960347070003460600F6
:1009F0008507318F2380E600E391A7FF4109C10CF1
:100A0000B9BD18089000B306F7003E963387FC0086
:100A100003470700034606008507318F2380E60061
:100A2000B5B798084E97034707001C10CE97238050
:100A3000E700850941BF85473546DA851305110270
:100A40002300F10293D9890097E00000E780209A03
:100A5000B3ED3D0190000C1022852317B1039700E0
:100A60000000E78040A2E31005EC814718089000E1
:100A7000B306F7003E963387FC00034707000346A2
:100A800006008507318F2380E600E391A7FF4146EA
:100A90000C084A8597E00000E780609581471810B0
:100AA000B306F700100898083E973E9603470700E4
:100AB000034606008507318F2380E600E391A7FFF8
:100AC00090080C10228597000000E780C09B1DD580
:100AD00099BD7D5582801713FFFFE702035D011169
:100AE0002A842E8593055100328902C002C202C4B5
:100AF00002C69304740097F0FFFFE780A03D1D46F7
:100B0000A6851305910097E00000E780408E10084D
:100B10008A854A8597000000E780E09619ED9307E3
:100B20001400180883C60700034607008507050759
:100B3000B18EA38FD7FEE397F4FE05611713FFFF75
:100B40006700E3581713FFFFE70283542E848C419C
:100B50004111AA89838715003289914463D3070024
:100B6000A1449757FF1F9387A75A9C43A1C7C1CAA7
:100B70008D472310F10083C725004A852301F1002A
:100B800083C73500A301F10083C745002302F100AC
:100B900083C75500A302F10083C765009305910048
:100BA000A30301002303F1002304010097F0FFFFDA
:100BB000E78040320C404A860A8597F0FFFFE780C5
:100BC00080330328040083564400A6881D0881470B
:100BD0000147E51642868A854E8597000000E7802A
:100BE000408E2A8919E5A685228597B0FFFFE78008
:100BF000E0C14A8541011713FFFF6700A34C4A86F5
:100C00000A8597F0FFFFE780002F6DB71713FFFFEE
:100C1000E70203482E848C414111AA89838715007D
:100C20003289914463D30700A1449757FF1F9387EC
:100C3000274E9C43A1C7C1C68D472310F10083C72F
:100C400025004A852301F10083C73500A301F10087
:100C500083C745002302F10083C75500A302F100BA
:100C600083C7650093059100A30301002303F100EE
:100C70002304010097F0FFFFE780C0250C404A865F
:100C80000A8597F0FFFFE78000278356440003287A
:100C900004008A85858EC2061D08C1822312D400F5
:100CA000A68881470147E51642864E8597000000D9
:100CB000E78060B041011713FFFF6700A3404A8639
:100CC0000A8597F0FFFFE78000234DBF1713FFFF52
:100CD000E702A33DB335B000011185052A8913153C
:100CE000F601336515012308B1009305110136841F
:100CF0003AC632C03EC442C297F0FFFFE780801D73
:100D0000A2471248425593D68700230BF100930562
:100D1000910193578800A30AD100A30BF100230C83
:100D2000010197F0FFFFE780E01A324702460328EF
:100D30000400B337E000835644009207914411C287
:100D4000A1444A85A68842860C0897F0FFFFE780F9
:100D500040772A8919E5A685228597B0FFFFE780AD
:100D6000E0AA4A8505611713FFFF67004336171392
:100D7000FFFFE702E33101113EC68647B335B000FD
:100D80008505AA891315F6015D8D2308B100930529
:100D9000110136843A89B28442C446C297F0FFFFFB
:100DA000E780401322489248164593578800A30ACB
:100DB000F1009305910193D78800230B0101A30B48
:100DC000F100230C110197F0FFFFE780A0103247DC
:100DD000104083564400B337E0009207032809000F
:100DE000914891C0A1480C084E8597000000E7800B
:100DF000809CAA8401E9835544004A8597B0FFFF8F
:100E0000E780C0A0268505611713FFFF6700832BCD
:100E1000AA959307F00F171701001307679E631732
:100E2000B50013C5F7FF1375F50F828005058346DE
:100E3000F5FFB58FBA9783C70700D5B703574500AD
:100E400014419307F00F171601001306669B36979F
:100E500042074183139506014181631BE500AD8F75
:100E6000B29703C50700130515F3133515008280EB
:100E7000850603C5F6FFA98FB29783C70700D9BFC0
:100E80001713FFFFE7026322B28736842E86BA86E5
:100E9000AA853E85BA8497F0FFFFE7806052634FD2
:100EA0000500228597E00000E78060802A86A686FC
:100EB000A285268597F0FFFFE78080501713FFFF7C
:100EC0006700E3201713FFFFE702831C5D712A8B85
:100ED000AE8A17150100130525902C00B284368ABE
:100EE000BA893E8997F0FFFFE780C04F2A845DE111
:100EF00034104146DA85280097F0FFFFE780404C28
:100F00002A8449E98547A303F100A6C2930771002B
:100F10002408BEC4A68685470D462C18281002DC7E
:100F200002DED6C0BEC697F0FFFFE78000442A84E9
:100F300035E183477102A6860D4693F7F707230034
:100F4000FA00C1473EDE2C188947281026DCA3038F
:100F5000F10097F0FFFFE78040412A8405ED41460C
:100F6000A6854E8597D00000E78060488D47A6860D
:100F70000D462C182810A303F10097F0FFFFE7801F
:100F8000C03E2A8401E94146A6854A8597D00000E3
:100F9000E780E045228561611713FFFF6700831238
:100FA0001713FFFFE702631097F70000938707EF1F
:100FB000984383C7470079712A89AE8417150100C9
:100FC000130505820C083AC42306F10097F0FFFFD1
:100FD000E78040412A8405ED14104146CA8508087F
:100FE00097F0FFFFE780C03D2A8415E114081546FD
:100FF0002C00081097F0FFFFE780803C2A8401E96D
:1010000021462C08268597D00000E780403E2285A7
:1010100045611713FFFF6700830B1713FFFFE702FC
:10102000C30897F70000938767E79C477971AA8404
:101030002E84170501001305257B0C083EC697F08A
:10104000FFFFE780203A0DE914104146A685080805
:1010500097F0FFFFE780C03605E1140811466C00E9
:10106000081097F0FFFFE780A03519E58347F101ED
:1010700093F7F7032300F40045611713FFFF6700A0
:1010800003051713FFFFE70243023688A148814793
:101090000147E54697F0FFFFE780A0421713FFFFE7
:1010A0006700E3021713FFFFE70223003688A14819
:1010B00081470147E54697F0FFFFE780C06F1713B0
:1010C000FFFF6700C3001713FFFFE70203FE0111D4
:1010D0002A842E850C0832C697F0FFFFE780803007
:1010E00009ED3247970601009386866E1008C145C8
:1010F000228597000000E780E0D805611713FFFF05
:101100006700E3FC1713FFFFE70223FA4111C14711
:101110002EC032C48A8509463EC23EC697F0FFFF04
:10112000E780A02441011713FFFF670043FA17135C
:10113000FFFFE70283F74111AE8613061009AA8567
:101140000A8502C002C202C402C697F0FFFFE78010
:10115000202741011713FFFF670063F71713FFFFF5
:10116000E702A3F4328797060100938666682E860D
:101170009305000297000000E780C0D01713FFFF1F
:101180006700E3F41713FFFFE70223F27971C14709
:101190002ACC2ED032D42C080D4628003ECE3ED28A
:1011A0003ED602C402C602C802CA97F0FFFFE7801B
:1011B000C01B45611713FFFF670063F11713FFFFA3
:1011C000E702A3EE0111AA842E841705010013057E
:1011D000A5628A8597F0FFFFE780C02015E5140817
:1011E0004146A6850A8597F0FFFFE780601D09ED5F
:1011F0008347E1010347F101A207D98FCA07C983D9
:101200006177D98F2310F40005611713FFFF670082
:1012100003EC15CD1713FFFFE70223E99757FF1FD4
:101220009387879C90439755FF1F9385259C17555F
:10123000FF1F1305659797D00000E78000C517557D
:10124000FF1F130565961713FFFF670043E8175547
:10125000FF1F1305659582808DCD1713FFFFE702F1
:10126000C3E49757FF1F93872798944301112E8457
:101270000A869755FF1F9385659797D00000E780F2
:1012800040C60A850294014505611713FFFF6700F8
:1012900003E47D5582801713FFFFE70203E197D037
:1012A0000000E78080D19757FF1F23AFA79217F563
:1012B000FFFF1305E5C997B00000E780C07417135E
:1012C000FFFF6700C3E01757FF1F1307279493170B
:1012D000150008433E95FD572310F5008280171333
:1012E000FFFFE70283DC2A84084009E51713FFFFAC
:1012F0006700E3DD1C4158401CC06313E5005CC07F
:101300008347550023200500F99BA302F50097A011
:10131000FFFFE780207CC9BF1713FFFFE70243D719
:101320009757FF1F9387879098432A8411CB834751
:10133000350093F7070289C70355050089450297D1
:101340001305440197B00000E780403B835504003B
:101350000355E40097300000E780A00C485819C5F9
:1013600097A0FFFFE7800077232A04021305840378
:1013700097000000E780E0F68144B1499790FFFFB5
:10138000E780C06D63CBA4028347340023200404AC
:1013900093F727FCA301F40000489790FFFFE78034
:1013A000E06C13161500814522859710FFFFE7803A
:1013B000C0D21713FFFF6700E3D0B38734030329BC
:1013C000040385043E994A8597000000E78060F198
:1013D0002304090065B78347350093F7070299E3B3
:1013E000014582808357E500E39CB7FEC167FD1786
:1013F0006316F60005458280054599A81713FFFF7F
:10140000E702A3CA93170601C187B2842A8401495F
:101410006359F002835705009DCB01456367F600D1
:10142000034584003E953325A6001375F50F0DA0E6
:101430001C4813171900BA9783D70700E38E97FA51
:1014400005099790FFFFE7806062E343A9FE01452D
:101450001713FFFF6700A3C71713FFFFE70243C37C
:10146000AE89AA849790FFFFE78000562A8497D020
:10147000FFFFE780A02EAA86014713068401970587
:101480000000938585E41745FF1F13056578979045
:10149000FFFFE780801C2A8925C98C441304C500FE
:1014A00022859E0593F5050897A0FFFFE780403C45
:1014B000CC4083877400E18163DD070493E5050870
:1014C000228597A0FFFFE780A03A0D469385440050
:1014D000228597A0FFFFE780C03683D504002285D0
:1014E00097A0FFFFE780E03D83D52400228597A0E9
:1014F000FFFFE780003D03D6490083A50900228550
:1015000097A0FFFFE780E0334A851713FFFF6700CE
:1015100063BB93F5F5076DB71713FFFFE702E3B859
:1015200001112A84328532C697A0FFFFE780E027A9
:101530009780FFFFE7806034835704001757FF1F31
:10154000130747863246231BF100930700F8A30DCB
:10155000F1001C471843231AA1008983858BB30728
:10156000F740B28548083ECE231C0100230D010040
:1015700097000000E78080EE05611713FFFF67000A
:1015800003B51713FFFFE702A3B0004101453DC4B7
:101590009304C40026853289AE8997A0FFFFE780B7
:1015A000C02495452A8A2685035B040197A0FFFF86
:1015B000E7802021268597A0FFFFE780603E8D45CC
:1015C000AA8A268597A0FFFFE780A01F268597A0FF
:1015D000FFFFE780E03C5C48420A135A0A01D297B9
:1015E0005CC423186401814763983A0146054D8124
:1015F000330625419337160013F5F70F1713FFFF36
:10160000670043AC1713FFFFE702A3A789692A8B82
:10161000AE8B328AB68A81440144314CFD199790D1
:10162000FFFFE780A04363CDA4009790FFFFE78012
:10163000E045018D33B5AA001713FFFF6700E3A74C
:101640003389840383270B003E9963170A0083477D
:10165000890085043E94E1B703560A00DE854A8579
:1016600033F6C90097000000E780E0F16DD1054531
:10167000E1B71713FFFFE70243A301112A847C009F
:101680000355E5003ECAB70707003ECC7C003ECEBE
:1016900097200000E78020082A898545480897A000
:1016A000FFFFE78020399945480897A0FFFFE780B2
:1016B000E015AA844A8597200000E780A0082380CF
:1016C000A4009747FF1F9387E76D9C43416613066D
:1016D00006F09396870113D78701558F93D687001D
:1016E000F18E558FA207B706FF00F58FD98F1146EF
:1016F0002C00138514003EC497D00000E78020CF53
:101700005008A38204008945228597000000E780E5
:10171000E0E019C9AA851305840397A0FFFFE780BD
:10172000E0313C4085073CC005611713FFFF6700AF
:10173000039A1713FFFFE70243979790FFFFE78095
:10174000E0342A8405049790FFFFE78020333305B7
:10175000A402F14791453305F50297200000E78088
:1017600020BA11E565551713FFFF670043969747A9
:10177000FF1F23A5A74A9790FFFFE78020312A8407
:1017800005049790FFFFE780602F3305A402894589
:10179000060597200000E780A0B669D59747FF1F90
:1017A00023A6A7469790FFFFE780402E2A840504D2
:1017B0009790FFFFE780802C3304A4029747FF1F18
:1017C000239887449790FFFFE780402C2A849790C6
:1017D000FFFFE780A02A930714003385A7029747ED
:1017E000FF1F2398A742970701009387A7C41747B5
:1017F000FF1F2323F7420145BDB71713FFFFE70281
:101800002389AA842E8901449749FF1F9389895906
:10181000130A80069790FFFFE78040266347A400E5
:1018200001451713FFFF6700E3893305440383A7CE
:1018300009024A86A6853E9597000000E780E0B938
:1018400019E10504C1BF0545E9BF1713FFFFE70212
:101850004383AA8A2E8BB28B368C3A8A8144014408
:101860008149974CFF1F938CEC53130D8006979082
:10187000FFFFE780A02063C9A40011E085494E85E1
:101880001713FFFF670063833389A40383A70C0248
:101890005E86D6853E994A8597000000E780E0B3D2
:1018A0001DC19790FFFFE780601E0544636D4501F1
:1018B000D2866286DA851305090397000000E78067
:1018C000A0D411C1854985045DB71703FFFFE70266
:1018D000237CC16441112A8901449749FF1F9389E0
:1018E000694C130A8006FD1436C632C42EC2979086
:1018F000FFFFE780A01892452246B2466348A40045
:10190000014541011703FFFF6700C37B3305440313
:1019100083A709023E9509C683473500C18B9DC741
:1019200091C68347350093F707028DC3630699007C
:101930008357E500639C27010357050001CB63E74C
:10194000E50083478500BA97E3CDF5FA050469BF42
:101950001703FFFFE702C373C1642A890144974953
:10196000FF1F93892944130A8006FD149790FFFFF7
:10197000E780C0106346A4001703FFFF670083746D
:101980003305440383A709023E958357E500638A24
:101990009700630499006396270197000000E78091
:1019A000E0970504E1B71703FFFFE702036D8969BC
:1019B0002A8AAE8A328BB68B8144174CFF1F130CD8
:1019C0006C3E930C8006314DFD199790FFFFE78028
:1019D000E00A63C6A4001703FFFF6700C36D3389E5
:1019E000940383270C028355CA015A863E994A857F
:1019F00097000000E780609E31C1814D15A03384BF
:101A0000AD038327090303D60B00D68533F6C9003F
:101A10003E94228597000000E780E0B609E9850D35
:101A20009790FFFFE7808003E3CBADFC01A8228500
:101A300097000000E780E08A23040400850471B762
:101A40001703FFFFE702E3634169AA8A014A174BC4
:101A5000FF1F130B2B357D19C14B054C9790FFFFD2
:101A6000E780C0016346AA001703FFFF6700E36435
:101A700093098006B3073A0383290B02BE9983D7E3
:101A8000E900638E270163842A01639A570103A446
:101A9000890301E84E8597000000E780C0BD050A74
:101AA00075BF83570401639977099304C4002685A1
:101AB00097A0FFFFE78060D385452A8D2685835C4C
:101AC000040197A0FFFFE780C0CF268597A0FFFF06
:101AD000E780A0E762056185635905048D45268589
:101AE00097A0FFFFE780E0CD8945268597A0FFFFFF
:101AF000E78020CD8945268597A0FFFFE78060CC51
:101B00008545268597A0FFFFE780E0CC8347050049
:101B1000094793F7F707639AE7009945268597A049
:101B2000FFFFE78040CBA30285014848337D2D01AC
:101B3000231894016A9548C40040A1BF1703FFFF12
:101B4000E702A35637E404008327041D82979747D2
:101B5000FF1F83C727121725FF1F13056599A300D1
:101B6000F5008327441C82978327841C8146130633
:101B7000F00F8145014582971703FFFF670023554A
:101B80001747FF1F130707FF18439745FF1F83C51C
:101B9000650E9747FF1F9387670C834687030346AD
:101BA00097036397D5009747FF1F2385C70C828053
:101BB00083C587010347A7036317B6009747FF1F35
:101BC000238AE70A828003C687016317C700974705
:101BD000FF1F2381D70A828083C687011307500223
:101BE0006319D700930760021747FF1F2304F70804
:101BF000828083C68701130660026315D6009307AF
:101C00007002DDB783C7870155BF9747FF1F9387D2
:101C1000E704D44B0947638DE6081703FFFFE7028B
:101C2000C3481749FF1F1309A9003E8483470900D1
:101C3000918B9DCFB7E4040083A7041D829783A7EF
:101C4000441C1745FF1F130525FF829783A7841C9B
:101C500081461746FF1F03462600814501458297AE
:101C600021C583470900ED9B1747FF1F2302F7FC9F
:101C70008347040093F7F70F85CB91471747FF1F62
:101C80002328F7FE97000000E78080EB9700000014
:101C9000E78040EFB7E70400BC4F41469145174548
:101CA000FF1F034525FC82971703FFFF67002342B0
:101CB00082801703FFFFE702433F8D474111630610
:101CC000F504C5476308F50285476310F502974799
:101CD000FF1F2383A7FAB7E70400BC4B930500104E
:101CE0001745FF1F034505F8829741011703FFFFC2
:101CF0006700E33D85471747FF1F230FF7F6B7E758
:101D00000400BC4B93050020E1BF9747FF1F93875A
:101D1000E7F4D44B1147638DE600B7E7040083A7CF
:101D2000071D8297B7E70400BC4B930500044DBF25
:101D300005491747FF1F232D27F383C7070032C626
:101D40002E8493F7F70FD5D3B7E4040083A7041DBF
:101D50007D141374F40F8297E37689FCB24599479A
:101D600003C61500E3F0C7FCFC4409061745FF1F36
:101D70001305C5F08297BC48930500081745FF1F5F
:101D8000034545EE829779BF1703FFFFE702E33172
:101D90001747FF1F130787EC4047184B1C40974617
:101DA000FF1F23A3F6EC6316E4001747FF1F232F42
:101DB000F7EA130584FE9790FFFFE78000AA03551A
:101DC00064FF9780FFFFE780807297A0FFFFE780A6
:101DD00060D01703FFFF6700832F1703FFFFE702A1
:101DE000C32C9747FF1F938767E7D84BDC4789C70A
:101DF00097000000E78080F985471747FF1F2329D8
:101E0000F7E69747FF1F9387E7D69C4393050002A9
:101E10001745FF1F034505E583C787031747FF1FC6
:101E2000230AF7E4B7E70400BC4B82971703FFFFD0
:101E30006700E3299747FF1F23A4A7E282801703C7
:101E4000FFFFE702E32437E404007C4CA14517457B
:101E5000FF1F034525E182977C48A1451745FF1FD9
:101E6000034545E09744FF1F938444DF8297DC4499
:101E700089EB97000000E78080D91703FFFF670018
:101E8000632403D567FF9780FFFFE7804066AA8938
:101E90006DD1D84891476310F7027C4C91451745A6
:101EA000FF1F034525DC82977C4891451745FF1F9E
:101EB000034545DB829703A9490103D409018947FA
:101EC000B7E904001747FF1F2324F7DA83A7091D8A
:101ED00021044204829783C784011715FF1F13054D
:101EE000256161191717FF1FA304F76083A7491C19
:101EF000418082979747FF1F238007D883A7C91C7B
:101F0000814609469375F40F4A85829711E99747F0
:101F1000FF1F83C7A7E689C79710FF1FE78020CA66
:101F2000B7E70400BC4F2146A1451745FF1F0345F5
:101F300065D3829799B71703FFFFE702031793F75B
:101F4000052001112E8481CF97000000E78020E951
:101F50001345042005611703FFFF6700431793F73C
:101F60000510A9CF9744FF1F938444CFDC48970006
:101F70000000E78020C11747FF1F1307A7BF1843C2
:101F800083C78401034787036318F700DC4489C7CC
:101F900097000000E78080DF85471747FF1F232950
:101FA000F7CCB7E70400BC4B930500021745FF1FB1
:101FB000034545CB82971345041069BF93F7050885
:101FC000BDC79747FF1F83C777CBE91719469745CA
:101FD000FF1F9385C5CA1305D10093F4F70F174966
:101FE000FF1F0349A9C997C00000E78040409397AD
:101FF0000401C1831747FF1F1307C7C8231DF10042
:10200000231CF1009747FF1F938747C53ACE3ACA72
:10201000D8432306010009CBDC43931589015408FA
:102020000D46E185680082971345040825B793F7AC
:102030002500A5C39747FF1F938747C2D84B894701
:102040006306F7029747FF1F83C787BE13F7270072
:1020500011EF918B99CFB7E70400BC4F1306000A2C
:1020600089451745FF1F0345E5BF829713452400A7
:10207000D5B59747FF1F9387E7AF9C4383C7870377
:102080001747FF1F2308F7BE97000000E78060DBBB
:10209000F1BF93F7050281CB97000000E78060DA7B
:1020A0001345040245BD93F7850081CB97000000DE
:1020B000E780E0D21345840071BD93F7150081CB12
:1020C00097000000E780A0B41345140061B593F7B2
:1020D000450081CB97000000E78060B313454400C2
:1020E00095BD93F7050495C39747FF1F83C707B7AF
:1020F00091CB97000000E780A0A491471747FF1FEE
:102100002328F7B613450404B1B593F7050101453B
:10211000E38207E49747FF1F938747B4D84B914763
:102120006310F7049747FF1F938787B09C4313D72B
:1021300027008583D98F858B91E7B7E7040083A7B4
:10214000071D8297B7E70400FC4F91451745FF1F15
:10215000034545B1829785471747FF1F232AF7B0EC
:1021600013450401C5BB9747FF1F2389A7C0828081
:102170001703FFFFE70263F39747FF1F23A607AE8E
:102180009747FF1F23A407AE85471744FF1F13047B
:10219000649E1747FF1F232DF7AC1C4083C787039E
:1021A0001747FF1F2308F7AC9790FFFFE780409386
:1021B00029C59717FF1F23A1A7341C40170500004E
:1021C0001305A5D783C787031747FF1F2304F7AA63
:1021D0001717FF1FA30EF7309747FF1FA38007A80D
:1021E000B7E7040083A7070882979747FF1F238B51
:1021F000A7A61703FFFF670083EDB7C7898E9387F4
:1022000067ED1717FF1F2329F72E45BF1747FF1F3D
:102210000347C7A4795555E79747FF1F938707A43E
:1022200003C7170005079746FF1FA389E6A203C748
:1022300017008D463377D7029746FF1FA380E6A28B
:1022400083C617001747FF1F1307C792184393F65B
:10225000F60FA9EE834787031747FF1F230CF7A04C
:1022600085471747FF1F230BF79E9747FF1F93874D
:10227000279C9C430145998BA9E71703FFFFE702C1
:10228000C3E237E404007C48C1451745FF1F0345FE
:10229000659D82973C4885451745FF1F0345859CF2
:1022A000829701451703FFFF670063E283C71700AA
:1022B00085466395F6008347970379BF8347A70355
:1022C00061BF82809747FF1F83C74799A1CF17033C
:1022D000FFFFE70283DD37E404009747FF1F238FEA
:1022E00007967C4885451745FF1F0345A5978297AC
:1022F0007C4C91451745FF1F0345C59682977C4846
:1023000091451745FF1F0345E59582973C48C14518
:102310001745FF1F03450595829701451703FFFFEA
:102320006700E3DA795582801703FFFFE702E3D7FE
:102330002A84035565FF9780FFFFE780401B97477E
:10234000FF1F9387A791D847BE841DEF9790FFFF8B
:10235000E78080779C48232004009DEB9747FF1F70
:1023600023A687909747FF1F23A08790B7E7040015
:10237000BC4B89451745FF1F0345C58E8297014514
:102380001703FFFF6700A3D4630A8700184375BFD4
:1023900080C39747FF1F23AB878CC9BF7955CDB743
:1023A0001703FFFFE70263D09747FF1F9387479DFF
:1023B00088432326050023240500510597A000002B
:1023C000E780C0331703FFFF670063D01703FFFFE9
:1023D000E702A3CD1744FF1F1304849A1C40411148
:1023E00099CF9C472302B5002AC61CC19700000064
:1023F000E78040FB1C409C4B99C3324582974101CA
:102400001703FFFF6700A3CC1703FFFFE702E3C931
:102410004111444D328532842EC69790FFFFE780EC
:10242000C0522AC422859790FFFFE780205403A85A
:102430004400630C0800B24583574400184022460C
:1024400083D54500AA862685029841011703FFFF20
:102450006700E3C71703FFFFE70223C5404D1DC810
:1024600008C097050000938565031305440197A0F4
:102470000000E78040169747FF1F938767909C43B3
:10248000014589E79747FF1F23AC878E1703FFFF9E
:102490006700E3C37D55DDBF1703FFFFE702E3C01D
:1024A000011168009305F00F02C602C802CA02CCEF
:1024B00002CE97000000E780A0F105611703FFFF3F
:1024C0006700E3C09747FF1F9387878B9C43D847DC
:1024D000A1679D076319F7021703FFFFE702E3BC3B
:1024E000011132859790FFFFE7802046230AA10063
:1024F0008145680097000000E78080ED05611703C3
:10250000FFFF6700C3BC82809747FF1F9387478701
:102510009C43D847A167938777036319F702170392
:10252000FFFFE70283B8011132859790FFFFE78034
:10253000C041230AA1008145680097000000E780A0
:1025400020E905611703FFFF670063B882809747A2
:10255000FF1F9387E7829C43D84795476316F7048C
:102560001703FFFFE70263B40111328532849790AD
:10257000FFFFE780803D230AA10022859790FFFF9F
:10258000E780C03E83574400231BA10081453ECC19
:102590001C4068003ECE97000000E78060E30561C4
:1025A0001703FFFF6700A3B28280930785FF8DC3E7
:1025B0008327C5FF91CFDC4B81CF1703FFFFE702D5
:1025C000C3AE032585FF82971703FFFF670023B083
:1025D00082801703FFFFE70243AD2A84328597907C
:1025E000FFFFE7808036BD4763EBA7001844937771
:1025F000F5000345B70041995D8DA305A7001703BA
:10260000FFFF6700C3AC1703FFFFE70203AA011136
:102610007C003ECAB70707003ECC7C003ECE5C4D36
:10262000A9C72A8413858700AE8497A00000E7809D
:10263000E0FCA1652A899D0548089770FFFFE780A7
:10264000603E9305803EB345B902480893F5F50F07
:102650009790FFFFE780C021014781465008A6857B
:1026600022859770FFFFE780406105611703FFFF38
:102670006700E3A51703FFFFE70223A3970000000D
:10268000E780A0F81703FFFF670063A41703FFFFAD
:10269000E702A3A101117C00AE843ECAA165B70781
:1026A00007002A843ECC48087C00938575033ECE03
:1026B0009770FFFFE78000371C44480883C5B700C8
:1026C000BD899790FFFFE780A01A50080147814617
:1026D000A68522859770FFFFE780205A05611703C2
:1026E000FFFF6700C39E1703FFFFE702039C2A84D6
:1026F000AE8497000000E78000EEA6852285970053
:102700000000E780E0F81703FFFF6700439C170312
:10271000FFFFE702839997000000E78060F7170347
:10272000FFFF6700C39A1703FFFFE702039803291F
:10273000C5014111630809022A843285B284979049
:10274000FFFFE78080202AC626859790FFFFE7805D
:10275000E021832749002A8691C7DC4781C7B2451B
:102760002285829741011703FFFF670043961703F5
:10277000FFFFE7028393444D91CC2A8432859790E2
:10278000FFFFE780A01EDC40AA8589C79C4799C34C
:10279000228582971703FFFF670063931703FFFFEC
:1027A000E702038F032AC5014111630D0A062E8932
:1027B000AA849545328532849770FFFFE780802692
:1027C000854522859790FFFFE7804004AA89CA8546
:1027D00022859790FFFFE780A00B83274A008DCBCF
:1027E000DC439DC722859790FFFFE780A0008327E9
:1027F0004A00104083564400DC437115A307A10032
:10280000B2961307F1004E86CA852685829701C5C8
:102810002380090001A88345F10022859790FFFFDE
:10282000E780C0FE41011703FFFF6700A38917037C
:10283000FFFFE702838765711C083EC2B70780016E
:102840003EC41C0832893EC62A84AE84970000002C
:10285000E780A0ED4A859790FFFFE780201183571E
:10286000A1008DC3AA855000228597000000E78053
:1028700020F3014781465000A68522859770FFFF0F
:10288000E780A03F59611703FFFF6700438417F3F8
:10289000FEFFE702E37F65711C088329C5013EC284
:1028A000B70780013EC41C082A84AE8432893EC624
:1028B00097000000E780E0EB638A09024A85979061
:1028C000FFFFE780A00A8357A100AA8585C35000B7
:1028D000228597000000E780A0EC01478146500068
:1028E000A68522859770FFFFE7802039596117F38D
:1028F000FEFF6700237D17F3FEFFE702037B657190
:102900001C083EC2B70780013EC42A841C083285D9
:102910003EC6AE849790FFFFE78040058357A10035
:102920008DC3AA855000228597000000E78040E70C
:10293000014781465000A68522859770FFFFE780FA
:10294000C033596117F3FEFF6700637817F3FEFF8A
:10295000E702A375444D81EC8347450093B7170008
:10296000B307F0403E8517F3FEFF67004376184536
:10297000FD576DDB97070000938747032A845CCBE4
:10298000970500009385A5C21385840097A00000D9
:10299000E78060C480C003474400814761F7173770
:1029A000FF1F2321973E7DBF17F3FEFFE702436E13
:1029B0008329C50141110329850081476387090ADD
:1029C0000324090191452A8A22859770FFFFE78039
:1029D0006005854522859790FFFFE78020E38945C4
:1029E000AA8A22859790FFFFE78040E2AA84977029
:1029F000FFFFE780400A83A749002A8B8DCB9C43C9
:102A00009DC722859790FFFFE780C0DE83A749001E
:102A1000A306A1001040835644009C431307D10035
:102A2000B296D6851306E1005285829709CD835769
:102A30000B002380F400A183A380F40023800A000C
:102A4000A306010039A88357E10022852380F40002
:102A50008345D100A183A380F4009790FFFFE78016
:102A6000E0DA8347D100B337F0000347B90092079B
:102A700001453D9BD98FA305F900410117F3FEFFE6
:102A80006700436417F3FEFFE702236241110DED77
:102A90009737FF1F9387072F804315C804401309FA
:102AA00084009DC95C4099C79C4B89C726852EC66A
:102AB0008297B2459307803EB385F5024A8597A079
:102AC0000000E78060C121A0404DAA8469F841015F
:102AD00017F3FEFF6700A35F4A8597A00000E78019
:102AE000E0C15C40EDD7DC4BFDD326858297C5B7AE
:102AF00017F3FEFFE702635B2A8432859790FFFF9E
:102B0000E780A0E4AA85228597000000E780C0F74F
:102B100017F3FEFF6700A35B17F3FEFFE702E3581E
:102B20002A84AE8497000000E780C0FCA685228539
:102B300097000000E78060AD17F3FEFF67002359A0
:102B400008413355B5000589828017F3FEFFE7027F
:102B5000C3551734FF1F1304E4241C5C0111231711
:102B600001008D83858BA303F1008327040B2318B9
:102B700001002319010003D7C7013ECA3C002314FA
:102B8000E1007D572315E1000357C4023ECC02CE7D
:102B90002316E1009770FFFFE78020CE8357E10105
:102BA000231EA10093F707E093E71710231FF100FE
:102BB0009737FF1F83C7A72195C305470145638A40
:102BC000E7008347840393E727001737FF1F230796
:102BD000F720056117F3FEFF6700634F814717F782
:102BE0000000130727E18546130671008545480854
:102BF00097900000E780408F69FD83478403F59B31
